:100000000C94C9230C94FA230C94FA230C94FA232D
:100010000C94FA230C94FA230C94FA230C94FA23EC
:100020000C94FA230C94FA230C94FA230C94FA23DC
:100030000C94FA230D94C4530C94FA230C94FA23D1
:100040000C94FA230C9487EF0C94FA230C94FA2363
:100050000C94FA230C94FA230C944EEC0D947A53DE
:100060000C94FA230C942B5F0C94215F0C94FA23CC
:100070000C94FA230C94FA230C94FA230C94FA238C
:100080000C94EA420C94FA230C94FA230C94FA236D
:100090000C94FA230C94FA230C94FA230C94FA236C
:1000A0000C94FA230C94FA230C94BC420C94FA237B
:1000B0000C94FA230C94FA230C94FA230C94FA234C
:1000C0000C94FA230C94FA230C94FA230C94FA233C
:1000D0000C94FA230C94FA230C94FA230C94FA232C
:1000E0000C94FA23084AD73B3BCE016E84BCBFFD7B
:1000F000C12F3D6C74319ABD56833DDA3D00C77FF8
:1001000011BED9E4BB4C3E916BAAAABE0000008090
:100110003F05A84CCDB2D44EB93836A9020C50B91F
:10012000918688083CA6AAAA2ABE000000803F004B
:100130000C94799C0D94DE4D0C947C9C0C94D15FB6
:100140000C94BBDB0C945B920C946AB20C94C1E0EF
:100150000C9455AD0D94D44D0C94659C0C94209A40
:100160000C94C5D40C94D0930C94A79A0C9480BF93
:100170000C94E4D40C940ECB0C94859C0C94C0A9E4
:100180000C9465920C9483A70C94B2290C94A6DD70
:100190000C94FCCA0C9408CB0C946B420C945C9AA3
:1001A0000C94A9940C9426CB0D94E84D0C94C19317
:1001B0000C94AFB80C94AE3B0C94D6260C94289AB1
:1001C0000C947D910C9444920C94829C0C944692D5
:1001D0000C94A5B80C94899B0C94C15F0C940C9161
:1001E0000C94BADB0C945E960C948DB10C94C5CB38
:1001F0000C9456920C945E900C94CADF0D949D4D15
:100200000D94F24D0C9484D40C9450990C94369027
:100210000C94FF230D94B14D0D94A74D0D94214DD9
:100220000C944C990C94CB9A0C941A920C944F9178
:100230000C94709C0C945C940C94EB9C0C94BE26D7
:100240000C9420CB0C94B4960C9427900C94FF99AA
:100250000C941F910C94C6920C94FDA70C94BAC6F2
:100260000C94A5900C9424970C94985F0D94054DD4
:100270000D946F4D0D941B4D0D94FB4C0C9458999F
:100280000C948A9C0C947F9C0C946C990C948E9A80
:100290000C9442DE0C9438910C944F900C94C09ABC
:1002A0000C94E89C0C94EA900C9405C10C9438DBF7
:1002B0000C94F0CA0C94F7DF0D94CE2E0C94858D1F
:1002C0000D94F54C0D94F24C0D94EE4C0C949D92C3
:1002D0000C94DECA0C940E900C94B8DF0C9436C2C9
:1002E0000D941F5E0C9492900C941FDF0C9425DEED
:1002F0000C94D1900C949B940C94E75F0C94EACAF4
:100300000C94A3940C94C9920C94BADE0D946A4D8B
:100310000C94DFAE0C9442920C94DBDE0C94609251
:100320000C940EDD0C9448990C94908D0C9414CB85
:100330000D94794D0C94B7920C9494910C9498BDB3
:100340000C9479900C94EF5F0C9411940D94D72D2C
:100350000C94F6CA0C94D55F0C94739C0C9465D4E1
:100360000D94624D0C94695F0C94C55F0C94B0962B
:100370000D94782D0C94DB290C94FC230C9489A407
:100380000C94F3D30C9419950C9412D40C94F9900A
:100390000C94759A0D94CF4C0D94D44C0C942392DC
:1003A0000D94254D0D94954D0C9460990C946D9B76
:1003B0000C94F58F0C9452960C94EA920C945192F2
:1003C0000C944D940D94BB4D0C9402CB0D948D4D1B
:1003D0000C94A7940D94CA4D0C94B65F0C949F4551
:1003E0000C9479240C94CC920C9455B00C949F945A
:1003F0000C9450420C941ACB0C94B8900C94A19489
:100400000C94E79E0C9486420C94A5940C946499E9
:100410000C9415CF0C94DC5F0C9479A70C94769C0B
:100420000C9468990C94BFAF0C9488A70C94929C80
:100430000C947F930C94679B0D94FC4D0C942F921D
:100440000C94BAA00C940ED50C9499BA0C943ADF83
:100450000C947E9B0C949D940D94715E0D94A52D2F
:100460000C948F9C0D94EA4C0C9454990C94A75FB7
:100470000C94F4B00C94AC960C948BCB0D940D4D65
:100480000C945C990C94628D0C94069D0D94E64C32
:100490000C947EA70C9466910D94094D0C94C7B8EA
:1004A0000C94BD5F0C94D0B50C9413C90C948C9C27
:1004B0000C94E4CA0C94E88D0D94834D0C94CF9267
:1004C0000D948F5E0D94174D0C94C5A10D94134D92
:1004D0000C9430AC0C94759B0C94CD5F0C94CF8D28
:1004E0000D94FF4C0C94A1420C94DBB30C94C95FA7
:1004F0000C943D2A0C9404B74E414E494E49545930
:10050000494E46CDCCCC3D0AD7233C17B7D13877DE
:10051000CC2B329595E6241FB14F0A0000204100F4
:1005200000C84200401C4620BCBE4CCA1B0E5AAE3E
:10053000C59D7400407A10F35A00A0724E1809004D
:1005400010A5D4E80000E87648170000E40B540238
:100550000000CA9A3B000000E1F505000080969873
:1005600000000040420F000000A0860100000010C3
:100570002700000000E80300000000640000000005
:10058000000A00000000000100000000002C76D8E6
:1005900088DC674F0823DFC1DFAE59E1B1B796E5CC
:1005A000E3E453C63AE651997696E8E6C28426EB30
:1005B000898C9B62ED407C6FFCEFBC9C9F40F2BA43
:1005C000A56FA5F490055A2AF75C936B6CF9676DDB
:1005D000C11BFCE0E40D47FEF520E6B500D0ED9030
:1005E0002E0300943577050080841E080000204EFD
:1005F0000A000000C80C333333330F986E12831196
:1006000041EF8D2114893BE65516CFFEE6DB18D16C
:10061000844B381BF77C1D901DA4BBE4242032843E
:10062000725E228100C9F124ECA1E53D27434F4DC4
:100630004D554E49434154494F4E0044525952552D
:100640004E004552524F525300494E464F004543CB
:10065000484F004572726F722077726974696E67D5
:1006600020746F20454550524F4D210A0053544F7E
:10067000505045442E20005072696E74657220738C
:10068000746F707065642064756520746F20657286
:10069000726F72732E2046697820746865206572C7
:1006A000726F7220616E6420757365204D3939391F
:1006B00020746F20726573746172742E20285465E3
:1006C0006D706572617475726520697320726573EF
:1006D00065742E2053657420697420616674657298
:1006E0002072657374617274696E67290A004E6FB7
:1006F00020436865636B73756D2077697468206C3F
:10070000696E65206E756D6265722C204C61737424
:10071000204C696E653A20004E6F20436865636B1C
:1007200073756D2077697468206C696E65206E75CD
:100730006D6265722C204C617374204C696E653A51
:100740002000636865636B73756D206D69736D61FF
:100750007463682C204C617374204C696E653A2078
:10076000004C696E65204E756D626572206973205C
:100770006E6F74204C617374204C696E65204E75E9
:100780006D6265722B312C204C617374204C696E44
:10079000653A20004D3131300053657269616C203B
:1007A000737461747573206D69736D617463680A25
:1007B00000776169740A00534420726561642065A2
:1007C00072726F720A00486F74656E642049646CBF
:1007D000652054696D656F757400486F74656E644B
:1007E0002049646C652054696D656F75740A002139
:1007F00021204B494C4C20636175736564206279FC
:10080000204B494C4C20627574746F6E2F70696E6A
:100810000A002121204B494C4C20636175736564AB
:1008200020627920746F6F206D75636820696E6136
:1008300063746976652074696D65202D2063757217
:1008400072656E7420636F6D6D616E643A20007026
:1008500061757365004D363030002066696C616DDE
:10086000656E745F72756E6F7574200066696C6179
:100870006D656E745F72756E6F7574205400466995
:100880006C616D656E7452756E6F75742054004D99
:10089000656469612052656D6F766564004D6564BD
:1008A000696120496E736572746564004D31303042
:1008B000305300627573793A2070617573656420F6
:1008C000666F7220696E7075740A00627573793A8A
:1008D0002070617573656420666F72207573657230
:1008E0000A00627573793A2070726F636573736979
:1008F0006E670A00506C656173652052657365749C
:10090000005052494E5445522048414C54454400F1
:1009100025533A20255300706F7765726F66660025
:100920004B494C4C45442E20005072696E746572E0
:100930002068616C7465642E206B696C6C282920BA
:1009400063616C6C6564210A0053544F50504544F8
:100950002E20005072696E7465722073746F70700F
:1009600065642064756520746F206572726F7273A0
:100970002E2046697820746865206572726F722037
:10098000616E6420757365204D39393920746F208C
:10099000726573746172742E202854656D7065726F
:1009A00061747572652069732072657365742E2099
:1009B0005365742069742061667465722072657372
:1009C00074617274696E67290A006563686F3A0022
:1009D0004572726F723A0042696C696E656172208D
:1009E0004C6576656C696E6720477269643A0A00E7
:1009F00021212053544F502063616C6C6564206248
:100A0000656361757365206F6620424C546F756332
:100A100068206572726F72202D2072657374617226
:100A2000742077697468204D3939390A00212120F2
:100A300053544F502063616C6C6564206265636140
:100A4000757365206F6620424C546F75636820652E
:100A500072726F72202D20726573746172742077C8
:100A6000697468204D3939390A005072696E7469A9
:100A70006E67204F626A6563740025532025690004
:100A80002F2F616374696F6E3A0073746172740022
:100A900070726F6D70745F00656E6400486F74658E
:100AA0006E6420746F6F20636F6C640A0053656E10
:100AB00064204D31303820746F20726573756D6518
:100AC0000A00496E736572742066696C616D656EAB
:100AD0007420616E642073656E64204D3130380A75
:100AE0000052656865617420446F6E6500526568E8
:100AF000656174696E672E2E2E005265686561749B
:100B0000004865617465722054696D656F75740085
:100B100053656E64204D31303820746F20686561F4
:100B200074206E6F7A7A6C650A004E6F7A7A6C6503
:100B3000205061726B65640070617573656400506C
:100B40006175736500726573756D656400526573D8
:100B5000756D696E67004732362043616E63656C60
:100B60006564004732362048656174696E67204EBF
:100B70006F7A7A6C65004732362048656174696E19
:100B800067204265640057616974696E6720666F0B
:100B900072206865617475702E0A00466978656414
:100BA000204C656E677468205072696D6500446FF3
:100BB0006E65205072696D696E67004D616E75617A
:100BC0006C207072696D696E672E2E2E004C656107
:100BD00076696E6720473236003F537065636966F9
:100BE00069656420582C5920636F6F7264696E6167
:100BF0007465206F7574206F6620626F756E647304
:100C00002E0A003F28522965706561742076616C58
:100C10007565206E6F7420706C61757369626C65A8
:100C20003B206D757374206265206174206C656172
:100C3000737420312E0A003F5370656369666965DD
:100C400064206E6F7A7A6C652074656D7065726170
:100C500074757265206E6F7420706C617573696253
:100C60006C652E0A003F5370656369666965642090
:100C700066696C616D656E742073697A65206E6F4C
:100C80007420706C61757369626C652E0A003F5345
:100C90007065636966696564207072696D65206C52
:100CA000656E677468206E6F7420706C617573690F
:100CB000626C652E0A003F537065636966696564FE
:100CC000206E6F7A7A6C652073697A65206E6F7416
:100CD00020706C61757369626C652E0A003F526505
:100CE0007472616374696F6E204D756C7469706C99
:100CF000696572206D757374206265207370656319
:100D000069666965642E0A003F53706563696669A8
:100D100065642052657472616374696F6E204D75ED
:100D20006C7469706C696572206E6F7420706C6190
:100D3000757369626C652E0A003F5370656369665E
:100D4000696564206C61796572206865696768749B
:100D5000206E6F7420706C61757369626C652E0A09
:100D60000043292E0A003F53706563696669656414
:100D7000206265642074656D70657261747572655A
:100D8000206E6F7420706C61757369626C652028C9
:100D900034302D00473236207374617274696E6787
:100DA0002E2E2E0A004F46460A00466164652048F2
:100DB00065696768742000426564204C6576656CDF
:100DC000696E6720004661696C656420746F2065F8
:100DD0006E61626C6520426564204C6576656C6965
:100DE0006E670A00496E76616C6964206D65736890
:100DF0002E0A0050726F62696E6720506F696E74C0
:100E00000025532025692F2569002E0A002F005048
:100E1000726F62696E67206D65736820706F696EAE
:100E2000742000202844525952554E290047323927
:100E3000204175746F20426564204C6576656C694D
:100E40006E67003F20284C2C522C462C4229206FE4
:100E50007574206F6620626F756E64732E0A003F92
:100E60002856296572626F7365206C6576656C2003
:100E7000696D706C61757369626C652028302D3402
:100E8000292E0A00426164205A2076616C75650A39
:100E9000004E6F2062696C696E65617220677269CD
:100EA000640A00446576696174696F6E0025533A7F
:100EB0002025730046696E6973686564210A003AEB
:100EC000207A3A2000206F662000476F696E672005
:100ED000746F3A20580043570A00206469723A0040
:100EE00020616E676C653A005374617274207261A0
:100EF000646975733A004D343820506F696E740020
:100F000025533A2025642F256400506F7369746956
:100F10006F6E696E67207468652070726F62652EEF
:100F20002E2E0A003F4C656773206F66206D6F762A
:100F3000656D656E7420696D706C61757369626C46
:100F4000652028302D3135292E0A003F2028582CC5
:100F50005929206F7574206F6620626F756E6473F7
:100F60002E0A0050726F6265206F7574206F6620C4
:100F7000626F756E6473003F53616D706C652073B2
:100F8000697A65206E6F7420706C61757369626C2C
:100F9000652028342D3530292E0A004D3438205A4A
:100FA0002D50726F6265205265706561746162696F
:100FB0006C69747920546573740A003F285629655A
:100FC00072626F7365206C6576656C20696D706CFC
:100FD00061757369626C652028302D34292E0A00F2
:100FE0005374616E646172642044657669617469EA
:100FF0006F6E3A20002052616E67653A2000204DE6
:1010000061783A2000204D696E3A200020536967CC
:101010006D613A20004D65616E3A2000205200411A
:101020006363656C65726174696F6E3A2050005736
:1010300041524E494E4721204C6F77205A204A6535
:10104000726B206D6179206C65616420746F20750E
:101050006E77616E746564207061757365732E0AB6
:10106000004F4646004F4E0020204D61783A200048
:10107000200020204D696E3A2000536F6674206571
:101080006E6473746F70733A20004D3234205325B0
:101090006C642054256C64004739322E3920452574
:1010A0007300473120462564004739322E39205AD3
:1010B0002573004731205A30204632303000473106
:1010C0002058257320592573204633303030004D89
:1010D00034323020532569205A2573004D31303683
:1010E0002050256920532569004D32303020442599
:1010F000730047323852305859004739322E392060
:101100004530205A300A47315A2573004D31303965
:1011100020532569004D31393020532569004D3465
:101120003230205330205A300020496E76616C698D
:1011300064206578747275646572200047322F47A9
:10114000332062616420706172616D6574657273D1
:101150000A00536C6565702E2E2E005A2050726F57
:1011600062652050617374204265640A005A205001
:10117000726F62652050617374204265640047326B
:10118000384C30004D3131372050726F6265206627
:1011900061696C65642E0A4732380A0070726F62AA
:1011A000655F7265776970650047323920526574F2
:1011B0007279696E670050726F62696E672046616E
:1011C000696C6564004D31313720426564206C657F
:1011D00076656C696E67206661696C65642E0A4786
:1011E00030205A31300A4D333030205032352053C0
:1011F0003838300A4D333030205035302053300AE3
:101200004D3330302050323520533838300A4D338A
:101210003030205035302053300A4D33303020509C
:10122000323520533838300A4D3330302050353085
:101230002053300A47342053310070726F62655F6B
:101240006661696C6564004D313137204265642008
:101250006C6576656C696E6720646F6E652E002024
:101260005A3A200020593A200042656420583A201A
:10127000004D65736820706F696E74206F757420FF
:101280006F662072616E67650A004D302053746F7F
:1012900070004D312053746F7000436C69636B2094
:1012A000746F20526573756D652E2E2E004E6F2063
:1012B0004D6F76652E00456E642066696C65206C06
:1012C0006973740A00426567696E2066696C6520FF
:1012D0006C6973740A004E6F206D656469610A0061
:1012E000526573756D696E6720534400286E6F20D8
:1012F00066696C65290043757272656E7420666953
:101300006C653A20005072696E742074696D653A9C
:1013100020000A53746174733A2046696C616D65EC
:101320006E7420757365643A20002C204C6F6E67D4
:10133000657374206A6F623A2000546F74616C2088
:1013400074696D653A200053746174733A20002CFF
:10135000204661696C65643A20002C2046696E69FC
:10136000736865643A20005072696E74733A2000A5
:1013700053746174733A2000436F6F6C696E672E0B
:101380002E2E0048656174696E672E2E2E00452052
:101390002553006F6B006F6666004E0649064206D5
:1013A0003B062D0644454255473A004D3131332026
:1013B000530042656420436F6F6C696E672E2E2E5A
:1013C000004265642048656174696E672E2E2E00A8
:1013D000544D334420435231305632204F46462E2E
:1013E000002F2F004D31343520533C696E646578F1
:1013F0003E206F7574206F662072616E67652028CD
:10140000302D31290A004D32303620580046523AEC
:101410000020466C6F773A20003A20002053657216
:10142000766F2000206F7574206F662072616E6782
:10143000650A00536572766F200020643A002069C7
:101440003A0020703A00496E76616C6964206578D4
:101450007472756465720A0020643A0020693A006B
:1014600020703A0064697300656E0043290A0061C8
:10147000626C656420286D696E2074656D70200053
:10148000436F6C6420657874727564657320617253
:1014900065200046696C616D656E742072756E6FB3
:1014A00075742064697374616E636520286D6D299D
:1014B0003A200046696C616D656E742072756E6FBE
:1014C000757420004D34323120696E636F7272651D
:1014D000637420706172616D6574657220757361EB
:1014E00067650A004D65736820706F696E74206FC0
:1014F0007574206F662072616E67650A004F6666BC
:1015000073657473204170706C6965640045727214
:101510003A20546F6F206661722100546F6F20660D
:1015200061722066726F6D207265666572656E63AA
:101530006520706F696E740A00454550524F4D200A
:101540004F4B0A00506F7765722D6C6F737320726A
:1015500065636F7665727920004D383400446F6E94
:1015600065207072696E74696E672066696C650AC1
:10157000004D3737004D3331004361703A004D451F
:1015800041545041434B00434F4F4C45525F5445EB
:101590004D5045524154555245004348414D4245F6
:1015A000525F54454D5045524154555245004241B9
:1015B00042595354455050494E47004152435300FD
:1015C0004D4F54494F4E5F4D4F444553005448458D
:1015D000524D414C5F50524F54454354494F4E0079
:1015E0004C4F4E475F46494C454E414D4500415595
:1015F000544F5245504F52545F53445F53544154DB
:1016000055530053445F5752495445005245504585
:101610004154005344434152440050524F4D5054A2
:101620005F535550504F525400454D455247454E1B
:1016300043595F50415253455200434153455F4C1B
:10164000494748545F4252494748544E4553530016
:10165000544F47474C455F4C494748545300534FFC
:101660004654574152455F504F57455200425549E5
:101670004C445F50455243454E54004C4556454CF2
:10168000494E475F44415441005A5F50524F4245D2
:101690000052554E4F5554004155544F4C455645F8
:1016A0004C005052494E545F4A4F420050524F47EF
:1016B00052455353004155544F5245504F52545F79
:1016C00054454D5000564F4C554D455452494300DA
:1016D000454550524F4D0042494E4152595F46498F
:1016E0004C455F5452414E53464552005345524972
:1016F000414C5F584F4E5F584F4646004649524D49
:10170000574152455F4E414D453A4D61726C696E8D
:1017100020322E302E375F4457372E3320544D332E
:10172000442053454D4442422028417072203234B7
:1017300020323032312032313A34363A35382920AD
:10174000534F555243455F434F44455F55524C3AC2
:1017500068747470733A2F2F6769746875622E63AA
:101760006F6D2F496E73616E6974794175746F6D19
:101770006174696F6E2F4D61726C696E2F74726542
:10178000652F437265616C6974794477696E5F3265
:101790002E302050524F544F434F4C5F56455253BA
:1017A000494F4E3A312E30204D414348494E455F16
:1017B000545950453A544D334420435231305632F7
:1017C0002045585452554445525F434F554E543A64
:1017D0003120555549443A63656465326132662D5E
:1017E000343161322D343734382D396231322D6342
:1017F00035356336326633363766660A0050726FA7
:101800006265204F6666736574205A0050726F627D
:1018100065204F6666736574205A00290A0020749B
:101820006F20003F5A206F7574206F662072616EC2
:101830006765202800290A0020746F20003F592086
:101840006F7574206F662072616E676520282D00A9
:10185000290A0020746F20003F58206F7574206F94
:10186000662072616E676520282D0050726F626578
:10187000204F666673657420580043616E6E6F7406
:10188000206F70656E20737562646972200025692F
:10189000730025696D202569730025696820256915
:1018A0006D202569730025696420256968202569F4
:1018B0006D202569730025697920256964202569D3
:1018C000682025696D202569730023646566696E4B
:1018D000652044454641554C545F00626564004BA9
:1018E0006420004B6920004B702000504944204187
:1018F00075746F74756E652066696E69736865646A
:10190000212050757420746865206C617374204BBD
:10191000702C204B6920616E64204B6420636F6ED5
:101920007374616E74732066726F6D2062656C6F84
:101930007720696E746F20436F6E66696775726198
:1019400074696F6E2E680A00504944204175746FA7
:1019500074756E65206661696C6564212074696DBB
:10196000656F75740A00504944204175746F747531
:101970006E65206661696C6564212054656D7065D3
:1019800072617475726520746F6F20686967680A88
:1019900000204B643A2000204B693A2000204B7015
:1019A0003A200020436C61737369632050494420DE
:1019B0000A00204E6F206F76657273686F6F740A2D
:1019C000002054753A2000204B753A2000206D61AC
:1019D000783A2000206D696E3A200020643A200099
:1019E00020626961733A2000504944204175746F48
:1019F00074756E652073746172740A0050494420D6
:101A00004175746F74756E65206661696C656421DB
:101A10002054656D706572617475726520746F6FA6
:101A200020686967680A00504944204175746F74E2
:101A3000756E6500504944204175746F74756E650C
:101A4000206661696C65642120426164206865617B
:101A50007465722069640A004572723A2075746672
:101A60003820666F6E74206E6F7420696E697469B9
:101A7000616C697A65642E004572723A20757466ED
:101A80003820666F6E74206E6F7420696E69746999
:101A9000616C697A65642E004572723A20757466CD
:101AA0003820666F6E74206E6F7420696E69746979
:101AB000616C697A65642E00000C0F00FE07022538
:101AC00003BB017FFE08FE08FE0508080600004073
:101AD000F0C88888987810050808060000C0F888C3
:101AE00088888888F80505050600012030F8302030
:101AF0000508080600002070F820202020E00509D5
:101B0000090600FF2070A8A8B8888870200705057E
:101B1000070001D86C366CD80509090600FFF8A843
:101B20008888888888A8F8050A0A0600FE20505090
:101B3000505088A8A8887003030306000340A04003
:101B4000FFFFFFFFFFFFFFFFFFFFFFFFFFFFFFFFA5
:101B5000FFFFFFFFFFFF0000000605FF010707066C
:101B6000020080808080800080030303060105A0BE
:101B7000A0A005060606000050F85050F8500509D0
:101B8000090600FF2070A8A07028A870200507078C
:101B9000060000C8C81020409898050707060000F6
:101BA00040A0A040A8906801030306020580808041
:101BB0000309090601FF2040408080804040200347
:101BC00009090601FF804040202020404080050791
:101BD0000706000020A8702070A820050505060053
:101BE000012020F820200203030601FFC0408005E9
:101BF0000101060003F8020202060100C0C0050749
:101C00000706000008101020404080050707060066
:101C100000708898A8C8887003070706010040C0B4
:101C200040404040E005070706000070880810208B
:101C300040F8050707060000F8081030088870050E
:101C4000070706000010305090F81010050707062F
:101C50000000F880F00808887005070706000030CB
:101C60004080F0888870050707060000F80810100B
:101C7000202020050707060000708888708888707B
:101C800005070706000070888878081060020505BF
:101C9000060100C0C000C0C00206060601FFC0C0A9
:101CA00000C040800305050601012040804020055A
:101CB0000303060002F800F8030505060101804051
:101CC00020408005070706000070881020200020B3
:101CD0000507070600007088B8A8B88070050707D8
:101CE000060000708888F8888888050707060000C5
:101CF000F04848704848F0050707060000708880E3
:101D000080808870050707060000F048484848486A
:101D1000F0050707060000F88080F08080F80507CE
:101D200007060000F88080F0808080050707060025
:101D300000708880809888700507070600008888F2
:101D400088F8888888030707060100E04040404083
:101D500040E00507070600003810101010906005DD
:101D600007070600008890A0C0A090880507070616
:101D70000000808080808080F805070706000088CA
:101D8000D8A8888888880507070600008888C8A81A
:101D900098888805070706000070888888888870FA
:101DA000050707060000F08888F080808005070797
:101DB00006000070888888A890680507070600005C
:101DC000F08888F0A09088050707060000708880DA
:101DD00070088870050707060000F82020202020E2
:101DE000200507070600008888888888887005070E
:101DF00007060000888888885050200507070600DD
:101E00000088888888A8A8500507070600008888E9
:101E10005020508888050707060000888850202039
:101E20002020050707060000F80810204080F8036E
:101E300009090601FFE080808080808080E005073E
:101E40000706000080404020101008030909060121
:101E5000FFE020202020202020E0050303060005CD
:101E60002050880501010600FEF803030306010562
:101E70008040200505050600007008788878050771
:101E8000070600008080F0888888F00505050600B8
:101E900000708080887005070706000008087888B1
:101EA0008888780505050600007088F080700507B1
:101EB00007060000304840E04040400507070600A4
:101EC000FE70888888780870050707060000808003
:101ED000F0888888880307070601004000C040405A
:101EE00040E00409090601FE1000301010101090A7
:101EF0006005070706000080808890E0908803074F
:101F000007060100C04040404040E00505050600CE
:101F100000D0A8A8A8A8050505060000B0C88888B4
:101F20008805050506000070888888700507070683
:101F300000FEF0888888F080800507070600FE789C
:101F4000888888780808050505060000B0C88080E4
:101F50008005050506000078807008F00507070673
:101F600000002020F8202020180505050600008824
:101F7000888898680505050600008888885020052F
:101F800005050600008888A8A8500505050600007C
:101F900088502050880507070600FE888888502052
:101FA0004080050505060000F8102040F8030909E7
:101FB0000601FF20404040804040402001090906C2
:101FC00002FF808080808080808080030909060174
:101FD000FF8040404020404040800503030600024F
:101FE00048A890FF554E4C4F41442046494C414D26
:101FF000454E54004C4F41442046494C414D454EBE
:10200000540046494C414D454E54204348414E47AB
:10201000450042656400456E636C6F7375726500C0
:102020002568753A25303268750025303268753A72
:10203000253032687500202020202020200020201C
:102040002020001FE0201020102010102010202041
:1020500010201030300840048003001FE03FF03FA4
:10206000F03FF01FE01FE03FF03FF03FF00FC007F0
:102070008003003FFFF038007030FC3020FC10205F
:1020800078102030102C00D02E31D02F7BD02F7B19
:10209000D02E31D02C00D020301020781020FC1011
:1020A00030FC303800703FFFF03FFFF038007031F7
:1020B00086302387102787902F87D02F03D020309A
:1020C000102078102078102030102F03D02F87D0C8
:1020D0002787902387103186303800703FFFF01F2C
:1020E000FFF81FFFF8041040020820020820041027
:1020F000400820801041001041000820800410405A
:102100000000001FFFF81FFFF8FFFFFF8000018E97
:1021100000E19F01F19381399F81F99F81F99FB976
:10212000F98F28F18038018000019FFFF99174999F
:102130009B06A99B54A99B56A99B54999FFFF9FF05
:10214000FFFF6E6F74696669636174696F6E20006A
:1021500063616E63656C005072696E742041626FDA
:1021600072746564004469736D6973730055492026
:1021700041626F72746564004D323520500A4D32F1
:102180003400526573756D65005549205061757353
:10219000650050617573696E672E2E2E007265732F
:1021A000756D65004D32340000FE0003FF8007C7E7
:1021B000C00701E00000E00000F0000070040070C3
:1021C0000E00701F00703F80F00E00E00F01E0076E
:1021D000C7C003FF8000FE0000FE0003FF8007C7AA
:1021E000C00F01E00E00E03F80F01F00700E007095
:1021F0000400700000700000F00000E00701E0073C
:10220000C7C003FF8000FE000E000E000E000E008F
:102210000E000E000E000E007FC03F801F000E005B
:10222000040004000E001F003F807FC00E000E005F
:102230000E000E000E000E000E000E00FFFFFF7FCE
:1022400080FFC0FFC0FFC07F807F80FFC0FFC0FF56
:10225000C03F001E000C0050726F6265205A204F74
:1022600066667365740052756E6F75742044697389
:1022700074206D6D004C6F6164206D6D00556E6C47
:102280006F6164206D6D0046696C2E204469612E7B
:10229000004520696E206D6D5E33004D3330332074
:1022A0005531204525692053256900504944204176
:1022B00075746F74756E65202A005049442D442052
:1022C0002A005049442D49202A005049442D5020CD
:1022D0002A0020082046616374002008204D6178A0
:1022E000002008204D696E004F6666004F6E004169
:1022F00075746F74656D70005654726176204D6907
:102300006E00566D696E00566D6178204500566D01
:102310006178205A00566D6178205900566D6178B9
:10232000205800416D6178204500416D6178205A48
:1023300000416D6178205900416D6178205800415D
:102340002D54726176656C00412D52657472616323
:102350007400416363656C0056652D4A65726B00BD
:10236000565A2D4A65726B0056592D4A65726B009C
:1023700056582D4A65726B0050726F6265205A2064
:102380004F66667365740050726F62652059204F06
:1023900066667365740050726F62652058204F66E0
:1023A0006673657400452073746570732F6D6D00DE
:1023B0005A2053746570732F6D6D005920537465E6
:1023C00070732F6D6D00582053746570732F6D6D91
:1023D00000416476616E6365642053657474696E50
:1023E0006773003F0043616E63656C00496E6974FA
:1023F000004D34323800496E697469616C697A65E0
:1024000020454550524F4D0046696C616D656E74B4
:102410000054656D70657261747572650053746502
:1024200070732F6D6D0050726F6265204F6666731A
:10243000657473004A65726B00416363656C657215
:102440006174696F6E0056656C6F636974790053CF
:10245000657420486F6D65204F6666736574730000
:10246000436F6E66696775726174696F6E003F00D5
:102470004E65787420506F696E7400446F6E65000D
:102480004E65787400486F6D696E672058595A0020
:102490003F0043616E63656C204F626A6563740040
:1024A0004E4F005945530043616E63656C204F6287
:1024B0006A656374203D004D61696E0053746F77E7
:1024C000004465706C6F790053656C662D546573BC
:1024D000740053572D4D6F64650052657365740029
:1024E000426564004E6F7A7A6C650046616E2053D7
:1024F0007065656400436F6E6669677572617469C3
:102500006F6E004C6F61642053657474696E6773FD
:1025100000526573746F72652044656661756C74F2
:10252000730053746F72652053657474696E6773BA
:102530000050726568656174202420436F6E6600E8
:10254000506F776572204F7574616765004F6666DE
:10255000004F6E0052756E6F75742053656E736F09
:102560007200424C546F7563680050726F62652050
:102570005A204F666673657400416476616E6365C8
:10258000642053657474696E6773004D61696E00F1
:102590004D37303220542564004D363030204230E3
:1025A00020542564004D373032203B2564004D37E0
:1025B000303120542564004D373032004D373031F2
:1025C000004D363030204230004D61696E004F665C
:1025D00066004F6E0052756E6F75742053656E7392
:1025E0006F72005075726765206D6F726500436F82
:1025F0006E74696E756500524553554D45204F50B8
:1026000054494F4E533A005052494E542050415570
:102610005345440020204E6F7A7A6C653A20005072
:1026200061726B696E672E2E2E000000576169740F
:1026300020666F720066696C616D656E74206368F8
:10264000616E676500746F20737461727400576106
:10265000697420666F720066696C616D656E7420C6
:10266000756E6C6F616400004E6F7A7A6C652068DD
:10267000656174696E6700506C6561736520776190
:1026800069742E2E2E00005072657373206275746B
:10269000746F6E00746F2068656174206E6F7A7A53
:1026A0006C650000496E736572742066696C616DBB
:1026B000656E7400616E642070726573732062755C
:1026C00074746F6E00746F20636F6E74696E7565DD
:1026D000005761697420666F720066696C616D6590
:1026E0006E74206C6F6164000050726573732042D9
:1026F0007574746F6E00746F20726573756D6520EC
:102700007072696E7400005761697420666F722080
:102710007072696E7400746F20726573756D652ECA
:102720002E2E00005761697420666F720066696C16
:10273000616D656E7420707572676500003E2000E3
:10274000256C642E25696D00457874727564656426
:1027500020546F74616C003E20004C6F6E6765738F
:1027600074204A6F622054696D65003E2000546FEA
:1027700074616C205072696E742054696D650043F9
:102780006F6D706C65746564003A20005072696EFC
:102790007420436F756E74003A2000313530003577
:1027A000004245443A204154432031303447542DAF
:1027B000320052756E617761792057617463683AAF
:1027C000204F4E004D61782054656D7000343530D7
:1027D000004D696E2054656D7000350045313A201A
:1027E000536C696365456E6720343530C2B0430071
:1027F0005053550047656E657269630050726F747F
:102800006F636F6C00312E300042617564003235A9
:102810003030303000437265616C69747933442024
:1028200052414D50530042696C696E656172204C93
:102830006576656C696E670045787472756465725B
:102840007300310074696E796D616368696E6573D8
:1028500033642E636F6D00544D3344204352313046
:10286000563200323032312D30342D313800322E94
:10287000302E375F4457372E33004D61726C696ECE
:10288000005072696E7465722053746174730054E1
:102890006865726D6973746F727300426F61726400
:1028A00020496E666F005072696E74657220496EC1
:1028B000666F004D61696E004D31303030005374E9
:1028C0006F70205072696E7400526573756D65206B
:1028D0005072696E7400506F776572204F75746125
:1028E0006765004D3139305335350A4732380A476C
:1028F00032390A4D3430300A4D31303453323135AB
:102900000A4732380A4D313039533231350A4D34A5
:10291000323053310A473158313030593130304636
:10292000353030300A47315A300A4D3530300A4D93
:1029300031313720536574205A204F6666736574B1
:10294000004D313036533132380A4D33303343384D
:10295000533231354530550A4D3530300A4D31311D
:1029600037205049442054756E6520446F6E6500D1
:102970004D3139305335350A4D31303453323135DC
:102980000A4732380A4732394C310A473120583128
:1029900030305931303046353030300A47315A30D6
:1029A000004D3530300A4D3131372053657474692C
:1029B0006E67732053746F72656400507265702087
:1029C000666F72205A2041646A75737400504944DE
:1029D0002054756E650053746F726520536574746E
:1029E000696E6773005365747570004D61696E00A0
:1029F0003F004261636B0053746F70005072696EE8
:102A0000742066726F6D204D656469610043686172
:102A10006E6765204D65646961004D323100416229
:102A20006F7574205072696E746572004368616ED0
:102A300067652046696C616D656E74004C657665EE
:102A40006C696E6720546F6F6C7300436F6E6669BC
:102A50006775726174696F6E0054656D706572613F
:102A600074757265004D6F74696F6E00486F737492
:102A700020537461727400526573756D65205072D5
:102A8000696E74004E6F204D656469610043616E2C
:102A900063656C204F626A6563740054756E6500EF
:102AA00053746F70205072696E7400506175736555
:102AB000205072696E7400496E666F2053637265B0
:102AC000656E003F005374617274205072696E74B9
:102AD0000043616E63656C005072696E74004361FF
:102AE0006E6E6F7420656E746572207375626469B2
:102AF000723A2000022E2E004D61696E00210048BE
:102B00006F74656E6420746F6F20636F6C64004235
:102B100061636B0050726F6365656400536F667428
:102B200020456E6473746F7073004D6F74696F6EBF
:102B30000044697361626C652053746570706572DE
:102B400073004D3834004D34382050726F62652068
:102B500054657374004732384F0A4D343820503171
:102B600030004C6576656C20436F726E6572730041
:102B70004661646520486569676874004F66660051
:102B80004F6E00426564204C6576656C696E670027
:102B90004C6576656C20426564004732394E0048CA
:102BA0006F6D65205A004732385A00486F6D6520B6
:102BB00059004732385900486F6D65205800473238
:102BC0003858004175746F20486F6D650047323882
:102BD000004D61696E005072656865617420242043
:102BE000456E6400507265686561742024204265FA
:102BF000640054656D706572617475726500436F31
:102C00006F6C646F776E0050726568656174202424
:102C10000046616E205370656564207E00426564E5
:102C2000004E6F7A7A6C65004D61696E0050726F6C
:102C30006265205A204F666673657400466C6F7734
:102C40000046616E205370656564207E00426564B5
:102C5000004E6F7A7A6C65005370656564004D6153
:102C6000696E00486F6D696E67204661696C6564C6
:102C7000006F70656E005452494747455245440005
:102C80003A200066696C616D656E74007A5F6D69EB
:102C90006E00795F6D696E00785F6D696E005265D8
:102CA000706F7274696E6720656E6473746F7020E4
:102CB0007374617475730A0020746F6F206C6F6E8B
:102CC0006720657874727573696F6E2070726576AF
:102CD000656E7465640A0020636F6C6420657874A7
:102CE000727573696F6E2070726576656E74656457
:102CF0000A00486F6D65202573257325732046698A
:102D0000727374005761726E696E673A20486F6D16
:102D1000696E672042756D702044697669736F72C1
:102D2000203C20310A0002020400000000000000E4
:102D3000000000000000809D4300009B430000C88D
:102D400043000000410000004100000040FFFFFF81
:102D500000000001000000010000800055555500F2
:102D60000000400033333300AAAA2A00499224000D
:102D700000002000C7711C0099991900D145170067
:102D8000555515003BB113002449120011111100D3
:102D9000000010000F0F0F00E3380E0043790D0004
:102DA000CCCC0C00C3300C00E8A20B0064210B005B
:102DB000AAAA0A00703D0A009DD80900427B0900BA
:102DC00092240900DCD3080088880800104208001B
:102DD00000000800F0C10700878707007550070052
:102DE000711C07003EEB0600A1BC060069900600BE
:102DF00066660600703E06006118060017F40500BE
:102E000074D105005BB00500B29005006272050048
:102E10005555050078390500B81E05000505050063
:102E20004EEC040087D40400A1BD040090A7040068
:102E300049920400C17D0400EE690400C7560400F5
:102E4000444404005C3204000821040041100400E2
:102E5000000004003FF00300F8E0030026D2030066
:102E6000C3C30300CCB503003AA803000A9B0300C8
:102E7000388E0300C08103009F750300D0690300F2
:102E8000505E03001D53030034480300913D0300CE
:102E90003333030016290300381F0300971503007E
:102EA000300C0300030303000BFA020049F1020097
:102EB000BAE802005CE002002DD802002DD002002A
:102EC00059C80200B0C0020031B90200DAB10200F4
:102ED000AAAA0200A0A30200BC9C0200FA9502006C
:102EE0005C8F0200DF88020082820200457C0200C3
:102EF0002776020027700200436A02007C64020009
:102F0000D05E02003F590200C8530200FFFDFCFAE8
:102F1000F8F6F4F2F0EEECEAE9E7E5E3E1E0DEDC16
:102F2000DAD9D7D5D4D2D0CFCDCBCAC8C7C5C3C2C2
:102F3000C0BFBDBCBAB9B7B6B4B3B2B0AFADACAA3E
:102F4000A9A8A6A5A4A2A1A09E9D9C9A9998979590
:102F5000949392908F8E8D8B8A89888786848382C2
:102F600081807F7E7D7B7A797877767574737271D4
:102F7000706F6E6D6C6B6A696867666564636261C9
:102F8000605F5E5D5C5B5A595858575655545352B2
:102F90005150504F4E4D4C4B4A4A49484746464582
:102FA0004443424241403F3E3E3D3C3B3B3A393840
:102FB0003837363535343332323130302F2E2E2DEE
:102FC0002C2B2B2A29292827272625252423232291
:102FD000212120201F1E1E1D1C1C1B1B1A19191825
:102FE00018171616151514131312121111100F0FAE
:102FF0000E0E0D0D0C0C0B0A0A090908080707062E
:1030000006050504040303020201000000809D433D
:1030100000009B430000C8430000000000000000C7
:103020000000000053657474696E67732053746FF9
:1030300072656400454550524F4D20496E69746970
:10304000616C697A65640A003B20003A0A0020201E
:103050004D363033200020440020204D34313220C2
:10306000530046696C616D656E742072756E6F7584
:10307000742073656E736F723A002055004C0046E1
:10308000696C616D656E74206C6F61642F756E6C18
:103090006F6164206C656E677468733A0020204D20
:1030A0003835312058005A2D50726F6265204F66B6
:1030B000667365740020204D343133205300506F07
:1030C0007765722D4C6F7373205265636F766572EE
:1030D000793A0020440020490020204D333034202C
:1030E000500020440020490020204D333031205032
:1030F000005049442073657474696E67733A002008
:10310000460020480020204D3134352053004D61C9
:1031100074657269616C2068656174757020706196
:1031200072616D65746572733A00204A0020204711
:103130003239205720490020204D343230205300AE
:103140004175746F20426564204C6576656C696ECC
:10315000673A0020204D323036205800486F6D65A8
:10316000206F66667365743A002058002053002073
:10317000204D323035204200416476616E636564D3
:103180003A20423C6D696E5F7365676D656E745F72
:1031900074696D655F75733E20533C6D696E5F6643
:1031A000656564726174653E20543C6D696E5F7440
:1031B000726176656C5F66656564726174653E20F8
:1031C000583C6D61785F785F6A65726B3E20593C50
:1031D0006D61785F795F6A65726B3E205A3C6D6104
:1031E000785F7A5F6A65726B3E20453C6D61785FFF
:1031F000655F6A65726B3E002054002052002020FB
:103200004D323034205000416363656C65726174E7
:10321000696F6E2028756E6974732F7332293A2096
:10322000503C7072696E745F616363656C3E2052DE
:103230003C726574726163745F616363656C3E20A8
:10324000543C74726176656C5F616363656C3E00CB
:1032500020204D3230312058004D6178696D756DF8
:1032600020416363656C65726174696F6E202875B7
:103270006E6974732F7332293A0020204D32303337
:103280002058004D6178696D756D206665656472C2
:10329000617465732028756E6974732F73293A0001
:1032A00053746570732070657220756E69743A008E
:1032B00020440020204D32303020530020446973D8
:1032C00061626C65640A0046696C616D656E7420AC
:1032D00073657474696E67733A0020204D31343918
:1032E0002043203B20556E69747320696E2043652E
:1032F0006C736975730A0020286D6D2900202047C2
:103300003231202020203B20556E69747320696E75
:10331000206D6D000000FA430000FA4300002041D8
:10332000000096420000A0420000A0420000C843F6
:103330000000BA42DC050000DC050000640000006B
:103340004B00000024F4D43050C38E20C2A240179A
:10335000828B7011127A910D816CD90AA861E108F3
:10336000C7586607615143061E4B5D05C145A7045A
:103370001A411104093D9803713931034036DB02CB
:1033800065339102D4305402802E1D02632CEE016D
:10339000752AC501B028A001102781018F2564017D
:1033A0002B244B01E0223401AC211F018D200D01A3
:1033B000801FFC00841EED00971DDF00B81CD200AA
:1033C000E61BC600201BBC00641AB200B219A8009C
:1033D0000A19A0006A189900D117910040178B00B4
:1033E000B516840031167E00B31579003A157300C6
:1033F000C7146F0058146A00EE1366008813630048
:1034000025135E00C7125B006C12570015125400A2
:10341000C111510070114F0021114B00D61049000D
:103420008D1047004610440002104200C00F4000BB
:10343000800F3E00420F3C00060F3B00CB0E3800D1
:10344000930E37005C0E3500270E3400F30D32006A
:10345000C10D3100900D3000600D2E00320D2D0099
:10346000050D2C00D90C2B00AE0C2900850C290071
:103470005C0C2700350C27000E0C2600E80B2400FE
:10348000C40B2400A00B23007D0B23005A0B21004A
:10349000390B2100180B2000F80A1F00D90A1E0062
:1034A000BB0A1E009D0A1D00800A1D00630A1C0045
:1034B000470A1B002C0A1B00110A1A00F7091A0000
:1034C000DD091900C4091900AB0919009209170098
:1034D0007B091800630917004C091600360916000D
:1034E000200916000A091500F5081500E008140067
:1034F000CC081400B8081400A408140090081300A5
:103500007D0812006B0813005808120046081200CC
:1035100034081100230811001208110001081100DD
:10352000F0071000E0071000D0071000C0071000DF
:10353000B0070F00A107100091070E0083070F00CE
:1035400074070F0065070E0057070E0049070E00AD
:103550003B070D002E070E0020070D0013070D007E
:1035600006070D00F9060C00ED060D00E0060C0044
:10357000D4060C00C8060C00BC060C00B0060C00FB
:10358000A4060B0099060C008D060B0082060B00AA
:1035900077060B006C060B0061060A0057060B004D
:1035A0004C060A0042060A0038060A002E060A00E7
:1035B00024060A001A060A001006090007060A0077
:1035C000FD050900F4050900EB050900E205090005
:1035D000D9050900D0050900C7050900BE05090085
:1035E000B5050800AD050800A50509009C05080003
:1035F000940508008C050800840508007C05080077
:10360000740508006C050700650508005D050700E6
:10361000560508004E05070047050700400508004D
:1036200038050700310507002A05070023050700B4
:103630001C050600160507000F0507000805060013
:1036400002050700FB040600F5040700EE0406006F
:10365000E8040600E2040700DB040600D5040600C7
:10366000CF040600C9040600C3040600BD0406001A
:10367000B7040600B1040500AC040600A604060069
:10368000A00405009B0406009504050090040600B4
:103690008A04050085040500800406007A040500FC
:1036A00075040500700405006B0405006604050040
:1036B000610405005C040500570405005204050080
:1036C0004D04050048040500430405003E040400C1
:1036D0003A04050035040500300404002C040500FC
:1036E00027040400230405001E0404001A04040037
:1036F00016040500110404000D040400090405006B
:103700000404040000040400FC030400F8030400A3
:10371000F4030400F0030400EC030400E8030400D5
:10372000E4030400E0030400DC030400D803040005
:10373000D4030400D0030400CC030400C803030036
:10374000C503030024F404D9201BC40C5C0E9804A8
:10375000C4095F0265077101F405F900FB04B300B9
:1037600048048700C103690058035500030345005E
:10377000BE023A008402310053022A0029022500C9
:1037800004022000E4011C00C8011900AF01170069
:1037900098011400840113007101100061011000F0
:1037A00051010E0043010D0036010B002B010B00EF
:1037B00020010B00150109000C010900030108009C
:1037C000FB000800F3000800EB000700E40006001F
:1037D000DE000600D8000600D2000600CC0005007E
:1037E000C7000500C2000500BD000400B9000400C8
:1037F000B5000400B1000400AD000400A9000400FD
:10380000A5000300A20003009F0004009B0003002A
:10381000980003009500020093000300900003004D
:103820008D0002008B000300880002008600020069
:1038300084000300810002007F0002007D0002007E
:103840007B00020079000200770001007600020090
:103850007400020072000100710002006F0002009B
:103860006D0001006C0002006A00010069000200A6
:1038700067000100660001006500010064000200AD
:103880006200010061000100600001005F000200B1
:103890005D0001005C0001005B0001005A000100B6
:1038A00059000100580001005700010056000100B6
:1038B00055000100540001005300000053000100B6
:1038C0005200010051000100500001004F000100B2
:1038D0004E0000004E0001004D0001004C000100B0
:1038E0004B0000004B0001004A00010049000100AC
:1038F00048000000480001004700010046000000A9
:1039000046000100450000004500010044000100A0
:10391000430000004300010042000000420001009B
:103920004100000041000100400001003F00000094
:103930003F0001003E0000003E0001003D0000008D
:103940003D0001003C0000003C0000003C00010084
:103950003B0000003B0001003A0000003A0001007B
:103960003900000039000100380000003800000074
:103970003800010037000000370001003600000069
:103980003600000036000100350000003500000060
:103990003500010034000000340000003400010054
:1039A000330000003300000033000100320000004B
:1039B0003200000032000100310000003100000040
:1039C0003100010030000000300000003000010034
:1039D0002F0000002F0000002F0000002F0001002A
:1039E0002E0000002E0000002E0001002D0000001F
:1039F0002D0000002D0000002D0001002C00000013
:103A00002C0000002C0000002C0001002B00000006
:103A10002B0000002B0000002B0001002A000000FA
:103A20002A0000002A0000002A00010029000000EE
:103A300029000000290000002900000029000100E1
:103A400028000000280000002800000028000000D6
:103A500028000100270000002700000027000000C8
:103A600027000000270001002600000026000000BB
:103A700026000000260000002600010025000000AE
:103A800025000000250000002500000025000000A2
:103A90002500010024000000240000002400000094
:103AA0002400000024000100230000002300000087
:103AB000230000002300000023000000230000007A
:103AC000230001002200000022000000220000006C
:103AD000220000002200000022000100210000005E
:103AE0002100000021000000210000002100000052
:103AF0002100000021000100200000002000000043
:103B00002000000020000000200000002000000035
:103B100020000000200001001F0000001F00000026
:103B20001F0000001F0000001F0000001F00000019
:103B30001F0001001E0000001E0000001E0000000B
:103B40001E000000393000003325000087190000F6
:103B5000B00F0000DB080000BD040000740200008C
:103B60003F01000020436F756E7420583A00426593
:103B70006400453100626564002C207379737465BC
:103B80006D2073746F707065642120486561746581
:103B9000725F49443A200048656174696E67204647
:103BA00061696C65640048656174696E672066616F
:103BB000696C6564004D3131322053687574646FEF
:103BC000776E001000C90210012C01400122017023
:103BD000011801B0010E01F00104015002FA00B019
:103BE00002F0003003E600D003DC009004D2007045
:103BF00005C800A006BE000008B400B009AA00D0A5
:103C00000BA000600E960060118C00001582002051
:103C1000197800C01D6E00A0226400B0275A0090E1
:103C20002C500000314600E0343C00103832009047
:103C30003A2800603C1E00A03D1400803E0A00208F
:103C40003F0000544845524D414C2052554E41577B
:103C5000415900546865726D616C2052756E6177D0
:103C60006179004572723A204D415854454D5000DB
:103C70004D415854454D50207472696767657265AF
:103C800064004572723A204D494E54454D50004DE6
:103C9000494E54454D50207472696767657265647A
:103CA00000202F002042403A0020403A0020573A9E
:103CB0000020573A00496E76616C6964206578741B
:103CC00072756465720A007C3C3E5E2B3D3F2F5B43
:103CD0005D3B2C2A225C0043616E6E6F74206F7016
:103CE000656E207375626469722000534420496ECA
:103CF0006974204661696C005344206361726420DA
:103D00006F6B0A006F70656E526F6F742066616929
:103D10006C65640A00766F6C756D652E696E6974EA
:103D2000206661696C65640A004E6F20534420630D
:103D30006172640A000A4D3234004D32332025731B
:103D40000041425300504C41002E0A006F70656ED6
:103D5000206661696C65642C2046696C653A2000B8
:103D600046696C652073656C65637465640A002040
:103D700053697A653A200046696C65206F70656EFC
:103D800065643A2000454E4420535542524F5554E5
:103D9000494E450A002220706F7300222070617224
:103DA000656E743A2200535542524F5554494E4560
:103DB0002043414C4C207461726765743A22005371
:103DC000756263616C6C204F766572666C6F77000C
:103DD0004578636565646564206D6178205355425C
:103DE000524F5554494E452064657074683A002E10
:103DF0000A0044656C6574696F6E206661696C6564
:103E0000642C2046696C653A200046696C65206424
:103E1000656C657465643A005344207072696E7411
:103E2000696E67206279746520004E6F7420534478
:103E3000207072696E74696E670A002F6175746F05
:103E400025632E670057726974696E6720746F204E
:103E500066696C653A2000667265736800646F6914
:103E60006E67002066696C653A20004E6F7720000F
:103E700002FD55555555555FFFFFFFFFFFFFFFFF43
:103E8000FFFE00000000003FFFFFFFFFFFFFFFFFFE
:103E9000FFFD000007FFFFFFFFFFFFFFFFFFFFFF2A
:103EA000FFFE07C00555555555555FFFFFFFFFFF46
:103EB000FFFC0A200600000000003FFFFFFFFFFF9D
:103EC000FFFE141005000007FFFFFFFFFFFFFFFFCD
:103ED000FFFC28080607C00555555555555FFFFFDF
:103EE000FFFE5404040A200600000000003FFFFF0C
:103EF000FFFC600406141005000007FFFFFFFFFF32
:103F0000FFFE50040428080607C0055555555555B1
:103F10005FFC6004065404040A2006000000000050
:103F20003FFE54041C60040614100500000000004D
:103F30001FFC28082E50040428080607C00001F0C2
:103F40003FFE1410546004065404040A20000208C2
:103F50001FFC0A206654041C6004061410000504AB
:103F60003FFE07C05428082E5004042808000A0207
:103F70001FFC00002E1410546004065404001501A8
:103F80003FFE00001C0A206654041C600400180157
:103F90001FFC00000607C05428082E50040014011E
:103FA0003FFE00000400002E1410546004001801AD
:103FB0001FFCFFFFFE00001C0A206654041C1501B4
:103FC0003FFED5555400000607C05428082A0A02AF
:103FD0001FFC84104600000400002E14105105043C
:103FE0003FFEC41044FFFFFE00001C0A206102884F
:103FF0001FFC841046D5555400000607C05101F03F
:104000003FFE84104484104600000400002A000093
:104010001FFCC41046C41044FFFFFE00001C00003B
:104020003FFE841044841046D55554000000000023
:104030001FFCD55556841044841046000000000033
:104040003FFCFFFFFCC41046C41044FFFFFFFFFF0E
:104050009FFE000006841044841046D555555555E2
:10406000BFFD555554D55556841044841041041055
:104070009FFFFFFFFCFFFFFCC41046C4104104116A
:10408000BFFFFFFFFE0000068410448410410410AF
:104090009FFFFFFFFD555554D55556841041041020
:1040A0009FFFFFFFFFFFFFFCFFFFFCC41041041157
:1040B000BFFFFFFFFFFFFFFE00000684104104105A
:1040C0009FFFFFFFFFFFFFFD555554D55555555533
:1040D000BFFFFFFFFFFFFFFFFFFFFCFFFFFFFFFF33
:1040E0009FFFFFFFFFFFFFFFFFFFFE00000000003C
:1040F0003FFFFFFFFFFFFFFFFFFFFD5555555555E4
:104100005FFFFFFFFFFFFFFFFFFFFFFFFFFFFFFF5F
:10411000FFFFFFFFFFFFFFFFFFFFFFFFFFFFFFFFAF
:10412000FFFFFFFFFFFFFFFFFFFFFFFFFFFFFFFF9F
:10413000FFFFFFFFFFFFFFFFFFFFFFFFFFFFFFFF8F
:10414000FFE02EFB7DFBFBCFC1DFBB3EC0E1FE3CB1
:104150001FFDEE7B39F9F3CF9EDFBB3EDFDEFCDDDA
:10416000E7FDEE3BBBF9EBD7BF5FBB5EDFDEFDEDEE
:10417000F7FDEEBBD3FAEBB73FDFBB4EDFDFFFCD82
:10418000F3FDEEDBC7FAEBBB7FC03B6EC0E3FF1D68
:10419000F3FDEECBEFFADBBB7FDFBB66DFF8FFCDD5
:1041A000F3FDEEEBEFFB5B033F5FBB76DFFE7FEDE6
:1041B000F3FDEEF3EFFB5B79BEDFBB7ADFDE7DED77
:1041C000F7FDEEF3EFFBBAFD9EDFBB7CDFDEFDCD3E
:1041D000E7FDEEFBEFFBBAFDC1DFBB7EC0E0FE1CDE
:1041E0001F6D61726C696E66772E6F726700322E7A
:1041F000302E375F4457372E33001FFFFFFFFFFF7E
:10420000FF600000000001FF400000000000FF8090
:1042100000000000007F83CF00000C303F87FF804C
:10422000000C301F867980000C000F8C30C7838C07
:1042300030E78C30CFC7CC31F38C30DCECEC33B9C9
:104240008C30D86C6C33198C30D06C0C33198C30AA
:10425000D86C0C33198C30DC6C0E3B198C30CF7C55
:10426000079F198C30C77C038F19400000000000A5
:1042700002600000000000061FFFFFFFFFFFF86064
:1042800001F4017001EA019001E001B001D601D012
:1042900001CC010002C2013002B8016002AE0190FF
:1042A00002A401D0029A012003900170038601C08C
:1042B000037C0130047201A004680120055E01B096
:1042C00005540160064A0120074001F0073601F05D
:1042D000082C01100A2201500B1801C00C0E0150CD
:1042E0000E04013010FA002012F0005014E600C055
:1042F00016DC007019D200501CC800501FBE0070A0
:1043000022B400B025AA00F028A000202C9600308E
:104310002F8C0010328200A0347800F0366E00E05E
:10432000386400803A5A00403B5500E03B5000F0B2
:104330003C4600C03D3C00603E3200E03E2800307C
:104340003F1E00503F1900703F1400A03F0A00C0FC
:104350003F0000D03FF6FFE03FECFF2020506C61B3
:104360006E6E657242756666657242797465733AFF
:1043700020002046726565204D656D6F72793A2088
:1043800000436F6D70696C65643A20417072203231
:104390003420323032310A00204C61737420557061
:1043A00064617465643A20323032312D30342D31FD
:1043B00038207C20417574686F723A2054696E7998
:1043C0004D616368696E657333440A00322E302E86
:1043D000375F4457372E330A004D61726C696E00A7
:1043E00020536F6674776172652052657365740A35
:1043F00000205761746368646F6720526573657449
:104400000A002042726F776E206F757420526573B8
:1044100065740A002045787465726E616C2052657F
:104420007365740A00506F77657255700A00737473
:104430006172740A004732385859004D31303031BA
:10444000006572726F722077726974696E6720748A
:104450006F2066696C650A00446F6E652073617633
:10446000696E672066696C652E0A004D3239004519
:104470006E6473746F707300255320256320256369
:1044800020256320256300205A3A0020593A002055
:10449000583A00656E6473746F7073206869743A7B
:1044A000200000000A0B02090C0D0E08070304018E
:1044B00000000000000000000000000000000000FC
:1044C00000000000000000000000000000001211C9
:1044D00010000000000000000000000000000000CC
:1044E0000000000000000000004D6F76652025737D
:1044F0006D6D004D6F766520302E316D6D004D6F06
:10450000766520316D6D004D6F76652031306D6DB3
:10451000004D6F7665204178697300457874727537
:10452000646572004D6F7665205A004D6F76652088
:1045300059004D6F7665205800453D413D43686107
:104540006E67652046696C616D656E7400556E6CB2
:104550006F61642046696C616D656E74004C6F61BB
:10456000642046696C616D656E74005072656865A3
:10457000617420437573746F6D0050726568656176
:10458000742024004261636B0050726F62696E6731
:10459000204661696C656400205A3A200020593A2F
:1045A000200042656420583A200073686F770062EB
:1045B0007574746F6E00626567696E00446973613B
:1045C000626C6552756E6F75740050757267654DDB
:1045D0006F72650050617573656400436F6E746936
:1045E0006E7565004C6F61642046696C616D656E27
:1045F00074205400496E736572742066696C616D35
:10460000656E7420616E642073656E64204D313078
:10461000380A00220A00556E6B6E6F776E20636F4A
:104620006D6D616E643A2022002042002050006FC0
:104630006B00544D33442043523130563220526582
:104640006164792E005072696E74696E672E2E2E29
:10465000005072696E742050617573656400204566
:1046600000205A00205900204D39322058002045A2
:104670003A00205A3A0020593A00583A0020746F04
:104680006F206C6F6E6720657874727573696F6EDA
:104690002070726576656E7465640A0020636F6CC5
:1046A0006420657874727573696F6E2070726576B8
:1046B000656E7465640A00526573656E643A200025
:1046C0006E6F74696669636174696F6E20000000C3
:1046D0002200250028002B002E00310034000201AA
:1046E0000000050108010B01000021002400270043
:1046F0002A002D00300033000101000004010701F1
:104700000A01050505050705080808080202020256
:104710000A0A08080404040401010101010101015D
:104720000303030303030303040707070C0C0C0C28
:104730000C0C0C0C02020202060606060606060611
:104740000B0B0B0B0B0B0B0B01021020200808109E
:1047500020401020408002010201080402010102F1
:1047600004081020408080402010080402018004CA
:104770000201804020100804020108040201010225
:1047800004081020408001020408102040806002CC
:104790002C0211241FBECFEFD1E2DEBFCDBF00E05F
:1047A0000CBF13E0A0E0B2E0E4E2FAEE02E00BBFDF
:1047B00002C007900D92A839B107D9F728E1A8E9FE
:1047C000B3E001C01D92AB3AB207E1F713E2C8ECC7
:1047D000D3E200E006C021970109802FFE010F946B
:1047E0006871C73CD10780E00807A9F70F94965F6E
:1047F0000D9400750C940000FC0184910895FC0157
:10480000808108951198000000009091020187FDB9
:104810009095917090930001119A000000000000A3
:1048200000001198000000009091020186FD909513
:10483000917090930001119A0000000000000000A8
:104840001198000000009091020185FD90959170F3
:1048500090930001119A00000000000000001198E0
:10486000000000009091020184FD9095917090935A
:104870000001119A000000000000000011980000E3
:1048800000009091020183FD90959170909300013A
:10489000119A0000000000000000119800000000C4
:1048A0009091020182FD9095917090930001119A70
:1048B000000000000000000011980000000090912E
:1048C000020181FD9095917090930001119A000072
:1048D000000000000000119800000000809102011B
:1048E000817080930001119A000000000000000018
:1048F000089590E080E00895CF93DF93DB01F90104
:104900009C919130C1F0943080F094509C93883009
:10491000D1F480819181009771F001979183808318
:10492000480F591FEA01188206C08C3539F49C5F84
:104930009C93943041F4DF91CF9108958B3339F7F4
:1049400081E08C93F8CF20813181B9016F5F7F4F77
:1049500071836083420F531FEA01888380819181B4
:104960008F3591056CF7E7CF0F931F9381E000918E
:104970009C1610919D1620919E1630919F16409185
:1049800098165091991660919A1670919B1604177B
:1049900015072607370708F480E01F910F91089547
:1049A00090E080E00895282F9091D708833021F47B
:1049B00095FD0FC094FD0FC0892F90E0B0E0A0E0FE
:1049C00004C0B695A795979587952A95D2F78170DB
:1049D000089581E0089580E00895CF92DF92EF92EC
:1049E000FF92CF93DF93EC01CC80DD80EE80FF80DF
:1049F00027E137EB41ED58EBC701B6010F94D173B6
:104A000087FD23C023E030E04BE953E4C701B60142
:104A10000F947F6A1816CCF0C880D980EA80FB809A
:104A200027E137EB41ED58EBC701B6010F94D17385
:104A300087FD0BC0C1E023E030E84DE953E4C70136
:104A4000B6010F947F6A18160CF4C0E08C2FDF912A
:104A5000CF91FF90EF90DF90CF9008952F923F92EB
:104A60004F925F926F927F928F929F92AF92BF927E
:104A7000CF92DF92EF92FF920F931F93CF93DF932A
:104A8000CDB7DEB72E970FB6F894DEBF0FBECDBF01
:104A9000E82ED62E042F122F282F30E03C872B87AC
:104AA000462F50E05A87498765E0F62EF29EC001F6
:104AB000F39E900D11249E878D87FA01E80FF91F50
:104AC000EE0FFF1FEE0FFF1FE65EF94F6081718151
:104AD000828193819B01AC010F946374882309F454
:104AE00034C1E00E612F6D0DFE9CF0011124A985EB
:104AF000BA85AE0FBF1FAA0FBB1FAA0FBB1FA65EB2
:104B0000B94FAC901196BC9011971296CC90129719
:104B10001396DC90E00EFE9CA0011124A985BA85B5
:104B2000A40FB51FAA0FBB1FAA0FBB1FA65EB94FCC
:104B3000EC901196FC90119712960C911297139687
:104B40009C90862F90E0AD85BE85A80FB91FAA0F57
:104B5000BB1FAA0FBB1FA65EB94F8C9011967C900D
:104B6000119712966C90129713965C90610F70E0FB
:104B7000AD85BE85A60FB71FAA0FBB1FAA0FBB1F0F
:104B8000A65EB94F4C9011963C90119712961C91CD
:104B9000129713962C90E80FF91FEE0FFF1FEE0FE0
:104BA000FF1FE65EF94FB081B98321812A833281EC
:104BB0003B8383818C83FA01E60FF71FEE0FFF1F03
:104BC000EE0FFF1FE65EF94F90819D83A181AE83BA
:104BD000B281BF83238128879701402F592DB701C8
:104BE000802F992D0F946374882321F0E12CF12CF0
:104BF00000E0912C9501A601B501C6010F946374E4
:104C0000882319F05701C02ED92C242D332D412F84
:104C1000522D642D732D812F922D0F946374882350
:104C200021F0412C312C10E0212C282D372D462D40
:104C3000552D682D772D862D952D0F94637488231F
:104C400021F0842C732C612E522C2D813E814F81BA
:104C500058856D817E818F8198850F946374882338
:104C600021F01D821E821F82188629813A814B8184
:104C70005C8169817A818B819C810F946374882324
:104C800041F03D8139834E814A835F815B83888512
:104C90008C8385E0EB85FC858E9FD0018F9FB00DC6
:104CA000112429853A85A20FB31FAA0FBB1FAA0F93
:104CB000BB1FA65EB94FBA87A9879501A601B501AA
:104CC000C6010F9471719701402F592D0F94707187
:104CD0006B017C01282D372D462D552D682D772D04
:104CE000862D952D0F947171242D332D412F522D2A
:104CF0000F9470719B01AC01C701B6010F947171E3
:104D00006B017C0129813A814B815C8169817A81C7
:104D10008B819C810F9471712D813E814F815885CB
:104D20000F9470719B01AC01C701B6010F947171B2
:104D300020E030E040E450E40F946B72A985BA851E
:104D40006D937D938D939C9313972E960FB6F89445
:104D5000DEBF0FBECDBFDF91CF911F910F91FF90AE
:104D6000EF90DF90CF90BF90AF909F908F907F900B
:104D70006F905F904F903F902F9008951092BA08D7
:104D80008091590290915A02A0915B02B0915C020D
:104D90008093930690939406A0939506B0939606FD
:104DA0000895129A0895269A2E9A0895AF92BF9266
:104DB000CF92DF92EF92FF920F931F93CF93DF93E7
:104DC0006B01E9014A3009F4C1C0453109F073C0F3
:104DD000DB011296ED91FC91F280C681D781809122
:104DE0000201809582708093000188E28A9500001C
:104DF000E9F7BF2CB29420EFB22230E1A32EAF0C22
:104E000048E2E42E88EF0E9402248E2D8A9500004D
:104E1000E9F7BFE1BF1508F485C08F2D8077806862
:104E20000E9402248B2D0E9402248E2D8A95000060
:104E3000E9F780E80E94022480E00E9402248E2D7F
:104E40008A950000E9F78AEF0E9402248E2D8A9548
:104E50000000E9F78E01005F1F4F8881807F0E946C
:104E6000022489918295807F0E940224C017D10775
:104E7000A1F78E2D8A950000E9F7F394E0E1BE0ECC
:104E8000FA10C0CF80910201827080930001D60198
:104E90001296CD91DC91CE010F946354811147C2DB
:104EA000DF91CF911F910F91FF90EF90DF90CF9006
:104EB000BF90AF900895FB0102811381423309F442
:104EC000F1C108F4F5C1463409F4E2C1473409F4EC
:104ED000E5C14B3329F589812B81D80112966C915C
:104EE000129713964C91213009F438C2233009F0FF
:104EF00002C238EF380F582F91E0431708F490E0C2
:104F000041E0531708F040E031E0561708F430E074
:104F1000592F542B352309F016C2942309F013C2DC
:104F200081E0BECF80EE8F0D8068807F0E940224DA
:104F30008F2D8295807F0E9402248E2D8A950000FD
:104F4000E9F780E80E94022480E877CF8091010190
:104F50008260809301018091020182708093000140
:104F60008091010181608093010180910201817033
:104F700080930001099A119A8091020180958270B4
:104F80008093000188E28A950000E9F788E790E0C5
:104F9000CEE9DFE0FE013197F1F70197D9F788EF0D
:104FA0000E94022418E2812F8A950000E9F780E22E
:104FB0000E94022480E00E940224812F8A95000032
:104FC000E9F780E00E94022480E80E940224812FF9
:104FD0008A950000E9F780E00E94022480E10E94A7
:104FE0000224812F8A950000E9F7CE010197F1F79D
:104FF000CE010197F1F7CE010197F1F7CE010197AC
:10500000F1F7CE010197F1F7CE010197F1F7CE014B
:105010000197F1F7CE010197F1F7CE010197F1F772
:10502000CE010197F1F7CE010197F1F7CE0101977B
:10503000F1F7CE010197F1F7CE010197F1F7219732
:10504000F1F780E20E94022480E40E940224812F72
:105050008A950000E9F780E20E94022480E60E941F
:1050600002241A950000E9F710E0D0E0C8E28D2F85
:10507000807780680E940224812F0E9402248C2F56
:105080008A950000E9F780E80E94022480E00E94EF
:1050900002248C2F8A950000E9F78AEF0E940224EF
:1050A0008C2F8A950000E9F790E21198000000002B
:1050B00080910201817080930001119A000000002C
:1050C0000000000011980000000080910201817032
:1050D00080930001119A0000000000000000119868
:1050E0000000000080910201817080930001119AFC
:1050F00000000000000000001198000000008091F6
:105100000201817080930001119A000000000000EC
:1051100000001198000000008091020181708093CE
:105120000001119A0000000000000000119800002A
:10513000000080910201817080930001119A0000AB
:1051400000000000000011980000000080910201A2
:10515000817080930001119A00000000000000009F
:10516000119800000000809102018170809300017D
:10517000119A0000000000000000119800000000DB
:1051800080910201817080930001119A000000005B
:105190000000000011980000000080910201817061
:1051A00080930001119A0000000000000000119897
:1051B0000000000080910201817080930001119A2B
:1051C0000000000000000000119800000000809125
:1051D0000201817080930001119A0000000000001C
:1051E00000001198000000008091020181708093FE
:1051F0000001119A0000000000000000119800005A
:10520000000080910201817080930001119A0000DA
:1052100000000000000011980000000080910201D1
:10522000817080930001119A0000000000000000CE
:1052300011980000000080910201817080930001AC
:10524000119A00000000000000008C2F8A950000D9
:10525000E9F7915009F029CF88EF0E9402248C2FA2
:105260008A950000E9F7DF5F105FD03209F0FFCECA
:1052700080E00E94022480EC0E940224CA95000073
:10528000E9F78091020182708093000181E008CEED
:10529000D80115968C91888381E002CEF801818136
:1052A0008883FACFB901C8010F94805481E0F8CD0A
:1052B000443171F0473109F033CE1882F801828110
:1052C0008983858181508A8383818B8381E0E8CDC6
:1052D000D80115964C91159750E0440F551F70E07A
:1052E00060E016968D919C910F94A174C8010F9463
:1052F000795481E0D5CD481708F412CE861708F40A
:105300000FCEFA80E12CD12C243070F41DC0BE01E8
:10531000C8010F948054898198819D0D98838E0DCA
:105320008983FF0C09F4FCCDF7FEF6CFF0CF4D8159
:1053300050E0440F551F70E060E08E819F810F9414
:10534000A17481E0ADCDFA8030E0F901E554FD4F64
:10535000D08029543D4FF901E080E6CF58E0580F46
:10536000382FCACDEF92FF920F931F93CF93DF9305
:10537000EC018B017A018A859B858617970731F0AE
:10538000888199810F9459561B870A87B7018881B4
:1053900099810F94AD472E813F81820F932F911DEC
:1053A0009F838E8390E080E0DF91CF911F910F91DA
:1053B000FF90EF9008959F92AF92BF92CF92DF92AD
:1053C000EF92FF920F931F93CF93DF93EC018B012A
:1053D000942EA52E8A859B858617970731F08881A4
:1053E00099810F9459561B870A878885998501965C
:1053F00049F5BC800A818E81080FC880D980D6010A
:105400005596ED91FC91C6011995B80EE92CFA2C30
:1054100010E0F70121917F01211127C08E819F812A
:10542000810F911D9F838E8390E080E0DF91CF916B
:105430001F910F91FF90EF90DF90CF90BF90AF90B2
:105440009F9008950E811F81692D7A2D8881998101
:105450000F94AD47800F912F911D2885398528170E
:10546000390738F681E090E0E1CF4B2D602FC6017F
:105470000F94B156080F180FCCCFDF92EF92FF9226
:105480000F931F93CF93DF93EC01D62E1CAD0BAD82
:105490007C0184E0E80EF11CE98DFA8DC7011995B5
:1054A000412F480F2D2D602FC7010F94B1569BAD92
:1054B000890F8BAF81E090E0DF91CF911F910F9129
:1054C000FF90EF90DF900895AB01BC0140939C16D4
:1054D00050939D1660939E1670939F1685E098E1F9
:1054E0000C940FE680932F028032B8F590916005FE
:1054F000891724F091E0980F9093600540915C0526
:1055000050915D0560915E0570915F05082E04C0A5
:1055100076956795579547950A94D2F741704093D1
:10552000201087FD1DC0282F082E000C330B3F9341
:105530008F938AE69AE09F938F938AE79AE09F93EE
:105540008F931F920E942CCB8DB79EB707960FB6F4
:10555000F8949EBF0FBE8DBF089510922010E1CF2A
:105560000D9477430F931F93CF93DF9300D01F9237
:10557000CDB7DEB79C0101EA18E090E1EDECF9E06F
:10558000D80101900D929A95E1F7F90120813181BE
:1055900042815381F80160857185828593850F94DE
:1055A0007171F801608771878287938780E090E04E
:1055B000A0EAB0E489839A83AB83BC83CE010196D1
:1055C0000F942D100F900F900F900F90DF91CF91AF
:1055D0001F910F9108952F923F924F925F926F9279
:1055E0007F928F929F92AF92BF92CF92DF92EF9273
:1055F000FF921F93CF93DF93CDB7DEB72C970FB6F3
:10560000F894DEBF0FBECDBF7A011901DC012D91E8
:105610003D914D915C912D833E834F835887FB01D3
:1056200040805180628073808090CD099090CE0937
:10563000A090CF09B090D009A50194016D817E8121
:105640008F8198850F947F6A81110EC011E0A301AC
:1056500092016091D1097091D2098091D309909102
:10566000D4090F947F6A811110E0D1012D913D91F1
:105670004D915C9129873A874B875C87F701C08001
:10568000D180E280F3802091130230911402409186
:10569000150250911602C701B6010F947F6A882344
:1056A00009F44EC0C0921302D0921402E092150287
:1056B000F09216028091D9099091DA09A091DB0944
:1056C000B091DC094091D1095091D2096091D30980
:1056D0007091D4098092A1089092A208A092A30888
:1056E000B092A4084093A5085093A6086093A70819
:1056F0007093A808C092A908D092AA08E092AB08BB
:10570000F092AC088093AD089093AE08A093AF08D8
:10571000B093B00820E030E040E05FE360914E10CD
:1057200070914F1080915010909151100F94E56A34
:1057300069837A838B839C83CE0101960F942D100D
:105740002D813E814F8158852093A1083093A20876
:105750004093A3085093A4084092A5085092A6082D
:105760006092A7087092A808D1012D913D914D91AA
:105770005C916091AD087091AE088091AF089091F6
:10578000B0080F9471716093AD087093AE08809368
:10579000AF089093B00811112FC020E030E0A901AC
:1057A00069857A858B859C850F947F6A811133C0CA
:1057B00060E070E088EC92E469837A838B839C8359
:1057C000CE0101960F942D102C960FB6F894DEBFE3
:1057D0000FBECDBFDF91CF911F91FF90EF90DF9073
:1057E000CF90BF90AF909F908F907F906F905F9081
:1057F0004F903F902F9008952AEF3EE74AE25FE3F3
:1058000060915210709153108091541090915510E6
:105810000F94E56AD1CF60E070E080EA91E4CCCFEC
:10582000CF93DF9300D01F92CDB7DEB780E090E03A
:10583000A0EAB0E489839A83AB83BC8361E0CE01A4
:1058400001960F9430080F900F900F900F90DF91FA
:10585000CF91089580911E0590911F05009731F01A
:105860004AE050E070E060E00D949A6860E070E01B
:10587000CB0108958091E10982FF0BC063E686E5C4
:105880009BE00E9447CB0F946D4E0E9447D281E06F
:10589000089580E0089580911E0590911F0500975E
:1058A00031F04AE050E070E060E00D946C6760E039
:1058B00070E0CB0108950E944B2C97FD0CC00E9414
:1058C0004B2C6F3F71058105910509F034F40E945E
:1058D0004B2C862F089580E008958FEF08958091D6
:1058E0001E0590911F05892B41F00E945B2C91E0D1
:1058F000811101C090E0892F089591E0FCCFCF92F3
:10590000DF92EF92FF920F931F93CF93DF936B0180
:105910007A01EC01C655DB4F28813CE0389F8001BD
:10592000399F100D112427FF24C0FB011182108222
:1059300088818F5F888388819801280F311D87FDBA
:105940003A95C90120911916F6012817190629F070
:1059500024F088818C300CF43CC0808191810496C5
:1059600080349C4908F475C0F601808191810496C9
:1059700072C088819801280F311D87FD3A95C901B1
:10598000209119162817190699F294F28881A80116
:10599000480F511D87FD5A95FA01EE0FFF1FE40FC6
:1059A000F51FEF52FA4E808187FFC2CF8881F80140
:1059B000E80FF11D87FDFA95CF01EE0FFF1FE80FED
:1059C000F91FEF52FA4E808160E08F770F949F4C61
:1059D000AFCF808191812881A801420F511D27FD01
:1059E0005A959A01FA01EE0FFF1FE20FF31FEF52D3
:1059F000FA4E21813281820F931FF70191838083B8
:105A000088819801280F311D87FD3A95F901EE0F25
:105A1000FF1FE20FF31FEF52FA4E808187FF20C075
:105A20008881080F111D87FD1A95F801EE0FFF1FE1
:105A3000E00FF11FEF52FA4E808161E08F77DF9126
:105A4000CF911F910F91FF90EF90DF90CF900D9429
:105A50009F4C80E49CE9F701918380838FEF8883DA
:105A6000DF91CF911F910F91FF90EF90DF90CF903A
:105A70000895AF92BF92CF92DF92EF92FF920F9371
:105A80001F93CF93DF93EC015B018A01FB01199512
:105A900087FD16C0C82ED12CF12CE12C2196F801DF
:105AA000C082D182E282F382CE01DF91CF911F9139
:105AB0000F91FF90EF90DF90CF90BF90AF9008953F
:105AC000982F907E903CA9F48F7190E0B0E0A0E018
:105AD0006C017D0156E0CC0CDD1CEE1CFF1C5A95C0
:105AE000D1F7CE010196F50119958F73C82A229638
:105AF000D6CF982F907F903E11F58F7090E0B0E058
:105B0000A0E06C017D0136E0CC0CDD1CEE1CFF1C1E
:105B10003A95D1F7CE010196F50119958F73C82AF0
:105B200046E0CC0CDD1CEE1CFF1C4A95D1F7CE01E3
:105B30000296F50119958F73C82A2396B0CF982F36
:105B4000987F903F79F5877090E0B0E0A0E06C011D
:105B50007D0186E0CC0CDD1CEE1CFF1C8A95D1F784
:105B6000CE010196F50119958F73C82A96E0CC0CE9
:105B7000DD1CEE1CFF1C9A95D1F7CE010296F501B3
:105B800019958F73C82A26E0CC0CDD1CEE1CFF1C77
:105B90002A95D1F7CE010396F50119958F73C82A7E
:105BA00024967DCF982F907C903841F4807C80386B
:105BB00069F42196CE01F5011995F8CF8E7F8D3FBE
:105BC00028F02196CE01F5011995F8CFC12CD12CE2
:105BD000760165CF9CE0899F802D112491E0980F7C
:105BE000909361052CE0280F20939B0830E02E5FF6
:105BF0003F4F40918E164217130619F014F080E0C3
:105C00000895209190169217D0F7662341F08E5F89
:105C10000F94735580919B088E5F0F9473558091FC
:105C20009B0890918E16891750F3209190169091B1
:105C30006105291720F3109291168093921681E046
:105C40000895CF9380915405811154C010929116FC
:105C5000109292161092931610925F1610925E1682
:105C600010926116109260161092631681E0809374
:105C7000621682E28093641610926916109268167A
:105C8000EDE7F6E12BE836E18FEF81932E173F0722
:105C9000E1F7C1E0C0937A1626EA31E0309370163E
:105CA00020936F16C093711610927216109273168D
:105CB00090E490937416109275162EE232E03093B1
:105CC0008C1620938B1622E232E030935D162093DF
:105CD0005C1697E19093811691E19093821690E182
:105CE00090937F1680937E1680937D160F949A541E
:105CF000C093540581E08093550588EB9AE1909319
:105D00008315809382151092851510928415CF917A
:105D1000089520915305022E000C330B82171306B1
:105D200041F08093530568EB7AE18AE596E10D94A2
:105D300059560895CF92DF92EF92FF920F931F93DF
:105D4000CF93DF93CDB7DEB72C970FB6F894DEBFB5
:105D50000FBECDBF6F3F71058105910509F0D0F4ED
:105D600086E596E10E943D2AE0915E16F0915F166D
:105D70003196849190E02C960FB6F894DEBF0FBE5A
:105D8000CDBFDF91CF911F910F91FF90EF90DF90EA
:105D9000CF900895F0909116E090921620915505BD
:105DA00021110FC048E95AE16E2D8F2D0F941D5718
:105DB00090E080E0F80EF0929116E092921699270A
:105DC000DACFC0905E16D0905F162AE536E13A83AE
:105DD00029832F2D30E03C832B832E2D30E03E8312
:105DE0002D8318861F822FEF3FEF3A8729871C8665
:105DF0001B860BED19E29E012F5F3F4FAB01BC01EB
:105E0000C6010F943230B6018AE596E10F945956D7
:105E10008F819885CFCFCF93DF93FC0125AD2111E2
:105E200004C021E025AF0F949A54C0915C16D09124
:105E30005D16E0918B16F0918C1682E01995E09139
:105E40008B16F0918C1681E0199530E020E044E14A
:105E5000BE018AE596E10F9496542DE836E147E1BC
:105E6000BE018AE596E10F949654E0918B16F0916D
:105E70008C1680E0DF91CF911994CF92DF92EF9250
:105E8000FF920F931F93CF93DF93CDB7DEB72C977D
:105E90000FB6F894DEBF0FBECDBFF0909116E09024
:105EA00092162091550521111DC048E75AE16E2D2B
:105EB0008F2D0F941D5790E080E0F80EF092911610
:105EC000E092921699272C960FB6F894DEBF0FBE7B
:105ED000CDBFDF91CF911F910F91FF90EF90DF9099
:105EE000CF900895C0905E16D0905F162AE536E1F7
:105EF0003A8329832F2D30E03C832B832E2D30E0F5
:105F00003E832D8318861F827A8769871C861B86AD
:105F10000BED19E29E012F5F3F4F4CEF53E2BC01A6
:105F2000C6010F94F630B6018AE596E10F945956F2
:105F30008F819885C2CF6FEF7FEF0C943D2FCF926A
:105F4000DF92EF92FF920F931F93CF93DF93CDB722
:105F5000DEB72C970FB6F894DEBF0FBECDBFF09022
:105F60009116E09092162091550521111DC048E52B
:105F70005AE16E2D8F2D0F941D5790E080E0F80EA2
:105F8000F0929116E092921699272C960FB6F894FB
:105F9000DEBF0FBECDBFDF91CF911F910F91FF905C
:105FA000EF90DF90CF900895C0905E16D0905F166E
:105FB0002AE536E13A8329832F2D30E03C832B8379
:105FC0002E2D30E03E832D8318861F827A876987C5
:105FD0001C861B860BED19E29E012F5F3F4F4FEF92
:105FE00053E2BC01C6010F94F630B6018AE596E192
:105FF0000F9459568F819885C2CFBF92CF92DF926E
:10600000EF92FF920F931F93CF93DF938B01F42EA8
:10601000E90141FB662760F90E94EA2D882309F413
:106020005AC0B12C0115110521F0C8010E9418D3E6
:10603000B82EE12C209721F0CE010E9403D5E82E46
:1060400080E8C82ED12CF0FE1EC085E190E08B19AF
:106050009109B7FC93958E199109E7FC939597FDEB
:10606000019695958795F82E30E8C32ED12CFA9499
:10607000F7FC09C060E270E080E090E00E949A2E98
:10608000C81AD90AF4CFBB2099F0C60166E070E0C7
:106090000F944071262F40919D0850919E08609169
:1060A0009C08C8010E9458D296E0899F6001112483
:1060B000EE2031F0B601CE010E949F2FC81AD90AF6
:1060C00087E0C816D10438F060E270E080E090E02C
:1060D0000E949A2EF3CFDF91CF911F910F91FF90E5
:1060E000EF90DF90CF90BF9008956FEF7FEF0C940B
:1060F0009F2FAF92BF92CF92DF92EF92FF920F93BA
:106100001F93CF93DF935C016B010E9418D3E82E9D
:10611000C6010E9403D5F12C03E110E0081B110910
:10612000C5E20E151F050CF4CFE18C2F90E09C0109
:106130002E5F3F4F40918E164217130609F0CCF5A3
:10614000099720919016281719069CF140919D08F7
:1061500050919E0860919C0810929116C0939216DF
:1061600025E1C5010E9458D2D1E0C114D104B1F09B
:106170006AE370E080E090E00E949A2E0E151F0501
:10618000D4F4C45F80918E16C81740F02091901609
:106190004C2F4950550B241715067CF4DF91CF91F5
:1061A0001F910F91FF90EF90DF90CF90BF90AF9035
:1061B0000895D0E0DACFDD2389F3802F880F080F10
:1061C000000F00939116C093921660E270E080E099
:1061D00090E00E949A2EC601DF91CF911F910F91FE
:1061E000FF90EF90DF90CF90BF90AF900C94753000
:1061F0008F929F92AF92BF92CF92DF92EF92FF92D7
:106200000F931F93CF93DF93CDB7DEB72C970FB6C5
:10621000F894DEBF0FBECDBF982F862F5A017901AB
:10622000D02E692F0E94EA2D882309F489C0C70166
:10623000002391F10E9418D3C82E80905E16909092
:106240005F1680915505811145C01FEF23E12C1980
:1062500040919D0850919E0860919C08C5010E9444
:1062600058D2CC2009F46CC0B6E08B9F50011124A9
:106270006AE370E080E090E00E949A2E57E0A51655
:10628000B10408F444C060E270E080E090E00E9455
:106290009A2EA81AB90AF2CF0E9403D5C82E809070
:1062A0005E1690905F1680915505882371F2FE016D
:1062B00033968AE0DF011D928A95E9F78AE596E137
:1062C0009A83898302EB19E29E012F5F3F4F4FEFC4
:1062D00053E212C0FE0133968AE0DF011D928A95D7
:1062E000E9F78AE596E19A83898302EB19E29E0138
:1062F0002F5F3F4F4CEF53E2B701C4010F94F630CC
:10630000B4018AE596E10F9459561F819FCF4091C1
:106310009B08212F30E0A6E0CA9EC00111242E5F09
:106320003F4F281739070CF49C0180E8821B8093AB
:10633000911640939216C701DD20A9F00E949B2F71
:106340002C960FB6F894DEBF0FBECDBFDF91CF9174
:106350001F910F91FF90EF90DF90CF90BF90AF9083
:106360009F908F9008950E947530EACFE6E5F6E1A0
:1063700083AF64AFCA010C9475302F923F924F9255
:106380005F926F927F928F929F92AF92BF92CF92C5
:10639000DF92EF92FF920F931F93CF93DF93D62F4D
:1063A000C72FFC0180809180A280B380C501B40119
:1063B00020E831E541E050E00F94C370C9016DE67B
:1063C00071E00F9440716B017C01C501B40120E1C3
:1063D0003EE040E050E00F94C370CA01B90128E1EB
:1063E00030E040E050E00F94C370362E272E062F89
:1063F000172F8CE3482E512C612C712CC501B40150
:10640000A30192010F94C370B62EA72ECA01B90141
:10641000A30192010F94C370CB01C114D10479F18F
:10642000AF92BF927F936F932F923F92FF92EF9222
:10643000DF92CF9286EB98E19F938F93CF93DF9378
:106440000F94166A8DB79EB70E960FB6F8949EBF3E
:106450000FBE8DBF8D2F9C2FDF91CF911F910F917C
:10646000FF90EF90DF90CF90BF90AF909F908F9074
:106470007F906F905F904F903F902F900895E11420
:10648000F104C9F0AF92BF927F936F932F923F9226
:10649000FF92EF9286EA98E19F938F93CF93DF93D9
:1064A0000F94166AEDB7FEB73C960FB6F894FEBF90
:1064B0000FBEEDBFCFCF012BB9F0AF92BF927F934C
:1064C0006F932F923F928AE998E19F938F93CF9396
:1064D000DF930F94166A8DB79EB70A960FB6F8949D
:1064E0009EBF0FBE8DBFB6CF892BA9F0AF92BF92D2
:1064F0007F936F9382E998E19F938F93CF93DF937C
:106500000F94166AEDB7FEB738960FB6F894FEBF33
:106510000FBEEDBF9FCFAF92BF928EE898E19F93E1
:106520008F93CF93DF930F94166A0F900F900F9075
:106530000F900F900F908ECF8F929F92AF92BF923D
:10654000CF92DF92EF92FF920F931F93CF93DF933F
:1065500010925205109251052FE320934C05109292
:106560004B0510924A051092490510924D05109264
:106570004E0510924F05109250059C01F901908133
:106580002F5F3F4F9032D1F39E34C9F4818190ED5B
:10659000980F9A3020F08D3211F08B3281F43296C0
:1065A0009F012F5F3F4F808180538A3008F47BC06A
:1065B0009F012F5F3F4F8081803209F476C0F093B6
:1065C000C008E093BF088F010F5F1F4FC0816AE2D0
:1065D00070E0C8010F94C674009731F0FC01319748
:1065E00080818032E1F31182CD3429F0C43519F075
:1065F000C73409F04BC0F80180810F5F1F4F803214
:10660000D1F380538A3008F041C0C0934C0530E08C
:1066100020E04AE0DF011196429FC001439F900DA8
:1066200011249C01205331098081280F311D87FDE1
:106630003A95818190ED980F9A30C8F130934B05CF
:1066400020934A058E3261F4329690E04AE0DF01F1
:1066500031968C9150ED580F5A3058F1909349056E
:10666000CD01DC0101964C914032D9F3CD3489F54E
:106670002E31310539F018F52731310519F02C315B
:10668000310539F5B0935205A0935105DF91CF91B3
:106690001F910F91FF90EF90DF90CF90BF90AF9040
:1066A0009F908F900895F9017BCFF90181CFFD0173
:1066B000B1CF949F800D112490ED980FC8CF25374E
:1066C000310538F027373105E8F2203A83E0380702
:1066D000C9F2D091BF0840E050E0BA0110E000E0FC
:1066E000C12CD12C7601C394FD0131968C91882365
:1066F00009F47FC08132E1F4CD34D1F42032310588
:10670000B9F440934D0550934E0560934F05709337
:106710005005F0935205E093510563E270E0CF011C
:106720000F94C674009709F4B1CFFC011082AECF6C
:1067300081548A3108F058C0DF019D91903291F068
:10674000A0EDA90FAA30E8F09E3271F49181905328
:106750009A30B8F00115110519F48F010150110993
:1067600090E013C0FD01E8CF9D3211F09B3291F70C
:106770009181A0EDA90FAA3020F09E3259F79281A5
:10678000E6CF9E2F9D1B309759F3A82FB0E046010E
:10679000570104C0880C991CAA1CBB1C8A95D2F70F
:1067A000482959296A297B29A15DBA4F9C93808188
:1067B0008154DF018A3108F497CFDF01819188236A
:1067C00009F492CF90ED980F9A30B8F393ED980FAB
:1067D000923098F38B3289F3CD010196EC91E0323F
:1067E00009F082CFDC01F8CF0115110501F78D0109
:1067F000DECF109352050093510540934D05509301
:106800004E0560934F057093500540CFFC01659194
:1068100075918591949108958091B208882319F01B
:1068200080E00F94A21380E008954F925F926F92E0
:106830007F928F929F92AF92BF92CF92DF92EF9210
:10684000FF92CF93DF9300D000D01F921F92CDB75D
:10685000DEB75C01DB01CD90DD90ED90FC90E09126
:106860002916F0912A16FE83ED8384819581A681F5
:10687000B78189839A83AB83BC839C01AD01C70137
:10688000B6010F9470712B013C01F501808091805D
:10689000A280B380AD81BE818D919D910D90BC9100
:1068A000A02D8D839E83AF83B88727E137EB41ED21
:1068B00058EBC301B2010F94D17387FDD1C023E01F
:1068C00030E04BE953E4C301B2010F947F6A18161C
:1068D0000CF4C6C02D813E814F815885C501B4019D
:1068E0000F9470712B013C0127E137EB41ED58EB20
:1068F0000F94D17387FDB4C023E030E84DE953E431
:10690000C301B2010F947F6A18160CF4A9C020E0ED
:1069100030E0A9016D817E818F8198850F9471711E
:106920002B013C0120E030E040E450E40F947F6A0A
:1069300087FF05C0412C512C30E4632E762C27E1D3
:1069400037EB41ED58E3C301B2010F9470719B0125
:10695000AC01C501B4010F94D17387FD81C020E063
:1069600030E84DE953E46D817E818F8198850F94E5
:1069700071712B013C0120E030E844E953E40F94AD
:10698000D17318163CF4412C20E8522E24E9622ED3
:1069900023E4722E27E137EB41ED58E3C301B20146
:1069A0000F9471719B01AC01C501B4010F947F6A12
:1069B00018160CF455C020E030E0A90169817A81F5
:1069C0008B819C810F9471714B015C0120E030E060
:1069D00040E951E40F947F6A87FF06C0812C912C17
:1069E00090E9A92E91E4B92E27E137EB41ED58E368
:1069F000C501B4010F9470719B01AC01C701B601D0
:106A00000F94D17387FD2CC020E030E04BE953E4B4
:106A100069817A818B819C810F9471714B015C013A
:106A200020E030E04DE853E40F94D173181634F4AD
:106A3000812C912C8DE8A82E83E4B82E27E137EB2A
:106A400041ED58E3C501B4010F9471719B01AC0194
:106A5000B1E0B983C701B6010F947F6A18160CF430
:106A60001982898128960FB6F894DEBF0FBECDBF7C
:106A7000DF91CF91FF90EF90DF90CF90BF90AF90DC
:106A80009F908F907F906F905F904F9008958F921E
:106A90009F92AF92BF92CF92DF92EF92FF92CF93ED
:106AA000DF93EC018090D8089090D908A090DA0884
:106AB000B090DB0820E030E0A901C501B4010F94DB
:106AC0007F6A882309F452C0C880D980EA80FB809D
:106AD000A7019601C501B4010F947F6A18160CF046
:106AE0004AC020911A0530911B0540911C05509118
:106AF0001D05C701B6010F947F6A882321F1C0925A
:106B00001A05D0921B05E0921C05F0921D052091FC
:106B10001605309117054091180550911905C701C8
:106B2000B6010F94E56A9B01AC0160E070E080E87B
:106B30009FE30F9470716093170270931802809313
:106B4000190290931A0260911702709118028091B5
:106B5000190290911A02DF91CF91FF90EF90DF9090
:106B6000CF90BF90AF909F908F90089560E070E0BD
:106B700080E89FE3F0CF60E070E0CB01ECCF9B01B9
:106B8000AC01485F5F4FBC016C5F7F4F0C94EB2AF8
:106B90000F931F93CF93DF9300D000D01F921F92CB
:106BA000CDB7DEB7FC018B0183A5811112C081E056
:106BB00083A784819581A681B781B05889839A8300
:106BC000AB83BC83BE016F5F7F4F81EA98E00E9478
:106BD000BF351D821E821F82188620E030E040E013
:106BE0005FE36091D5097091D6098091D7099091A2
:106BF000D8090F94717169837A838B839C839E017A
:106C00002B5F3F4FAE014F5F5F4F61ED79E08DEC41
:106C100099E00E94EB2A1D821E821F82188620E0C6
:106C200030E040E05FE3F8016085718582859385FF
:106C30000F94717169837A838B839C83B8016C5F35
:106C40007F4F9E012B5F3F4FAE014F5F5F4FC801EB
:106C50000E94EB2A28960FB6F894DEBF0FBECDBF78
:106C6000DF91CF911F910F9108952F923F924F92F4
:106C70005F926F927F928F929F92AF92BF92CF92CC
:106C8000DF92EF92FF920F931F93CF93DF93CDB7D5
:106C9000DEB7A2970FB6F894DEBF0FBECDBF8C0152
:106CA0001B015E834D834090CD095090CE096090CA
:106CB000CF097090D0098090D1099090D209A0900E
:106CC000D309B090D409DB018D919D910D90BC91B9
:106CD000A02D8F87988BA98BBA8B9C01AD01C30126
:106CE000B2010F9470716B017C01D10114968D91EA
:106CF0009D910D90BC91A02D8B8B9C8BAD8BBE8BF1
:106D00009C01AD01C501B4010F9470716F8B788F38
:106D1000898F9A8FAD81BE818D919D910D90BC918F
:106D2000A02D8F839887A987BA879C01AD01C301E5
:106D3000B2010F9470716B8F7C8F8D8F9E8FAD81A0
:106D4000BE8114968D919D910D90BC91A02D8B8745
:106D50009C87AD87BE879C01AD01C501B4010F942E
:106D600070716F8F78A389A39AA3A7019601C701B9
:106D7000B6010F94E56A6B017C012F89388D498D2E
:106D80005A8DCA01B9010F94E56A9B01AC01C70194
:106D9000B6010F9471714B015C012F8538894989C7
:106DA0005A896F81788589859A850F9470712B0136
:106DB0003C012B893C894D895E896B857C858D855D
:106DC0009E850F9470716B017C01A3019201C30138
:106DD000B2010F94E56A2B013C01A7019601C7019E
:106DE000B6010F94E56A9B01AC01C301B2010F9497
:106DF00071710F941F746B017C012B8D3C8D4D8D37
:106E00005E8DCA01B9010F94E56A2B013C012F8DFB
:106E100038A149A15AA1CA01B9010F94E56A9B01A1
:106E2000AC01C301B2010F9471719B01AC01C501AA
:106E3000B4010F94D1731816B4F520E030E0A90125
:106E4000C701B6010F94D17387FF2AC0C701B601ED
:106E5000905820E030E040EA50E40F94D1731816C7
:106E600014F5A1016D817E81C8010E943536A2967C
:106E70000FB6F894DEBF0FBECDBFDF91CF911F914B
:106E80000F91FF90EF90DF90CF90BF90AF909F90C9
:106E90008F907F906F905F904F903F902F900895CC
:106EA000C701B601D6CF20E030E040E050E4C50194
:106EB000B4010F94D173181624F4B101C8010E94D3
:106EC000C83519821A821B821C82BE016F5F7F4FF8
:106ED000C1010E94BF352DEC3CEC4CEC5CE3C701DA
:106EE000B6010F94E56A9B01AC01F80160817181E4
:106EF000828193810F94E56A69837A838B839C8373
:106F0000C8010F94DF46BE016F5F7F4F8D819E8168
:106F10000E94BF35ACCF3F924F925F926F927F92AB
:106F20008F929F92AF92BF92CF92DF92EF92FF9299
:106F30000F931F93CF93DF93CDB7DEB76C970FB648
:106F4000F894DEBF0FBECDBFDB010C91142F100FE4
:106F5000153008F067C11196DC90C22ECD0CB4E05C
:106F6000BC1508F45FC1ED2DF0E0E35FFA4F8080BF
:106F7000912CB12CA12C002E04C0B694A794979408
:106F800087940A94D2F780FE4DC1EC2DF0E0E35FC8
:106F9000FA4F8080912CB12CA12C012E04C0B69404
:106FA000A794979487940A94D2F780FE3BC1322E1F
:106FB000642F7C0140907E0650907F066090800692
:106FC000709081068091860690918706A091880630
:106FD000B0918906898F9A8FAB8FBC8F660F770B24
:106FE000072E000C880B990B0F94866A4B015C01ED
:106FF000602F000F770B880B990B0F94866A298DF1
:107000003A8D4B8D5C8D0F94E56AA30192010F942C
:107010007171A50194010F9471716D877E878F87BF
:10702000988B612F110F770B880B990B0F94866A41
:10703000298D3A8D4B8D5C8D0F94E56AA3019201E9
:107040000F947171A50194010F94707169837A8313
:107050008B839C83409082065090830660908406C8
:107060007090850680918A0690918B06A0918C067F
:10707000B0918D06898F9A8FAB8FBC8F632D660F71
:10708000770B072E000C880B990B0F94866A4B0127
:107090005C016D2DDD0C770B880B990B0F94866AC4
:1070A000298D3A8D4B8D5C8D0F94E56AA301920179
:1070B0000F947171A50194010F947171698B7A8B92
:1070C0008B8B9C8B6C2DCC0C770B880B990B0F94B6
:1070D000866A298D3A8D4B8D5C8D0F94E56AA301EC
:1070E00092010F947171A50194010F9470716D83D9
:1070F0007E838F839887F70180859185A285B385EC
:1071000089879A87AB87BC878D8B9E8BAF8BB88F17
:1071100045E351E061E070E0CE0141960E9451EDFF
:1071200045E351E061E070E0CE0105960E9451ED2B
:107130004AE351E061E070E0CE010D960E9451ED0E
:107140004AE351E061E070E0CE0101960E9451ED0A
:1071500089889A88AB88BC8827E137EB41ED58EBEA
:10716000C501B4010F94D17387FD5CC023E030E00A
:107170004BE953E4C501B4010F947F6A18160CF46F
:1071800051C08D849E84AF84B88827E137EB41EDF0
:1071900058EBC501B4010F94D17387FD43C023E0C0
:1071A00030E84DE953E4C501B4010F947F6A181625
:1071B000CCF18D809E80AF80B88427E137EB41ED24
:1071C00058EBC501B4010F94D17387FD2BC023E0A8
:1071D00030E04BE953E4C501B4010F947F6A1816FF
:1071E0000CF189809A80AB80BC8027E137EB41EDC0
:1071F00058EBC501B4010F94D17387FD13C023E090
:1072000030E84DE953E4C501B4010F947F6A1816C4
:107210004CF0AE014F5F5F4FBE01635F7F4FC70110
:107220000E9435366C960FB6F894DEBF0FBECDBF08
:10723000DF91CF911F910F91FF90EF90DF90CF9052
:10724000BF90AF909F908F907F906F905F904F9086
:107250003F9008958C38910514F08CE890E090935D
:10726000E4088093E3080C94A6DD0E944B2CCB012C
:1072700008950F931F93CF9380911E0590911F0542
:107280000097E9F0FC018F01C1912C2F2F7D81F037
:10729000C53411F0C536B9F7F801108270E060E02E
:1072A0000F940E66F801C083CF911F910F9108953E
:1072B00070E060E0CF911F910F910D940E6660E039
:1072C00070E0CB01F1CF2FEB280F2A3108F047C037
:1072D000E22FF0E080914D0590914E05A0914F0571
:1072E000B091500504C0B695A795979587952A95B6
:1072F000D2F780FD02C081700895E15DFA4FE08110
:10730000EE2341F18091BF089091C008E80FF92F5A
:10731000F11D808190ED980F9A3030F08E3251F44B
:10732000818180538A3098F4F0931F05E0931E0505
:1073300081E008958D3211F08B3249F4818190ED16
:10734000980F9A3088F38E3211F48281EACFF0E000
:10735000E0E0EACF10921F0510921E05E9CF80E011
:1073600008950E946339882341F081E020911E0531
:1073700030911F05232B09F480E00895CF93DF930C
:10738000EB010E94B139882319F00E944B2CEB01CC
:10739000CE01DF91CF91089583E50E94B139882312
:1073A000E9F00F94344E6093B3087093B40880935F
:1073B000B5089093B6080E94393920E030E04AE7DA
:1073C00054E40F94E56A0F94E47260931B02709387
:1073D0001C0280931D0290931E02089580914D051A
:1073E00084FD0AC080914F0587FD06C0809150053D
:1073F000837011F40C9431F40E9420F488E50E940B
:107400006339882331F05F9A8091B1088E7F809331
:10741000B10889E50E946339882331F08A9A809106
:10742000B1088D7F8093B1088AE50E946339882373
:1074300059F08091080180958170809306018091B8
:10744000B1088B7F8093B10885E40E946339811174
:107450000C94D1260895CF93C62F0E94B13988236A
:1074600019F0CF910C945B2C8C2FCF910895CF9273
:10747000DF92EF92FF926A017B010E94B13988236B
:1074800031F0FF90EF90DF90CF900C943939C70125
:10749000B601FF90EF90DF90CF9008954F925F92EA
:1074A0006F927F928F929F92AF92BF92CF92DF9214
:1074B000EF92FF921F93CF93DF9300D01F92CDB72F
:1074C000DEB719821A821B821C82CE0101964C0102
:1074D0008DECC82E89E0D82E91EAE92E98E0F92E9D
:1074E00021ECA22E29E0B22E10E088E5810F0E9447
:1074F000B139F40181934F01882341F00E94393959
:107500002B013C0180912010882359F0F6018081E5
:107510009181A281B381F70180839183A283B38398
:1075200014C0812F0E94D324882309F4D0C0F6010F
:107530002081318142815381C301B2010F94717165
:10754000F70160837183828393831F5FF4E0CF0E22
:10755000D11C84E0E80EF11C94E0A90EB11C13309C
:1075600021F685E40E94B1398C83882309F4B9C0DF
:107570000E9439396B017C0183E00E94D324882367
:1075800071F02091D9093091DA094091DB095091CD
:10759000DC09C701B6010F9471716B017C01C092C7
:1075A000AD08D092AE08E092AF08F092B00880919A
:1075B0001906882359F18091A01682FF27C08C817B
:1075C000882321F18981811103C08A818823F1F008
:1075D0002DEC3CEC4CE45DE36091180970911909C5
:1075E00080911A0990911B090F9471719B01AC0154
:1075F0006091D5097091D6098091D7099091D809E9
:107600000F94D173181614F40F94325840E050E0E0
:10761000BA0186E40E94373A20E030E0A9010F94D5
:10762000D173181684F40E94393920E030E040E725
:1076300052E40F946B726093800270938102809386
:107640008202909383028091211083FD2CC080914F
:107650002010811128C080911408882321F12091E5
:10766000D9093091DA094091DB095091DC09609128
:10767000AD087091AE088091AF089091B0080F945A
:107680007071209121083091220840912308509177
:1076900024080F94717160932108709322088093DD
:1076A0002308909324080F900F900F900F90DF9174
:1076B000CF911F91FF90EF90DF90CF90BF90AF9050
:1076C0009F908F907F906F905F904F900895F501FD
:1076D0002081318142815381C301B2010F947071C5
:1076E0002FCF8091D9099091DA09A091DB09B0914F
:1076F000DC098093AD089093AE08A093AF08B093D7
:10770000B00855CFCF93DF93EB010E94B1398823A6
:1077100021F0DF91CF910C943539CE01DF91CF91DB
:107720000895CF93DF93C82FD62F0E94B1398823B5
:1077300021F0DF91CF910C946F2C8C2F0E94633934
:10774000811101C08D2FDF91CF910895EFE0F9E015
:1077500082EBDF011D928A95E9F708958091190661
:10776000811104C00E94A63B0D94F7598091A01688
:1077700082FD0D943258089580910F09882361F09D
:107780009091C009891308C08091A01683FF04C09E
:107790008DE499E00D94025A80E00895FC01238164
:1077A00021110C946BE90895CF92DF92EF92FF9232
:1077B0000F931F93CF9390913002913009F461C0E1
:1077C000662351F01092FC041092F8041092F90410
:1077D0001092FA041092FB04C82F0F94344EC090FC
:1077E000F804D090F904E090FA04F090FB049B01B7
:1077F000AC012C193D094E095F0969017A01F7FCBA
:1078000040C02091FC04C7FD15C04C2F0C2E000C6D
:10781000550B4C5F5F4FE22F022E000CFF0B4E17F3
:107820005F077CF144EFC42EDD24D394E12CF12CCE
:107830002C1734F438EEC32E33E0D32EE12CF12C88
:10784000C60ED71EE81EF91EC092F804D092F904A5
:10785000E092FA04F092FB04022F017010E084E23F
:10786000809FB001819F700D701B112460597C4F67
:1078700082E390E00E946A968091FC048F5F80937F
:10788000FC04CF911F910F91FF90EF90DF90CF906C
:1078900008950F931F9301E010E020E030E0082EE0
:1078A00004C0000F111F221F331F0A94D2F740910A
:1078B0005C0550915D0560915E0570915F05402B00
:1078C000512B622B732B40935C0550935D056093A5
:1078D0005E0570935F0590912F02891303C081E0CC
:1078E000809320101F910F9108954F925F926F9295
:1078F0007F928F929F92AF92BF92CF92DF92EF9240
:10790000FF920F931F93CF93DF93EC0120917E069C
:1079100030917F064091800650918106688179817F
:107920008A819B810F9470716B017C01209182068A
:107930003091830640918406509185066C817D814B
:107940008E819F810F9470714B015C01A70196019C
:1079500060910B0270910C0280910D0290910E02C9
:107960000F947F6A882309F450C0C0920B02D09212
:107970000C02E0920D02F0920E022091F004309180
:10798000F1044091F2045091F304C701B6010F9441
:10799000E56A2B013C010F9413736B017C0120E01D
:1079A00030E0A9010F947F6A87FD70C020E030E0CD
:1079B00040E450E4C701B6010F94D17318162CF4BB
:1079C000C12CD12CC0E4EC2EFE2CA7019601C301E2
:1079D000B2010F9470716093E8047093E90480938E
:1079E000EA049093EB04C701B6010F94DD72609333
:1079F000E604062E000C770B6F5F7F4F6430710535
:107A000014F064E070E06093E404D09109021091F6
:107A1000E604A501940160910F027091100280911B
:107A20001102909112020F947F6A811133C0D11319
:107A300081C02091CC043091CD044091CE0450916E
:107A4000CF046091E8047091E9048091EA04909178
:107A5000EB040F94E56A2091D0043091D104409159
:107A6000D2045091D3040F947171DF91CF911F9183
:107A70000F91FF90EF90DF90CF90BF90AF909F90CD
:107A80008F907F906F905F904F900895C12CD12C74
:107A900076019BCF80920F0290921002A092110269
:107AA000B09212022091F4043091F5044091F60452
:107AB0005091F704C501B4010F94E56A4B015C01D4
:107AC0000F9413736B017C0120E030E0A9010F9447
:107AD0007F6A87FDF3C020E030E040E450E4C70156
:107AE000B6010F94D17318162CF4C12CD12CB0E42C
:107AF000EB2EFE2CA7019601C501B4010F94707105
:107B00006093EC047093ED048093EE049093EF0483
:107B1000C701B6010F94DD726093E704062E000CD6
:107B2000770B6F5F7F4F6430710514F064E070E095
:107B30006093E504C091E704D11305C080910A0267
:107B40008C1709F470C08091E6049091E70490933B
:107B50000A02809309020C2E000CDD0B25E01203B3
:107B6000C0011124FC01EC0FFD1FEE0FFF1FEE0FF3
:107B7000FF1FE65EF94F20813181428153812093BE
:107B8000E0043093E1044093E2045093E304009155
:107B9000E504002E000C110BFC01E00FF11FEE0FAD
:107BA000FF1FEE0FFF1FE65EF94F6081718182813A
:107BB00093810F9470716093DC047093DD04809363
:107BC000DE049093DF042091E40435E02303F00108
:107BD0001124CE0FDF1FCC0FDD1FCC0FDD1FC65EC3
:107BE000D94F288139814A815B812093D804309311
:107BF000D9044093DA045093DB04E00FF11FEE0F39
:107C0000FF1FEE0FFF1FE65EF94F608171818281D9
:107C100093810F9470716093D4047093D504809312
:107C2000D6049093D7048090EC049090ED04A0903B
:107C3000EE04B090EF042091DC043091DD0440911B
:107C4000DE045091DF04C501B4010F94E56A209170
:107C5000E0043091E1044091E2045091E3040F9478
:107C600071716B017C01C092D004D092D104E0927A
:107C7000D204F092D3042091D4043091D5044091E1
:107C8000D6045091D704C501B4010F94E56A209140
:107C9000D8043091D9044091DA045091DB040F9458
:107CA0007171A70196010F9470716093CC04709369
:107CB000CD048093CE049093CF04BBCEC12CD12CA5
:107CC000760118CF1F93CF93DF93CDB7DEB72C97F4
:107CD0000FB6F894DEBF0FBECDBF182F882379F002
:107CE00020E030E0A90160918606709187068091BE
:107CF0008806909189060F947F6A8823F9F0809115
:107D0000DC088117D9F00E9420F48CE0EFE8F2E063
:107D1000DE01119601900D928A95E1F7CE01019650
:107D20000E94753C8091DC08882391F08DEC99E0ED
:107D30000E9443F41092DC080F943C092C960FB675
:107D4000F894DEBF0FBECDBFDF91CF911F91089594
:107D500081E08093DC088DEC99E00E9470F3ECCF19
:107D600080E00E94623E109282061092830610927A
:107D700084061092850610927E0610927F0610925D
:107D800080061092810610928A0610928B0610923D
:107D90008C0610928D06109286061092870610921D
:107DA000880610928906EAE1F6E02EE736E080E0E8
:107DB00090E0A0ECBFE780839183A283B3838483A8
:107DC0009583A683B78380879187A287B3878487AB
:107DD0009587A687B787808B918BA28BB38B749680
:107DE0002E173F0741F708954F925F926F927F924F
:107DF0008F929F92AF92BF92CF92DF92EF92FF92BB
:107E00001F93CF93DF93EC01162F2091D808309168
:107E1000D9084091DA085091DB08688179818A811C
:107E20009B810F947F6A882309F4AEC0B090DC0870
:107E300080E00E94623EC880D980EA80FB8020E01A
:107E400030E0A901C701B6010F94D17318161CF0D8
:107E5000C12CD12C7601C092D808D092D908E092DA
:107E6000DA08F092DB082DEB37E346E855EBC70163
:107E7000B6010F94D17387FD0BC02DEB37E346E8B5
:107E800055E3C701B6010F947F6A18160CF078C04D
:107E9000A701960160E070E080E89FE30F946B72A9
:107EA0006093160570931705809318059093190534
:107EB00080EF9FEFA9E7B4EC80931A0590931B0520
:107EC000A0931C05B0931D05BB2009F45DC0409034
:107ED000CD095090CE096090CF097090D009809064
:107EE000D1099090D209A090D309B090D409C09044
:107EF000D509D090D609E090D709F090D80981E053
:107F00000E94623E112309F43FC02091CD093091B7
:107F1000CE094091CF095091D009C301B2010F940D
:107F20007F6A81111CC02091D1093091D209409102
:107F3000D3095091D409C501B4010F947F6A81110E
:107F40000EC02091D5093091D6094091D7095091A2
:107F5000D809C701B6010F947F6A8823A9F0DF9181
:107F6000CF911F91FF90EF90DF90CF90BF90AF9097
:107F70009F908F907F906F905F904F900D94BD1069
:107F800060E070E0CB018CCFDF91CF911F91FF902B
:107F9000EF90DF90CF90BF90AF909F908F907F90A9
:107FA0006F905F904F9008958F929F92AF92BF9283
:107FB000CF92DF92EF92FF92C0908606D090870614
:107FC000E0908806F090890620E030E0A901C70122
:107FD000B6010F947F6A8823E1F1A701960160E062
:107FE00070E080E89FE30F946B726B017C018090DE
:107FF0008A0690908B06A0908C06B0908D0620E0AB
:1080000030E0A901C501B4010F947F6A882329F1EA
:10801000A501940160E070E080E89FE30F946B722B
:10802000C092F004D092F104E092F204F092F304D2
:108030006093F4047093F5048093F6049093F7042E
:10804000FF90EF90DF90CF90BF90AF909F908F9078
:108050000895C12CD12C7601CACF60E070E0CB012D
:10806000DFCFEFE6F0E08081826080830895809129
:10807000B7089091B808892B79F48091B70890914E
:10808000B808892B49F42091B7083091B80881E0ED
:10809000232B19F480E0089581E00895CF92DF92B8
:1080A000EF92FF926B017C0183E3C816D104E104D7
:1080B000F10470F082E3C81AD108E108F10862E324
:1080C00070E080E090E00F94014E0F943E09ECCFF9
:1080D000C701B6010F94014EFF90EF90DF90CF9053
:1080E0000D943E098091A90681110AC08091D6089D
:1080F000813041F08091A01682FB882780F9089595
:1081000080E0089581E008955F9A8091B1088E7FA4
:108110008093B1088A9A8091B1088D7F8093B108CD
:108120008091080180958170809306018091B1084B
:108130008B7F8093B1080C94D1269091A01693FB6D
:10814000882780F993FF06C081E09091081891116B
:1081500001C080E008958091A906811110C080912E
:10816000D608823061F00E949D40882349F08091BA
:10817000A01682FB882780F991E08927089581E085
:1081800008950E94AB4081110DC010925C051092C1
:108190005D0510925E0510925F05109260058FEFED
:1081A0000E94722A0D94C01781E00D943017EBE005
:1081B000FAE010821182089581E00895DC01EC91CB
:1081C0008E2F90E0FC01EE0FFF1FE80FF91FEF521A
:1081D000FA4E80818F77808308958F929F92AF921D
:1081E000BF92CF92DF92EF92FF920F93CF93DF93E4
:1081F0001F92CDB7DEB75C017B0149016B01C40E54
:10820000D51EF501808191810F949D708983002393
:1082100011F0F7018083BE016F5F7F4FC4010F949F
:108220001C30F50180819181019691838083FFEF5D
:10823000EF1AFF0AEC14FD0421F780E00F90DF91A4
:10824000CF910F91FF90EF90DF90CF90BF90AF90C4
:108250009F908F900895009781F41092900082E093
:10826000809391001092950010929400C19A809191
:1082700071008260809371000895019761F41092FB
:10828000A00082E08093A1001092A5001092A400AB
:1082900089BB8093720008957F928F929F92AF92D4
:1082A000BF92CF92DF92EF92FF920F931F93CF93E3
:1082B000DF93EC017B018881883108F0C3C090E036
:1082C000FC01EE0FFF1FE80FF91FEF52FA4E8081FD
:1082D0008F770F94DA3119821A8288812CE0622F0D
:1082E0000F942671829FB001112430E020E0AB0191
:1082F000420F531FFA01EE0FFF1FE40FF51FEF525D
:10830000FA4E908197FD08C02F5F3F4F2C3031050A
:1083100071F790E00E942B417880072D10E06801F2
:10832000CC0CDD1CF601E00FF11FEF52FA4E8081FC
:108330008068808377FC86C080E2E81682E0F806D9
:108340000CF03FC08A8128E532E0281B310987FD07
:108350003395220F331F220F331F032E000C440BC3
:10836000550B898178E8872E912C881A910887FD12
:108370009394880C991C880C991C092C000CAA0851
:10838000BB0860E070E0CB01F7FC0AC0B701653BB9
:10839000710514F064EB70E0072E000C880B990B4C
:1083A000281939094A095B090F94B37024EB30E0AE
:1083B00040E050E00F94E570820E931EA41EB51E9F
:1083C000740187E18715D8F0298188E890E0821B45
:1083D000910927FD9395880F991F880F991FE8161B
:1083E000F90604F502972FB7F894E601C00FD11FE4
:1083F000CF52DA4E880F991F9A8389832FBF62E389
:1084000070E080E090E0DF91CF911F910F91FF909D
:10841000EF90DF90CF90BF90AF909F908F907F9024
:108420000C944E402A8188E592E0821B910927FD39
:108430009395880F991F880F991FE816F90694F6EF
:10844000C701D0CFDF91CF911F910F91FF90EF9097
:10845000DF90CF90BF90AF909F908F907F900895C6
:10846000CF93DF93EB01682F70E08AE196E10E94E1
:108470004C41688179818A819B81643F21E0720748
:108480008105910520F464EF71E080E090E00E94A6
:108490004E4089B182FB882780F9DF91CF91089502
:1084A000CF93DF9300D01F92CDB7DEB78EEE92E070
:1084B000A0E0B0E089839A83AB83BC83BE016F5F89
:1084C0007F4F8AE50E9430420F900F900F900F90DF
:1084D000DF91CF910895CF93DF9300D01F92CDB756
:1084E000DEB78EEE92E0A0E0B0E089839A83AB83A2
:1084F000BC83BE016F5F7F4F8AE00E9430420F90C5
:108500000F900F900F90DF91CF910895CF93DF934D
:1085100000D01F92CDB7DEB784EF91E0A0E0B0E0CD
:1085200089839A83AB83BC83BE016F5F7F4F8CE3EB
:108530000E9430420F900F900F900F90DF91CF91DB
:108540000895CF93DF9300D01F92CDB7DEB784EFAD
:1085500091E0A0E0B0E089839A83AB83BC83BE0145
:108560006F5F7F4F80EA0E9430420F900F900F9014
:108570000F90DF91CF9108951F920F920FB60F9237
:1085800011240BB60F922F933F934F935F936F93EA
:108590007F938F939F93AF93BF93EF93FF9348EA9B
:1085A00050E064EA70E081E090E00E947F2CFF914F
:1085B000EF91BF91AF919F918F917F916F915F915B
:1085C0004F913F912F910F900BBE0F900FBE0F90C8
:1085D0001F9018951F920F920FB60F9211240BB691
:1085E0000F922F933F934F935F936F937F938F934C
:1085F0009F93AF93BF93EF93FF9348E950E064E9F3
:1086000070E090E080E00E947F2CFF91EF91BF919D
:10861000AF919F918F917F916F915F914F913F911A
:108620002F910F900BBE0F900FBE0F901F901895BB
:108630009091C00095FFFCCF8093C6000895CF9322
:10864000DF93EC018991882319F00E941843FACF37
:108650008DE00E9418438AE0DF91CF910C9418437B
:10866000CF92DF92EF92FF92CF936B017C01C42FE8
:108670004A3069F4F7FE0BC0F094E094D094C094B3
:10868000C11CD11CE11CF11C8DE20E9418434C2F2F
:10869000C701B601CF91FF90EF90DF90CF900D947E
:1086A0009457CF93DF93EC01FE01849121968823A8
:1086B00019F00E941843F8CFDF91CF9108950F93DE
:1086C0001F93CF938C01C62F89E795E10E945143F8
:1086D000C8010E9451438AE30E94184380E38C0F33
:1086E0000E9418438AE0CF911F910F910C94184378
:1086F0008CEF96E10E94514360E08CEE96E10E947F
:108700005F4360E087ED96E10E945F4361E080EDAA
:1087100096E10E945F4361E085EC96E10E945F4331
:1087200061E085EB96E10E945F4360E08CEA96E1B0
:108730000E945F4361E082EA96E10E945F4361E04C
:1087400088E996E10E945F4361E081E996E10E9439
:108750005F4361E089E896E10E945F4361E08BE757
:1087600096E10E945F4361E08DE696E10E945F43DF
:1087700060E08EE596E10E945F4360E080E596E16F
:108780000E945F4360E08AE396E10E945F4361E0FC
:1087900089E296E10E945F4361E08AE196E10E94EE
:1087A0005F4361E083E196E10E945F4360E08CE01B
:1087B00096E10E945F4361E083E096E10E945F439F
:1087C00061E08EEE95E10E945F4361E080EE95E10D
:1087D0000E945F4361E08DEC95E10E945F4360E0A1
:1087E00080EC95E10E945F4361E08BEB95E10E9494
:1087F0005F4361E08EEA95E10E945F4360E08AE9B1
:1088000095E10E945F4360E087E895E10E945F4345
:1088100060E084EA96E10E94D024682F61708EE7C0
:1088200095E10C945F4380914D05827149F48091EC
:108830004F058C7829F480915005837009F475C038
:1088400082E40E946339882351F00E942A2C6093AD
:10885000321070933310809334109093351083E569
:108860000E946339882351F00E9439396093621065
:1088700070936310809364109093651084E50E9458
:108880006339882351F00E943939609366107093E0
:108890006710809368109093691088E50E9463398F
:1088A000882351F00E9439396093E3097093E409F9
:1088B0008093E5099093E60989E50E94633988234E
:1088C00051F00E9439396093E7097093E809809369
:1088D000E9099093EA098AE50E9463398823B1F097
:1088E0000E9439396093EB097093EC098093ED098C
:1088F0009093EE092DEC3CEC4CEC5DE30F947F6A19
:10890000181624F08FE290E10E94514385E40E9402
:108910006339882351F00E9439396093EF097093CD
:10892000F0098093F1099093F2090895AF92BF92F4
:10893000CF92DF92EF920F931F93CF93DF935B0160
:10894000EA016901882309F463C085E190E10E948E
:108950005143F501608171818281938146E00F94DA
:108960007321E1100BC08CE090E10E9451436881BB
:1089700079818A819B8146E00F94732185E090E1A3
:108980000E945143F601608171818281938143E0AD
:108990000F9473218EEF9FE00E945143F801608194
:1089A00071818281938143E00F94732185EF9FE071
:1089B0000E945143F6012081318142815381F801A7
:1089C00060817181828193810F94707143E00F9473
:1089D0007321EE20F9F08AE00E94184380EE9FE0B8
:1089E0000E945143688179818A819B8146E00F947E
:1089F00073218AE00E9418438AE0DF91CF911F9192
:108A00000F91EF90DF90CF90BF90AF900C941843F0
:108A1000E110E4CFDF91CF911F910F91EF90DF90A4
:108A2000CF90BF90AF9008950F931F93CF938C0179
:108A3000C62F80E89AE00E945143C8010E9451432A
:108A4000CC2331F08AE0CF911F910F910C94184301
:108A5000CF911F910F9108950F931F93CF938C0186
:108A6000C62F60E080E99AE00E941445C8010E9488
:108A70005143CC2331F08AE0CF911F910F910C9498
:108A80001843CF911F910F91089561E088E99AE012
:108A90000C942C45EF92FF920F931F93CF937C0180
:108AA0008B01C42F60E080E99AE00E941445C70161
:108AB0000E94514380E20E941843C8010E94514322
:108AC000CC2319F08C2F0E9418438AE0CF911F917C
:108AD0000F91FF90EF900C941843DF92EF92FF926A
:108AE0000F931F93CF93DF93D82E7B018A01E90167
:108AF0000E944545D092B90840E0B70186EB95E465
:108B00000E944A450115110531F040E0B8018FEA95
:108B100095E40E944A45209731F040E0BE018FEA7B
:108B200095E40E944A4561E08AEA95E4DF91CF919D
:108B30001F910F91FF90EF90DF900C942C4561E016
:108B40008AE89AE00C941445AF92BF92CF92DF92DC
:108B5000EF92FF920F931F93CF93DF9387ED99E0EE
:108B60000E945143C0E0D7E0D15021F080E20E9442
:108B70001843FACF8C2F0F94FB57CF5FC53099F76E
:108B80008AE00E9418430AE116E0C0E080E20E94F9
:108B900018438C2F0F94FB575801D5E080E20E94B8
:108BA0001843F501C080D180E280F380A7019601CF
:108BB000C701B6010F946374882369F180E20E94B3
:108BC00018438DE30E9418438DE30E9418438DE300
:108BD0000E9418438DE30E9418438DE30E941843BE
:108BE000D150F4E1AF0EB11CD111D8CF8AE00E9470
:108BF0001843CF5F0C5F1F4FC53041F68AE0DF910D
:108C0000CF911F910F91FF90EF90DF90CF90BF9089
:108C1000AF900C94184320E030E0A901C701B601E1
:108C20000F94D17387FD03C08BE20E94184343E089
:108C3000C701B6010F947321D3CF811107C081E61C
:108C400090E10E9451438AE00C94184385E690E13C
:108C5000F8CFCF93DF93EB010E945143CE01DF9118
:108C6000CF910D940258CF93C62F0E9451438C2F61
:108C7000CF910D94FB57CF92DF92EF92FF926A0152
:108C80007B010E94514342E0C701B601FF90EF9083
:108C9000DF90CF900D94732180914E0587FD2BC0FE
:108CA00080914F058E7039F54091561050915710B4
:108CB00060915810709159108FE190E10E943B46ED
:108CC00040915A1050915B1060915C1070915D1052
:108CD0008CE190E10E943B4640915E1050915F1004
:108CE000609160107091611088EF91E30E943B46A3
:108CF0008AE00C94184383E50E94B139882391F0EF
:108D00000E94393960935610709357108093581011
:108D10009093591060935E1070935F108093601071
:108D20009093611080E50E94B139882351F00E9430
:108D30003939609356107093571080935810909360
:108D4000591082E50E94B139882351F00E943939C7
:108D500060935A1070935B1080935C1090935D1039
:108D600084E50E94B139882351F00E94393960931B
:108D70005E1070935F10809360109093611008955F
:108D8000CF92DF92EF92FF926A017B010E945143E2
:108D90004AE0C701B601FF90EF90DF90CF900C94AE
:108DA00030432F923F924F925F926F927F928F92B9
:108DB0009F92AF92BF92CF92DF92EF92FF920F936A
:108DC0001F93CF93DF93CDB7DEB7C654D1090FB64B
:108DD000F894DEBF0FBECDBF70E060E085E40E9476
:108DE000823B182F8F3F09F483C08823E9F084E386
:108DF0009AE1CA5BDF4F0FB6F894DEBF0FBECDBF5E
:108E0000DF91CF911F910F91FF90EF90DF90CF9066
:108E1000BF90AF909F908F907F906F905F904F909A
:108E20003F902F900C94514324EB30E03A832983F8
:108E300083E50E94B139882321F00E9435399A8355
:108E4000898365E070E083E40E94823B8AA760E04A
:108E500085E50E94913B25968FAF259760E087E2DC
:108E60009AE10E9447CBA981BA81BD01BB0F880B53
:108E7000990B0F94866A6D837E838F8327969FAFAD
:108E800027970F94344E688B798B8A8B9B8B1F3F6F
:108E900009F045C420E030E04CE053E46D817E8170
:108EA0008F8127969FAD27970F94D17318160CF0DA
:108EB000AAC18CEF99E10E945143CA5BDF4F0FB604
:108EC000F894DEBF0FBECDBFDF91CF911F910F9100
:108ED000FF90EF90DF90CF90BF90AF909F908F90DA
:108EE0007F906F905F904F903F902F900D947743BD
:108EF00046E450E05A8349839BCF1FAEAFC124960E
:108F0000EEADFFAD2497808383C2FBEE4F2E512C34
:108F1000612C712C04C384E190E0A0E0B0E08C8B64
:108F20009D8BAE8BBF8BE4E14E2E512C612C712CAE
:108F300004C34C8A5D8A6E8A7F8AFFC22496EEAD96
:108F4000FFAD24978083D4C389819A81AB81BC8192
:108F500029A93AA94BA95CA9821B930BA40BB50BB9
:108F6000B7FD59C08FAD0F9417228AE00E941843B5
:108F700089819A81AB81BC818053984FAF4FBF4F9D
:108F800089AB9AABABABBCAB9DA9911177C02EA9B5
:108F90003FA948AD59ADB101802F26969FAD2697C8
:108FA0000F94D17318160CF053C020E030E040E06D
:108FB00050E4B101802F26969FAD26970F947171D2
:108FC0006EAB7FAB88AF99AF2CA53DA54EA55FA535
:108FD00089819A81AB81BC81280F391F4A1F5B1F91
:108FE0002AAF3BAF4CAF5DAF20E030E040EC50E447
:108FF0006D817E818F8127969FAD27970F94707129
:109000009101402F26965FAD26970F947F6A881FA7
:109010008827881F8DAB88899989AA89BB89C8163A
:10902000D906EA06FB0610F4D701C60129813A8168
:109030004B815C81281B390B4A0B5B0BDA01C901A0
:1090400081389F44A241B105A8F188E499E10EC29C
:1090500089819A81AB81BC812AAD3BAD4CAD5DADC0
:10906000821B930BA40BB50B47E95BE366EA7BE33A
:10907000B7FDD1CF812F0E9493EDCDCF20E030E01E
:1090800040EF51E46D817E818F8127969FAD2797B8
:109090000F9470719B01AC01B101802F26969FAD9A
:1090A00026970F947F6A87FFB6CF43E45CE363E5BE
:1090B0007CE3E0CF4AA55BA5888D998D48175907B9
:1090C0000CF09EC003970CF49BC08BEE98E10E94BD
:1090D00051431F3F09F076C0ABEDB8E1BA83A983D5
:1090E0008AEC98E10E94514389819A810E94514300
:1090F000488559856A857B8587EE98E10E943B46C5
:109100008AE00E9418438AEC98E10E9451438981C9
:109110009A810E94514349A15AA16BA17CA183EE7F
:1091200098E10E943B468AE00E9418438AEC98E14D
:109130000E94514389819A810E945143B501A40143
:109140008FED98E10E943B468AE00E9418432596E5
:10915000FFAD2597FF2391F12CEA35EC47E25EE362
:1091600069A17AA18BA19CA10F94E56A6B017C0196
:109170002CEA35EC47E25EE3C501B4010F946B7253
:10918000288539854A855B851F3F09F52093E608C8
:109190003093E7084093E8085093E908C092EA0842
:1091A000D092EB08E092EC08F092ED086093EE08A4
:1091B0007093EF088093F0089093F10881E080931A
:1091C00065027BCEE8EEF4E4FA83E98389CF20934D
:1091D0009515309396154093971550939815C09216
:1091E0009915D0929A15E0929B15F0929C15609378
:1091F0009D1570939E1580939F159093A015DECFBB
:109200000E9484CF80C088EE99E10E9451430E9461
:1092100086EC8FE78093E50824EB30E0A8EEB3E01E
:109220000F9417716CA77DA78EA79FA728893989EE
:109230004A895B89260F371F481F591F2AAF3BAF4A
:109240004CAF5DAF1092650281E08093740232E012
:10925000310F3EAF323008F450CE1FAFC888D988E6
:10926000EA88FB88C9AADAAAEBAAFCAA812C912C6D
:10927000540189A29AA2ABA2BCA288869986AA862A
:10928000BB868FE790E0A0E0B0E08C8B9D8BAE8B2F
:10929000BF8B1C8690E49A8FACE1AB8FB6E4BC8F99
:1092A0001D8E1E8E1F8E18A23FE7432E512C612C5F
:1092B000712C1DAA8EAA9FAAA8AEB9AE1EA21FA28B
:1092C00018A619A6E1E0EDA3198E188E212C312CD9
:1092D00000E026961FAE2697F5E11F02C00111247B
:1092E0009C0124573A4E22963FAF2EAF2297285F1B
:1092F0003F4F24963FAF2EAF24974AA5042E000C73
:10930000550B5BA74AA780917402882309F4B0C06B
:109310000F94344E69837A838B839C835091A70684
:1093200058AB552309F48BC00E9439ED6091E108D8
:109330007091E2081F3F39F02296AEADBFAD229783
:1093400014966D917C91072E000C880B990B0F944D
:10935000866A1B01082F26969FAF26972D8D3E8D7E
:109360004F8D58A126969FAD26970F94D17318164E
:109370003CF42D8E3E8E0F8F2696BFAD2697B8A358
:109380002C853A8D4B8D5C8DB101802F26969FAD3B
:1093900026970F947F6A87FF07C02C863A8E0B8F23
:1093A0002696EFAD2697EC8FFDA19101402F2696D2
:1093B0005FAD26976D817E818F8127969FAD279720
:1093C000FF2309F45AC00F947F6A87FF38C0498190
:1093D0005A816B817C814C195D096E097F09DB0123
:1093E000CA0188589341A109B109B7FD28C08C89E9
:1093F0009D89AE89BF8984199509A609B709B595D4
:10940000A795979587951F3F09F079CD8093E5083B
:109410004EA35FA368A779A7FD81FD8F2E812E8FB4
:109420003F813F8F27964FAD279748A389819A8127
:10943000AB81BC81888B998BAA8BBB8B1DA220E052
:1094400030E040EF51E46D817E818F8127969FADA2
:1094500027970F9471719101402F26965FAD269743
:109460000F947F6A87FF70CD86E699E10E94514391
:10947000109274020E9486ECA1CE0F94D17318163C
:10948000F4F689819A81AB81BC81288939894A891E
:109490005B89821B930BA40BB50BAC01BD01485833
:1094A00053416109710977FDCACF488D598D452B0C
:1094B00009F40DC1CEA0DFA0E8A4F9A4C80ED91EFE
:1094C000EA1EFB1E2EA13FA148A559A5281B390B5A
:1094D0004A0B5B0BC301B2010F94B370A701960155
:1094E0000F94E5704C885D886E887F88420E531E0D
:1094F000641E751E54E145165104610471040CF498
:109500000ACD8CEE48165104610471040CF0FDCCB8
:1095100090E849165104610471040CF40ACD4C8A98
:109520005D8A6E8A7F8A2EEF30E040E050E0241999
:1095300035094609570929013A014C895D896E8927
:109540007F8980EE99E10E94C046B301A2018BEDB4
:1095500099E10E94C0464C855A8D6B8D7C8D84EDBF
:1095600099E10E943B464D8D5E8D6F8D78A18DEC0B
:1095700099E10E943B46A88DB98D13970CF4A7C0C2
:10958000C301B2010F94866A20E030E040E850E465
:109590000F94E56A4B015C012C853A8D4B8D5C8DF7
:1095A0006D8D7E8D8F8D98A10F9470712BED3FE0A6
:1095B00049E450E40F94E56A20E030E040E05FE3E6
:1095C0000F94E56A9B01AC01C501B4010F946B7265
:1095D0006C877D878E879F87C701B6010F94866A47
:1095E0002FE632E143E85AE30F94E56A6B017C0110
:1095F0001E3F59F02AE939E949E15FE3812C912CBA
:10960000A12C6EE3B62E1F3F59F42DEC3CEC4CE43C
:109610005EE37BEA872E7AEA972EA92C7EE3B72EAB
:109620006C857D858E859F850F94E56A688779872F
:109630008A879B879B01AC010F947171A7019601EA
:109640000F946B7269A37AA38BA39CA32885398599
:109650004A855B85C701B6010F94E56AA5019401AF
:109660000F94E56A4B015C014C855D856E857F85B5
:1096700087EC99E10E943B46B701A60181EC99E194
:109680000E943B468AE00E941843BEAD82EB99E1FE
:10969000B23010F083EA99E10E9451434885598520
:1096A0006A857B858DE999E10E943B4649A15AA1D3
:1096B0006BA17CA187E999E10E943B46B501A40119
:1096C00081E999E10E943B468AE00E9418438C8917
:1096D0009D89AE89BF89840D951DA61DB71DB595C1
:1096E000A795979587951F3F09F028CC8093E508AB
:1096F000288D398D2F5F3F4F398F288F3D813C87D3
:109700004E814A8F5F815B8F27968FAD27978C8F15
:10971000C980DA80EB80FC8098A99DA390CEE12ED1
:10972000012E000CFF08F70183E0EE0FFF1F8A9562
:10973000E1F7E459FD4F668177816F507109072E7B
:10974000000C880B990B0F94866A9B01AC016D810C
:109750007E818F8127969FAD27970F94D17318161E
:109760000CF4A7CB88EE99E10E9451430E9486EC4D
:1097700085E18E9DF0018F9DF00D1124E457FA4E86
:109780008FE7808722E330E049CDCF93DF93EB0171
:109790000E945143CE01DF91CF910D94D3313F927E
:1097A0004F925F926F927F928F929F92AF92BF92F1
:1097B000CF92DF92EF92FF920F931F93CF93DF939D
:1097C00080914F0587FD38C0809150058370A1F5C9
:1097D000C0912916D0912A16488159816A817B81CE
:1097E0008BE698E10E943B464C815D816E817F81D2
:1097F00084E696E40E943B46409125165091261639
:10980000609127167091281681E696E40E943B46E7
:109810008AE0DF91CF911F910F91FF90EF90DF9041
:10982000CF90BF90AF909F908F907F906F905F9000
:109830004F903F900C94184360901D1670901E1628
:1098400080901F1690902016A0902116B09022169E
:109850000091231610912416C0902516D09026163C
:10986000E0902716F090281688E50E94B139C82F9D
:10987000882309F49AC00E943939362E472E582E73
:10988000D92F20E030E046E953EC0F94D17387FDE7
:109890000DC020E030E046E953E4632D742D852DA2
:1098A0009D2F0F947F6A18160CF081C06CE271E056
:1098B00088E598E10E94C54B6CE271E083E598E190
:1098C0000E94C54B80E598E10E945143C0E089E5C4
:1098D0000E94B139882361F10E943939362E472E12
:1098E000582ED92F20E030E046E953EC0F94D17385
:1098F00087FD0DC020E030E046E953E4632D742D70
:10990000852D9D2F0F947F6A18160CF055C06CE2C0
:1099100071E08DE398E10E94C54B6CE271E088E351
:1099200098E10E94C54B85E398E10E945143C0E055
:109930008AE50E94B139882309F443C00E9439396D
:109940006B017C0120E030E040E151EC0F94D173D9
:1099500087FD0AC020E030E040E151E4C701B601D4
:109960000F947F6A18166CF567EF7FEF83E298E13A
:109970000E94C54B69E070E08EE198E10E94C54B02
:109980008BE198E1DF91CF911F910F91FF90EF90C4
:10999000DF90CF90BF90AF909F908F907F906F900F
:1099A0005F904F903F900C945143C1E090CF632C57
:1099B000742C852C9D2E8BCFA32CB42C052D1D2F04
:1099C000B7CFCC23E1F0C301D40180931D1690934F
:1099D0001E16A0931F16B0932016C501D8018093C0
:1099E000211690932216A0932316B0932416C092AA
:1099F0002516D0922616E0922716F0922816DF91AF
:109A0000CF911F910F91FF90EF90DF90CF90BF907B
:109A1000AF909F908F907F906F905F904F903F900E
:109A200008952F923F924F925F926F927F928F9202
:109A30009F92AF92BF92CF92DF92EF92FF920F93DD
:109A40001F93CF93DF93CDB7DEB7CB54D1090FB6B9
:109A5000F894DEBF0FBECDBF2DB73EB739AF28AFEC
:109A600087E00F94FC2C81110BC061E086E50E9419
:109A70002B3A8DA3853060F08BEB9FE00E94514321
:109A8000A8ADB9AD0FB6F894BEBF0FBEADBF40C311
:109A90003DA1332321F08BE99FE00E9451436AE00E
:109AA00080E50E942B3A182F8CEF810F8F3218F02F
:109AB00087E79FE0E3CF60E085E40E94913B882345
:109AC00009F448C081E08FABE0902916F0902A1687
:109AD000D7012D913D914D915C916091CD0970918F
:109AE000CE098091CF099091D0090F947171AB018B
:109AF000BC0188E50E94373A69877A878B879C8703
:109B0000F70124813581468157816091D109709197
:109B1000D2098091D3099091D4090F947171AB014E
:109B2000BC0189E50E94373A6D877E878F87988BC5
:109B3000BE01635F7F4FCE0109960E941534382E17
:109B400081110BC063E683E69FE00E9447CB8BE464
:109B50009FE094CF92E09FABB7CF8CE40E94633933
:109B6000082F882309F431C10E945B2C8EA3803119
:109B700018F084E29FE082CFFEA1F13009F427C102
:109B800060E083E50E94913B8AAF882321F00111B8
:109B900002C037E03EA38DA1833020F08AE09FE031
:109BA0000E9451439091DC089DAF80E00E94623E8C
:109BB0000F94F9061D8A1E8A1F8A188E198E1A8E16
:109BC0001B8E1C8E83EF9FE4A3ECB7E48D8F9E8FDA
:109BD000AF8FB8A383EF9FE4A3ECB7EC89A39AA35C
:109BE000ABA3BCA3A12FB0E0BCA7ABA7EDB7FEB75A
:109BF00024E0129FE019F10911240FB6F894FEBF7A
:109C00000FBEEDBF8DB79EB701969CAF8BAF2DA158
:109C10004FA9BE01635F7F4FCE0109960F94F244B6
:109C20009B01AC010F946374811162C20F94344E96
:109C3000611571058105910511F00F940566212CC0
:109C40001BAA1CAA1DAA1EAAAEA1A150BB0B2C9632
:109C5000BFAFAEAF2C97E22DF0E0F8A7EFA32BA596
:109C60003CA5E217F3070CF074C23196FEA7EDA7EE
:109C70003F932F93FF93EF9386EF9EE09F938F93F5
:109C800080E09FE09F938F931F920E942CCB8DB713
:109C90009EB709960FB6F8949EBF0FBE8DBF9EA1CA
:109CA000992309F458C10F94B6652AE030E040E0EA
:109CB00050E00F94E5700F94866A20E030E040EAAF
:109CC00050E40F94D1730FEF1FEF181614F001E05A
:109CD00010E00F94B66528E631E040E050E00F94C4
:109CE000E5700F94866A2B013C010F94B66520E263
:109CF00030E040E050E00F94E5706B5F7F4F8F4F96
:109D00009F4F0F94866A4B015C01ADA1A430D1F442
:109D1000BC01A40188EE9EE00E943B46B301A20173
:109D200080EE9EE00E943B468AED9EE00E945143F9
:109D30000130110519F483E40E94184386ED9EE07A
:109D40000E945143312CC801110FAA0BBB0B2A965C
:109D50008CAF9DAFAEAFBFAF2A972C96AEADBFAD67
:109D60002C973A161B060CF0F6C02A966CAD7DAD0A
:109D70008EAD9FAD2A970F94866A6B017C01BAADB8
:109D8000BB2341F1AC019B010F94717120E030E0E5
:109D900040E952E40F94E56A9B01AC01C301B201B2
:109DA0000F9471712B013C0120E030E044EB53E44F
:109DB0000F94D1731816FCF420E030E044EB53E428
:109DC000C301B2010F947071EDCF1EA2D9CE22E073
:109DD0002EA3D6CE0F94B66524E130E040E050E0EB
:109DE0000F94E570675E7F4F8F4F9F4F0F94866A89
:109DF000A7019601CFCF20E030E0A901C301B20155
:109E00000F947F6A87FF0BC020E030E044EB53E4FF
:109E1000C301B2010F9471712B013C01ECCF009191
:109E2000291610912A16F80124813581468157811F
:109E30006D857E858F8598890F94707122966CAFA1
:109E40007DAF8EAF9FAF22972BED3FE049E450E40A
:109E5000C301B2010F94E56A20E030E044E353E42B
:109E60000F946B726B017C010F9466726FA778ABD5
:109E700089AB9AABD8012D913D914D915C9169854B
:109E80007A858B859C850F94707126966CAF7DAF1B
:109E90008EAF9FAF2697A50194016FA578A989A9D8
:109EA0009AA90F94E56A9B01AC0126966CAD7DAD35
:109EB0008EAD9FAD26970F94717169837A838B83E2
:109EC0009C83C701B6010F941174A50194010F94EE
:109ED000E56A22962CAD3DAD4EAD5FAD22970F9455
:109EE00071716D837E838F8398874BE351E070E0BF
:109EF00060E0CE0101960E9451ED46E351E070E032
:109F000060E0CE0105960E9451EDBDA1B43099F4F8
:109F100049815A816B817C818AEC9EE00E943B469C
:109F20004D815E816F81788584E696E40E943B4690
:109F30008AE00E941843198A1A8A1B8A1C8AAE0179
:109F40004F5E5F4FBE016B5F7F4FCE0101960F9456
:109F5000EF07339402CF20E04FA9BE01635F7F4F2C
:109F6000CE0109960F94F2444B015C01312CAC01F7
:109F70009B010F946374811102C033243394A501B3
:109F80009401C501B4010F9463748111E2C0EFA183
:109F9000F8A5EE0FFF1FEE0FFF1F2BAD3CADE20F3C
:109FA000F31F80829182A282B382A50194016D8DFC
:109FB0007E8D8F8D98A10F94D173181624F48D8EF9
:109FC0009E8EAF8EB8A2A501940169A17AA18BA142
:109FD0009CA10F947F6A87FF04C089A29AA2ABA2BA
:109FE000BCA2A50194016BA97CA98DA99EA90F947F
:109FF00071716BAB7CAB8DAB9EABADA5BEA5BD014E
:10A00000BB0F880B990B0F94866A6FA378A789A75B
:10A010009AA79B01AC016BA97CA98DA99EA90F945D
:10A020006B722B013C014D8A5E8A6F8A788EEBAD94
:10A03000FCADF8ABEFA710E0C12CD12C7601AFA599
:10A04000B8A96D917D918D919D91B8ABAFA7A301FA
:10A0500092010F9470719B01AC010F94E56A9B0112
:10A06000AC01C701B6010F9471716B017C011F5FD8
:10A07000211628F72FA138A549A55AA50F946B7270
:10A080000F941F74698F7A8F8B8F9C8FBDA1B23014
:10A0900068F18DA59EA50F94D3316BA57CA585ECA9
:10A0A0009EE00E94C54B8FEB9EE00E94514343E02F
:10A0B000C501B4010F94732180E20E94184381E02E
:10A0C000EDA1E3300CF480E0E12C8E010F5D1F4F19
:10A0D0009E01235E3F4FAE01475E5F4FBE016B5E48
:10A0E0007F4F0E9496448AE00E9418432394B3CD88
:10A0F0000E940C340F94E0068DAD0E94623E0F94D6
:10A10000BD1088AD99AD0FB6F8949EBF0FBE8DBF40
:10A11000E8ADF9AD0FB6F894FEBF0FBEEDBFC55B5D
:10A12000DF4F0FB6F894DEBF0FBECDBFDF91CF91EA
:10A130001F910F91FF90EF90DF90CF90BF90AF9065
:10A140009F908F907F906F905F904F903F902F9057
:10A1500008950E940C34332069F284EB9EE00E9443
:10A16000514381E0FDA11F160CF080E0EE24E39442
:10A170008E010F5D1F4F9E01235E3F4FAE01475E74
:10A180005F4FBE016B5E7F4F0E949644698D7A8D52
:10A190008B8D9C8D0052110926E042E00F944C6596
:10A1A0009F938F9383EA9EE09F938F938DEA9EE027
:10A1B0009F938F931F920E942CCB2DB73EB7295FA0
:10A1C0003F4F0FB6F8943EBF0FBE2DBF93CF2F92D7
:10A1D0003F924F925F926F927F928F929F92AF9237
:10A1E000BF92CF92DF92EF92FF920F931F93CF9384
:10A1F000DF93CDB7DEB7CC58D1090FB6F894DEBFE8
:10A200000FBECDBF84E99DE00E94514387E00F94CB
:10A21000FC2C81118FC084E50E94B139882329F07C
:10A220000E94353981110E943CEC80E090E0A0E86A
:10A23000BFE389839A83AB83BC838D839E83AF8383
:10A24000B8878DEC9CECACE4BEE389879A87AB873A
:10A25000BC8780E090E0A0E2B1E48D879E87AF8765
:10A26000B88B8CE390E09A8B898B8DEC90E09C8B83
:10A270008B8B8DEC9CECACECBEE38D8B9E8BAF8B13
:10A28000B88F80E090E0A0EEBFE3898F9A8FAB8F0C
:10A29000BC8F1BA61CA64AE959E969E97EE38FE455
:10A2A0000E94373A6D8F7E8F8F8F98A360E083E492
:10A2B0000E94913B89A360E08BE40E94913B8AA3BA
:10A2C00089E40E94B13910E0F12CE12C8823C1F01F
:10A2D0000E945B2C90E01816190614F481E090E0BF
:10A2E00011E0180F212F2150330BC90126E0289FC0
:10A2F000F001299FF00D1124E359F74FE280F3801C
:10A3000082E40E94B139882319F00E9435397C011A
:10A31000E114F10459F1C70188978536910520F1C0
:10A320006CE870E086E69DE00E94C54B81E69DE00A
:10A330000E945143C457DF4F0FB6F894DEBF0FBEE3
:10A34000CDBFDF91CF911F910F91FF90EF90DF90E4
:10A35000CF90BF90AF909F908F907F906F905F90C5
:10A360004F903F902F900895FA8AE98A8CE40E94DA
:10A37000B1398823E1F00E9439396B017C01C9862B
:10A38000DA86EB86FC8620E030E0A9010F94D173D9
:10A3900087FD0AC020E030E040E050E4C701B6018C
:10A3A0000F947F6A18161CF489E39DE0C1CF81E504
:10A3B0000E946339882331F180911E0590911F0519
:10A3C000892BE9F00E9439396B017C01CD82DE8254
:10A3D000EF82F8862DEC3CEC4CE45DE30F94D173F6
:10A3E00087FD0AC020E030E040E751E4C701B60134
:10A3F0000F947F6A181634F488E09DE099CF8DEDB4
:10A400009CE096CF83E50E94B1398823E9F00E9451
:10A4100039396B017C01CD8ADE8AEF8AF88E2DEC0A
:10A420003CEC4CEC5DE30F94D17387FD0AC020E057
:10A4300030E040E050E4C701B6010F947F6A18167F
:10A440001CF486EB9CE074CF80E50E94633988237E
:10A4500041F080911E0590911F05892B29F58FEF02
:10A460008BA786E40E94B139882309F43DC00E947D
:10A4700039396B017C01C98EDA8EEB8EFC8E20E0BF
:10A4800030E040E85FE30F94D17387FD0AC020E01D
:10A4900030E040E850E4C701B6010F947F6A181617
:10A4A0001CF585E69CE044CF8BA58F5F8BA70E94AF
:10A4B00039396B017C01CD86DE86EF86F88A20E093
:10A4C00030E0A9010F94D17387FD0BC020E030E08C
:10A4D00048EC51E4C701B6010F947F6A18160CF0DE
:10A4E000C0CF8EE89CE024CFC98CDA8CEB8CFC8C3E
:10A4F0008D889E88AF88B88CA7019601C701B601E8
:10A500000F94E56A9B01AC0160E070E084E490E4A4
:10A510000F946B7229813A814B815C810F94E56ABB
:10A520002B013C01A5019401C501B4010F94E56A1A
:10A53000A70196010F94E56A2CEE31E548EB5DE347
:10A540000F946B729B01AC01C301B2010F94E56AD9
:10A5500069837A838B839C83112309F1412F4150B6
:10A56000550B26E0249FF001259FF00D1124E3599F
:10A57000F74F0081118188E40E94B139882319F0D6
:10A580000E9435398C010115110571F0C801855AF9
:10A5900091098F30914030F087E39CE0C9CE10E004
:10A5A00000E0E9CF1C8B0B8B85E50E946339882383
:10A5B000C9F00F94344E611571058105910511F0B4
:10A5C0000F94056680911E0590911F05892BC9F097
:10A5D0000E94393960931205709313058093140516
:10A5E000909315056AE170E082E50E94823BAD968A
:10A5F0009FAF8EAFAD971816190644F083E09CE02C
:10A6000097CE60E070E088E492E4E4CF89E50E94B0
:10A61000B139882381F10E9439392091C5093091DF
:10A62000C6094091C7095091C8090F9470716B0118
:10A630007C0188E50E94B139882331F10E943939C3
:10A640002091C1093091C2094091C3095091C409B8
:10A650000F9470716BA37CA38DA39EA3CFA2D8A6E9
:10A66000E9A6FAA6CE0183960E94ED24811115C0B9
:10A6700089ED9BE05DCEC090D109D090D209E090E9
:10A68000D309F090D409D5CF6091CD097091CE094E
:10A690008091CF099091D009DDCF84E40E94633985
:10A6A00011E081270E94623E80E090E0A0EAB0E4E1
:10A6B0008DA79EA7AFA7B8AB60E0CE018D960F9493
:10A6C00030088091F608CD57DF4F8883C358D040BB
:10A6D0001092F6080E940EDD86E89BE00E9451432E
:10A6E00089899A894A970CF091C063E683E69BE0DA
:10A6F0000E9447CB0F946D4E8B899C890E94A2F3D8
:10A7000041E061E080E00F940F24882309F491C0B8
:10A710000F9477430F946D4E1092D9091092DA0975
:10A720001092DB091092DC0989ED99E00F944A043C
:10A730001BA5112309F4E2C020E030E040E751E41A
:10A740006091521070915310809154109091551057
:10A750000F946B7221966CAF7DAF8EAF9FAF219738
:10A760001F3F09F00DC581E080935A0563E68BEB2E
:10A770009BE00E9447CB68E873E182E090E00E9492
:10A780006A9680E1EDECF9E0A1EAB8E001900D9263
:10A790008A95E1F7CE0101960F94DF46C12CD12CAA
:10A7A00076018091E10982FD9EC068E873E182E054
:10A7B00090E00E946A9620E030E040E85EE360911D
:10A7C000AD087091AE088091AF089091B0080F94D9
:10A7D00071716093AD087093AE088093AF08909349
:10A7E000B00820E030E040E85EE3C701B6010F9416
:10A7F00071716B017C0120E030E84BE354E40F946D
:10A80000D17387FD60C010925A0513C063E686E7D6
:10A810009BE00E9447CB0F946D4E10935A05898997
:10A820009A890E942A3961E081E00F948A2281117D
:10A830005CCF6FEF8DEC9BE00E9447CB8CA5811124
:10A8400012C081E08CA78D819E81AF81B885B05800
:10A850008DA79EA7AFA7B8ABBE01635D7F4F81EA0E
:10A8600098E00E94BF3580E090E0A0EAB0E48093D9
:10A87000A9089093AA08A093AB08B093AC081DA6B2
:10A880001EA61FA618AABE01635D7F4F81EA98E04D
:10A890000E94BF35CD57DF4F5881C358D0405093E9
:10A8A000F6080E940EDD10925A058AA1811142CD50
:10A8B0001092E4081092E3080E94A6DD90E080E088
:10A8C0000E94A2F337CDCE01CD960F942D1080E1DA
:10A8D000EDECF9E0A1EAB8E001900D928A95E1F77C
:10A8E0000E9420F45ECF0E9447D263E68EEA9BE08E
:10A8F0000E9447CB0F946D4E10925A05EDE0F5E0A3
:10A9000085E0DF011D928A95E9F780E1EDECF9E041
:10A91000A1EAB8E001900D928A95E1F789859A85C0
:10A92000AB85BC858093A9089093AA08A093AB0837
:10A93000B093AC081DA61EA61FA618AABE01635D93
:10A940007F4F81EA98E00E94BF35BE01635E7F4F72
:10A9500081EA98E00E94BF3581E080935A0589A181
:10A96000882309F463C42091CD093091CE09409128
:10A97000CF095091D009E5962CAF3DAF4EAF5FAFF8
:10A98000E5978091D1099091D209A091D309B09116
:10A99000D409E1968CAF9DAFAEAFBFAFE197312C3C
:10A9A000212C9FEFA4969FAFA497AFEFA896AFAFCF
:10A9B000A897BFEFC158DF4FB883CF57D040EFE41F
:10A9C000C058DF4FE883C058D040F3ECCF57DF4F7B
:10A9D000F883C158D04027E4CE57DF4F2883C258B0
:10A9E000D04081E090E0A0E0B0E0022C04C0880FED
:10A9F000991FAA1FBB1F0A94D2F7CC57DF4F888339
:10AA00009983AA83BB83C458D040ADE0B5E0E796F4
:10AA1000BFAFAEAFE79710E000E09101032C000C50
:10AA2000440B550BC857DF4F288339834A835B8318
:10AA3000C858D040C457DF4F2882CC58D040E79642
:10AA4000AEADBFADE7978D91E796BFAFAEAFE797DD
:10AA500090E0B0E0A0E0CC57DF4F288139814A81F7
:10AA60005B81C458D04082239323A423B523892B30
:10AA70008A2B8B2B09F024C1C857DF4F688179815D
:10AA80008A819B81C858D0400F94866A209186069F
:10AA90003091870640918806509189060F94E56AA7
:10AAA00020917E0630917F0640918006509181066C
:10AAB0000F947171EB966CAF7DAF8EAF9FAFEB973C
:10AAC000B801012E000C880B990B0F94866A209117
:10AAD0008A0630918B0640918C0650918D060F941A
:10AAE000E56A209182063091830640918406509158
:10AAF00085060F9471716B017C01EB962CAD3DAD19
:10AB00004EAD5FADEB97E5966CAD7DAD8EAD9FAD77
:10AB1000E5970F9470712B013C01A7019601E19616
:10AB20006CAD7DAD8EAD9FADE1970F9470714B0113
:10AB30005C01A3019201C301B2010F94E56A2B01EC
:10AB40003C01A5019401C501B4010F94E56A9B0184
:10AB5000AC01C301B2010F9471710F941F744B01CA
:10AB60005C01EB962CAD3DAD4EAD5FADEB976BA1AF
:10AB70007CA18DA19EA10F9470712B013C01A701B6
:10AB800096016FA178A589A59AA50F9470716B01A4
:10AB90007C01A3019201C301B2010F94E56A2B016C
:10ABA0003C01A7019601C701B6010F94E56A9B011C
:10ABB000AC01C301B2010F9471710F941F7420E0B6
:10ABC00030E040E751E40F946B72A50194010F94BB
:10ABD00071716B017C018090120590901305A0901B
:10ABE0001405B090150520E030E040E85FE3C501B2
:10ABF000B4010F94D1731816F4F4C501B4010F9485
:10AC0000DD724B015C0160E070E0CB0118141904A7
:10AC10001A041B0434F40F94B665A50194010F9433
:10AC2000E5700F94866A9B01AC01B601C7010F94D1
:10AC300071716B017C01C158DF4F2881CF57D04023
:10AC4000C058DF4F3881C058D040CF57DF4F4881C0
:10AC5000C158D040CE57DF4F5881C258D040B601BE
:10AC6000C7010F947F6A87FF2BC0A4960FAFA497EC
:10AC7000C457DF4F3881CC58D040A8963FAFA89733
:10AC8000EC96CFAEEC97ED96DFAEED97EE96EFAE8D
:10AC9000EE97EF96FFAEEF97C158DF4FC882CF57C0
:10ACA000D040C058DF4FD882C058D040CF57DF4F78
:10ACB000E882C158D040CE57DF4FF882C258D0400A
:10ACC0000F5F1F4F0530110509F0B9CE4FEF241A61
:10ACD000340A55E02516310409F083CEA4968FADD1
:10ACE000A497E82FF0E0E35FFA4F208181E090E045
:10ACF000A0E0B0E0A8960FACA89704C0880F991FF9
:10AD0000AA1FBB1F0A94D2F7822B8083A8969FADFF
:10AD1000A8976A969FAF6A97A496AFADA4976B96D3
:10AD2000AFAF6B97EC968FADEC97ED969FADED972F
:10AD3000EE96AFADEE97EF96BFADEF976F968CAFF7
:10AD40009DAFAEAFBFAF6F97A896BFADA897BF3FFF
:10AD500009F4FAC1A496EFADA497EF3F09F4F4C14A
:10AD60006B2FBB0F770B880B990B0F94866A209182
:10AD700086063091870640918806509189060F9487
:10AD8000E56A20917E0630917F06409180065091C1
:10AD900081060F947171162F072F382E292E862FBA
:10ADA000902FA32DB22D65968CAF9DAFAEAFBFAFE8
:10ADB0006597A496FFADA4976F2FFF0F770B880BB5
:10ADC000990B0F94866A20918A0630918B064091E8
:10ADD0008C0650918D060F94E56A20918206309181
:10ADE000830640918406509185060F9471716B0122
:10ADF0007C016996CCAEDDAEEEAEFFAE6997CE01BA
:10AE00008F5A9F4F0E94ED24882309F4A1C120E0AE
:10AE100030E040EA50E4612F702F832D922D0F9483
:10AE200071714B015C01CB01D50121968CAF9DAFB7
:10AE3000AEAFBFAF21972596CCAEDDAEEEAEFFAE86
:10AE40002597A8962FADA89721112AC2A4963FADA9
:10AE5000A4973111FAC120E030E040EA50E4C70184
:10AE6000B6010F9471716B017C01A4964FADA4974C
:10AE7000442309F40CC2A4968FADA49784300CF03F
:10AE800006C222ED422E23E5522E2BE7622E21E44C
:10AE9000722E21968CAC9DACAEACBFAC21972596A2
:10AEA0008CAD9DADAEADBFAD2597A7968CAF9DAFD8
:10AEB000AEAFBFAFA7979C01AD0169966CAD7DADFC
:10AEC0008EAD9FAD69970F947071AB966CAF7DAFEF
:10AED0008EAF9FAFAB97A501940165966CAD7DAD2C
:10AEE0008EAD9FAD65970F9470712D966CAF7DAF51
:10AEF0008EAF9FAF2D97AB962CAD3DAD4EAD5FADF8
:10AF0000AB9761962CAF3DAF4EAF5FAF6197A50198
:10AF100094016091CD097091CE098091CF099091F3
:10AF2000D0090F9470714B015C01A7962CAD3DAD1B
:10AF30004EAD5FADA7976091D1097091D209809114
:10AF4000D3099091D4090F947071A7966CAF7DAF1F
:10AF50008EAF9FAFA797812F902FA32DB22D8DA7D6
:10AF60009EA7AFA7B8ABC9AADAAAEBAAFCAAC98464
:10AF7000DA84EB84FC84CDAADEAAEFAAF8AE2DEC2D
:10AF80003CEC4CEC5CE3C301B2010F94E56A29810F
:10AF90003A814B815C810F94E56A2091D909309107
:10AFA000DA094091DB095091DC090F94717169AFA6
:10AFB0007AAF8BAF9CAFA5019401C501B4010F948A
:10AFC000E56A4B015C01A7962CAD3DAD4EAD5FAD82
:10AFD000A797CA01B9010F94E56A9B01AC01C501AD
:10AFE000B4010F94717120E030E040E050E40F9420
:10AFF000D1731816ACF420E030E040E05FE3C70105
:10B00000B6010F94717129966CAF7DAF8EAF9FAF73
:10B010002997BE01635C7F4FCE0101960E94C8351F
:10B0200089859A85AB85BC8529968CAF9DAFAEAFDF
:10B03000BFAF2997A3961CAE1DAE1EAE1FAEA39741
:10B04000BE01615A7F4FCE01CD960E94BF35CE0121
:10B0500001960F94DF46E0904A10F0904B1000915B
:10B060004C1010914D10A0904610B0904710C09019
:10B070004810D09049109501A601B701C8010F945E
:10B08000D173181614F47501860180908002909097
:10B090008102A0908202B09083022DEC3CEC4CEC3B
:10B0A0005DE3B701C8010F94E56A60938002709375
:10B0B0008102809382029093830240E0BE01675B2D
:10B0C0007F4FCE018D960F942E4F80E1EDECF9E08D
:10B0D000A1EAB8E001900D928A95E1F78092800292
:10B0E00090928102A0928202B09283020E943A2C36
:10B0F00081119FCB20E04FEFBE01675A7F4FCE01F9
:10B1000001960E948B3720E041E0BE01675A7F4FD5
:10B11000CE0101960E948B372FEF40E0BE01675AA7
:10B120007F4FCE0101960E948B3721E040E0BE01A7
:10B13000675A7F4FCE0101960E948B370E9420F400
:10B140000E943A2C811175CB80916A1080936B100C
:10B15000AD964EAD5FADAD9741505109AD965FAF25
:10B160004EAFAD97452B09F464CB6A968FAD6A97C5
:10B1700087FD5FCB6B968FAD6B9787FFF0CB59CB7D
:10B1800063E68BE99BE00E9447CB0F946D4E80E114
:10B19000EDECF9E0A1EAB8E001900D928A95E1F7B3
:10B1A0002D853E854F8558896091AD087091AE0818
:10B1B0008091AF089091B0080F9471716093AD08C1
:10B1C0007093AE088093AF089093B008CE01CD96EF
:10B1D0000F942D102D853E854F8558896091AD08BF
:10B1E0007091AE088091AF089091B0080F94707183
:10B1F0006093AD087093AE088093AF089093B00849
:10B200008CA581117BCB81E08CA78D819E81AF8144
:10B21000B885B0588DA79EA7AFA7B8ABBE01635D38
:10B220007F4F81EA98E00E94BF3568CB2BA13CA1FB
:10B230004DA15EA1E5962CAF3DAF4EAF5FAFE59758
:10B240008FA198A5A9A5BAA5A4CB812F902FA32D36
:10B25000B22D21968CAF9DAFAEAFBFAF219720E04E
:10B2600030E040EA50E4C701B6010F9470712596B2
:10B270006CAF7DAF8EAF9FAF2597A4965FADA497BF
:10B2800054300CF4E8CD182D092D3A2C2B2C92EDCE
:10B29000492E93E5592E9BEF692E90E4792EF9CD36
:10B2A000A8969FADA89794300CF452C0A496AFAD69
:10B2B000A497A4300CF120E030E040EA50E4612F84
:10B2C000702F832D922D0F94707121966CAF7DAFEE
:10B2D0008EAF9FAF219720E030E040EA50E4C701F5
:10B2E000B6010F9470716B017C01A496EFADA49729
:10B2F000E4300CF4C6CDCBCF812F902FA32DB22DEF
:10B3000021968CAF9DAFAEAFBFAF219720E030E06C
:10B3100040EA50E4C701B6010F94717125966CAFF5
:10B320007DAF8EAF9FAF2597A496BFADA497B11107
:10B33000D2CF20E030E040EA50E4612F702F832D1F
:10B34000922D0F947071162F072F382E292E9FCF14
:10B35000A496FFADA497F1110DC020E030E040E2CB
:10B3600051E4B401C5010F947071162F072F382EC8
:10B37000292E87CDA4962FADA49724309CF020E0F1
:10B3800030E040E251E4B401C5010F9470712196A0
:10B390006CAF7DAF8EAF9FAF2197182D092D3A2C42
:10B3A0002B2C6FCD182D092D3A2C2B2C82ED482EED
:10B3B00083E5582E8BEF682E81E4782E6ACD80EDE0
:10B3C00099E00C9451438AEC99E00C945143CF924C
:10B3D000DF92EF92FF928AE50E94B139882309F447
:10B3E0005AC00E94393920E030E040E050EC0F9420
:10B3F0007F6AC12CD12CE12C90ECF92E87FD0FC077
:10B400000E94393920E030E040E050E40F94D173DD
:10B4100018160CF462C00E9439396B017C0120912E
:10B420003E1030913F104091401050914110C701A3
:10B43000B6010F94E56A0F94DD72CB010F94E84ECC
:10B4400080E50E94633981114EC0A7019601609189
:10B4500025167091261680912716909128160F9424
:10B46000717160932516709326168093271690931A
:10B4700028160E94E3594091251650912616609196
:10B480002716709128168CE098E10E943B468AE0CE
:10B490000E94184305C083E50E94B1398111A1CFF4
:10B4A00080914F0587FD24C080915005837001F580
:10B4B0000E94E35940912516509126166091271657
:10B4C000709128168DEF97E10E943B468AE0FF902D
:10B4D000EF90DF90CF900C941843C12CD12CE12C2D
:10B4E00080E4F82E9CCF0E946F2C8111AECFD8CF74
:10B4F00082E50E9463398111DBCFFF90EF90DF90EE
:10B50000CF900895CF9384E50E94B139C0E088239D
:10B51000D9F00E945B2CC82F1816B4F40E94E3598E
:10B520008DE40E94184380914A0590914B050F9439
:10B5300002586C2FCC0F770B89E291E10E94C54B2A
:10B540008AE00E941843CFEF8C2FCF9108954F923D
:10B550005F926F927F928F929F92AF92BF92CF92A3
:10B56000DF92EF92FF92CF93DF93CDB7DEB72C97A8
:10B570000FB6F894DEBF0FBECDBF4090C10950900A
:10B58000C2096090C3097090C409209141023091B2
:10B5900042024091430250914402C301B2010F9410
:10B5A000717169837A838B839C838090C5099090A5
:10B5B000C609A090C709B090C809209145023091F2
:10B5C00046024091470250914802C501B4010F94D0
:10B5D00071716D837E838F839887C090C909D090E5
:10B5E000CA09E090CB09F090CC0920914902309132
:10B5F0004A0240914B0250914C02C701B6010F9490
:10B60000717169877A878B879C8720914D02309171
:10B610004E0240914F0250915002C301B2010F946B
:10B6200071712B013C0120915102309152024091E5
:10B63000530250915402C501B4010F9471714B0132
:10B640005C01209155023091560240915702509171
:10B650005802C701B6010F9471716B017C010E9401
:10B66000E3598AE790E10E94514383E50E946339E0
:10B67000882321F00E946F2C80933F0280913F022B
:10B68000811151C081E690E10E94514382E790E12F
:10B690000E94514349815A816B817C8189E691E303
:10B6A0000E943B464D815E816F81788584E696E4F9
:10B6B0000E943B4649855A856B857C8581E696E4E8
:10B6C0000E943B4680E790E10E94514388E690E16A
:10B6D0000E945143B301A20189E691E30E943B46D7
:10B6E000B501A40184E696E40E943B46B701A60199
:10B6F00081E696E40E943B468AE02C960FB6F894C9
:10B70000DEBF0FBECDBFDF91CF91FF90EF90DF90F6
:10B71000CF90BF90AF909F908F907F906F905F90F1
:10B720004F900C94184385E690E1AECF2F923F9254
:10B730004F925F926F927F928F929F92AF92BF9241
:10B74000CF92DF92EF92FF920F931F93CF93DF93ED
:10B75000CDB7DEB76A970FB6F894DEBF0FBECDBF88
:10B7600083E50E946339182F3090DC08882319F094
:10B770000E946F2C382E4090CD095090CE096090D9
:10B78000CF097090D0098091D1099091D209A091F0
:10B79000D309B091D4098B8B9C8BAD8BBE8B8091E0
:10B7A000D5099091D609A091D709B091D8098F8B6E
:10B7B000988FA98FBA8F112329F0311003C080E030
:10B7C0000E94623E86E50E946339888B20E030E06B
:10B7D000A9016091860670918706809188069091F4
:10B7E00089060F947F6A882309F4C5C083E40E9408
:10B7F0006339882309F498C00E9439396B017C01B0
:10B80000AAE1B6E0B987A887BF83AE83F5E0FD83E0
:10B810001D861E8628EC2F8702EC1A86212C88ECC8
:10B820008B8792E49C87AE81BF81BA8BA98B15E090
:10B83000E989FA8981909190A190B190FA8BE98B76
:10B840002A85322D4B855C85C501B4010F947F6A32
:10B8500087FF04C08A86292CAB86BC862D853E8551
:10B860004F85502FC501B4010F94D173181624F4DD
:10B870008D869E86AF860B2D1150D1F6FD81F1503D
:10B88000FD838E819F8144969F838E83F111CBCF60
:10B890002D853E854F85502F6A85722D8B859C8521
:10B8A0000F94717120E030E040E05FE30F94E56AAF
:10B8B000A70196010F9471716B017C012DEB37E3A9
:10B8C00046E855EB0F94D17387FD0AC02DEB37E3A3
:10B8D00046E855E3C701B6010F947F6A181624F5B0
:10B8E00080E00E94623E15E0A884B98405E0D5019D
:10B8F0006D917D918D919D915D014D01B4E08B1A0B
:10B900009108A70196010F947071F401608371830F
:10B9100082839383015059F7115088859985449605
:10B92000998788871111E0CFA889AA2381F020E0A8
:10B9300030E0A901609186067091870680918806A3
:10B94000909189060F947F6A81110E94A4458AE52F
:10B950000E946339882359F00E94393969837A83B8
:10B960008B839C8360E0CE0101960E94F43E832D80
:10B970000E94623E0BC0311003C09889992339F3AD
:10B980000E94E35984EE9DE00E945143332051F020
:10B990008091DC08811106C00E94DF5985EC9DE092
:10B9A0000E9451430E94E35987EB9DE00E9451435E
:10B9B0008091DC080E941D460E94E3598AEA9DE0BE
:10B9C0000E945143C090D808D090D908E090DA087E
:10B9D000F090DB0820E030E0A901C701B6010F9428
:10B9E000D17318160CF053C042E0C701B6010F9492
:10B9F00073218DE00E9418438AE00E941843A3013E
:10BA000092016091CD097091CE098091CF099091FA
:10BA1000D0090F947F6A81111FC02B893C894D8901
:10BA20005E896091D1097091D2098091D30990917A
:10BA3000D4090F947F6A81110FC02F89388D498DE9
:10BA40005A8D6091D5097091D6098091D70990914E
:10BA5000D8090F947F6A81110F94BD106A960FB6B2
:10BA6000F894DEBF0FBECDBFDF91CF911F910F9134
:10BA7000FF90EF90DF90CF90BF90AF909F908F900E
:10BA80007F906F905F904F903F902F90089585EA40
:10BA90009DE00E945143B3CFCF93C82F82E0C111E4
:10BAA00084E040E060E00E94489C0E94E3598DEAF7
:10BAB0009AE0CC2311F082EC9AE0CF910C945143A0
:10BAC0000E9486EC0E94D44080E00F9499438091BC
:10BAD0006C088130A1F40E94DF5983E599E00E944F
:10BAE000514360E089E499E00E9447CB6EE571E044
:10BAF00080E090E00E944E4088E080936C080895BA
:10BB0000CF92DF92EF92FF921F93CF93DF9300D0FB
:10BB10001F92CDB7DEB78EEEC82E82E0D82EE12C74
:10BB2000F12CC982DA82EB82FC82BE016F5F7F4F0B
:10BB30008AE50E94304281110EC010E0812F0F90E3
:10BB40000F900F900F90DF91CF911F91FF90EF908A
:10BB5000DF90CF9008950E94A142C982DA82EB82E1
:10BB6000FC82BE016F5F7F4F8AE50E943042182F32
:10BB7000882319F30E94DF598DE29AE00E94514315
:10BB80000E94605DDBCFCF92DF92EF92FF921F9316
:10BB9000CF93DF9300D01F92CDB7DEB78EEEC82EC5
:10BBA00082E0D82EE12CF12CC982DA82EB82FC8271
:10BBB000BE016F5F7F4F8AE00E94304281110EC04C
:10BBC00010E0812F0F900F900F900F90DF91CF9189
:10BBD0001F91FF90EF90DF90CF9008950E94A142B7
:10BBE0000E9450420E946B420E945042C982DA82F7
:10BBF000EB82FC82BE016F5F7F4F8AE00E94304281
:10BC0000182F8823E9F20E94DF5980EF99E00E9403
:10BC100051430E94605DD5CFFF920F931F93CF9346
:10BC2000DF93EC018B01F42E0E9486EC0E94DF5919
:10BC300089E299E00E9451430115110511F408EEC3
:10BC400014E4209711F4C0E2D9E00E9438D21F9387
:10BC50000F93DF93CF9380E199E09F938F9381E0DF
:10BC60008F930E942CCB0E945F9BC0915B16C69560
:10BC7000C69586E596E10E940B2FDC2FDD0F1D2F68
:10BC80001C0FEDB7FEB737960FB6F894FEBF0FBE88
:10BC9000EDBF83E00E94892E41E253E16C2F80E0EA
:10BCA0000E94B63110929116D093921681E099E0DD
:10BCB0000E949B2F109291161093921684EF98E099
:10BCC0000E949B2F8AE596E10F9427568111E1CFC0
:10BCD00061E087E199E00E94144589EE93E030E647
:10BCE000019729F0232F2A950000E9F7F9CFF8945E
:10BCF00089EE93E038EE019729F0232F2A95000072
:10BD0000E9F7F9CF0E9486ECFF2041F00E948440C1
:10BD10000E94D326909905C0A895FCCF0E94D126F9
:10BD2000F7CF909B02C0A895FCCFF0E0E0E0DF9158
:10BD3000CF911F910F91FF9019945F926F927F9214
:10BD40008F929F92AF92BF92CF92DF92EF92FF922B
:10BD50000F931F93CF93DF931F92CDB7DEB77C0174
:10BD600039018B015B01A40EB51ED12CC12CA0168C
:10BD7000B10609F450C0F70180809180F80151901C
:10BD80008F015982C4010F949D705816B9F1652D29
:10BD9000C4010F94A570FFEFCF1ADF0AC6018F7799
:10BDA0009927892B21F162E070E080E090E00F9408
:10BDB000014EC4010F949D7099818917F9F00E947A
:10BDC000E35983E596E00E94514381E00F90DF91B3
:10BDD000CF911F910F91FF90EF90DF90CF90BF9088
:10BDE000AF909F908F907F906F905F90089562E0EA
:10BDF00070E080E090E00E944E40DBCFBE016F5FBC
:10BE00007F4FC3010F941C30F7018081918101960F
:10BE100091838083ACCF80E0D9CF80916A109091DC
:10BE20006B102FEF3FEF981751F0E92FF0E0E65934
:10BE3000FF4E228130E09F5F9F7790936B10C90186
:10BE400008951F920F920FB60F9211240F900FBEFC
:10BE50000F901F9018951F920F920FB60F921124FA
:10BE60000BB60F920F931F932F933F934F935F93B4
:10BE70006F937F938F939F93AF93BF93CF93DF93F2
:10BE8000EF93FF93C091C60000916B10D0916A10A0
:10BE900011E01D0F1F779091A904913108F09FC008
:10BEA000E92FF0E08827E85AF04A8F4F0D94687127
:10BEB000695F985FA75FB65FBD5FEF5FC15FEF5FD0
:10BEC000C55FC95FEF5FCD5FD15FD55FDC5FEF5FBF
:10BED000E75FC03229F028F5CA3011F0CD3031F5D6
:10BEE000011731F0ED2FF0E0E659FF4EC283D12F5C
:10BEF000D0936A10FF91EF91DF91CF91BF91AF91F5
:10BF00009F918F917F916F915F914F913F912F9171
:10BF10001F910F910F900BBE0F900FBE0F901F90AF
:10BF20001895CD3481F081E0CE3471F080E10CC001
:10BF3000CA3338F4C033A0F6C03291F2CD32B1F733
:10BF4000CFCFCD3499F782E08093A904C9CFC13314
:10BF500059F018F4C03221F2E9CF88E0C433A1F3DC
:10BF60008BE0C83389F3E2CF83E0EECF84E0C033C7
:10BF700059F386E0C13341F3D9CF85E0C833B1F638
:10BF8000E3CF87E0C23391F6DFCF89E0C13371F6AA
:10BF9000DBCF8AE0C03351F6D7CF8CE0C73331F620
:10BFA000D3CF8DE0C63311F6CFCFC03209F498CF8E
:10BFB0008EE0C33549F2BACF80ED8C0F8A3008F09D
:10BFC0008FCF9FE09093A9048093A80489CFCA30B3
:10BFD00019F0CD3009F084CF1092A90481CFCA3076
:10BFE00019F0CD3009F07CCF809194168823A1F30D
:10BFF000973041F138F4953079F71092740210922D
:10C00000BC08EACF9A3011F19F3031F79091A80423
:10C010008091B9081092B908823089F38430E9F030
:10C020008130D1F69923B1F09130B1F682E080935E
:10C03000BB088091BA08882379F210925D020E94B1
:10C04000BE26CACF81E080939C06C6CF81E0809354
:10C050009B06C2CF8093BB08BFCF84EA91E2909346
:10C060002A0880932908B8CF8EBD0DB407FEFDCFF6
:10C0700008958FEF8EBD0DB407FEFDCF8EB50895E8
:10C08000909164009B7F90936400982F906A96959E
:10C090009CBD80FD03C091E0863009F490E09DBD19
:10C0A0000895CF93DF93EB010E945143CE01DF91BE
:10C0B000CF910C9403E6AF92BF92CF92DF92EF92B2
:10C0C000FF920F931F93CF93DF93CDB7DEB7E69721
:10C0D0000FB6F894DEBF0FBECDBF00915105109191
:10C0E0005205F80101900020E9F731976F01C01A5D
:10C0F000D10AF801CF01801B910B8C159D053CF4F2
:10C1000081918F32B9F7DF0111971C92F3CF8BE148
:10C11000E1ECF6E1DE015C9601900D928A95E1F783
:10C12000F12CE12CEC14FD040CF05DC0F801EE0DD7
:10C13000FF1D8081811103C08FEFE81AF80A5801B2
:10C14000AE0CBF1CF5018081882309F44CC0FFEFC1
:10C15000EF1AFF0AF801EE0DFF1D7F01E01AF10A48
:10C1600081918111FACFCE014C960E9469EA8BE150
:10C17000FE017C96DE01119601900D928A95E1F701
:10C18000B501CE0101960E9475E2CE0101960E9492
:10C19000CE3B8FE20E9418438091DE1281113BC09A
:10C1A00087E893E00E9403E68091A01684FF1BC0FD
:10C1B00019821C8221E0A501BE01645E7F4FCE0181
:10C1C00001960F94941F811129C08AE00E941843A0
:10C1D0000E94E359B5018AE798E10E945160CE01BF
:10C1E00001960E94CE3B8AE00E941843CE014C96F5
:10C1F0000E94CE3BE6960FB6F894DEBF0FBECDBFD1
:10C20000DF91CF911F910F91FF90EF90DF90CF9032
:10C21000BF90AF9008958EED92E1C4CFCE014C96C1
:10C220000E946BE98BE1FE013196DE015C96019084
:10C230000D928A95E1F7CE0101960E94CE3B72CF16
:10C240002F923F924F925F926F927F928F929F9226
:10C25000AF92BF92CF92DF92EF92FF920F931F9314
:10C26000CF93DF9300D000D000D01F921F92CDB7A4
:10C27000DEB7B82E80915711843008F0D1C10F94E9
:10C28000344E6B017C0180915711811108C080915F
:10C290006A1090916B10891B8F7709F4D9C681E6DB
:10C2A000A82E13C08A3019F08D3009F0F6C0109214
:10C2B00052118091F0109091F110FC01E451FF4E69
:10C2C0001682892BF1F40F943E0980915711843026
:10C2D00008F0ECC080916A1090916B10891B8F77E9
:10C2E00009F4E4C00E940D5F97FFDCCF0E94DF5984
:10C2F00089E997E00E94514380916A1080936B1006
:10C30000E4CF1092F1101092F01002EF10E1F8015A
:10C310008191803209F446C08E3409F0A9C064E9E5
:10C3200077E0C8010F94FC694C01892B41F06EE461
:10C3300070E0C80104960F94C674009709F4C80110
:10C340004AE050E070E060E001960F946C672B01CA
:10C350003C018091EC109091ED10A091EE10B09105
:10C36000EF100196A11DB11D481659066A067B06FD
:10C3700029F060E081E697E0892851F16AE270E0F7
:10C38000C8010F94F5749C01009729F1982F901B18
:10C39000912C992349F09150F801E90FF11D80810A
:10C3A0009826F7CF8F01B3CF4AE050E070E060E00D
:10C3B000C90101960F946C67292D30E050E040E0F0
:10C3C000621773078407950751F060E082E497E0F5
:10C3D0000F941B357ACF60E088E197E0F9CF409267
:10C3E000EC105092ED106092EE107092EF10809170
:10C3F0006C088130E1F067E470E0C8010F94C67406
:10C400000097A9F04AE050E070E060E001960F94D8
:10C410006C67643071058105910548F487E796E003
:10C420000E94514360E08DE696E00E9447CBC092A7
:10C43000C108D092C208E092C308F092C40880916B
:10C44000F2108B3309F441CF80915711843008F0FA
:10C450003CCF809159118A9DC001112462EF70E197
:10C46000865A9E4E0F94D17480E00F94D5342DCF10
:10C470008091A01680FFBBCF6BE674E4C8010F94D7
:10C48000FC69009731F0FC01838180538A3008F009
:10C49000AECF60E08EEE96E09BCF20EF30E142EF32
:10C4A00050E162E571E10E947C240FCF8091A016DB
:10C4B00082FFB6C01A82198271E6F72EE0E1EE2EF5
:10C4C000F9E6DF2E80915711843008F0A9C00E9450
:10C4D000B4248111A5C041E050E0BE016B5F7F4FE5
:10C4E00085E098E10E94A3E60D8110E0019711F02C
:10C4F0000FEF1FEF80910D1890910E18A0910F185B
:10C50000B091101880939C1690939D16A0939E1640
:10C51000B0939F160E94B4240F3F100749F4811175
:10C5200007C00E94DF5987EB97E00E945143CACFB2
:10C5300040915911242F30E00A3061F00D3051F054
:10C54000882309F45FC089819A81009719F00196C8
:10C550009A8389831092AC0489819A81F29EF001BA
:10C56000F39EF00D1124E95AFE4EE80FF91F1382D5
:10C57000892B69F50F943E090E94B424882309F49D
:10C58000A1CF0E9420F485E098E10E946BE98091A0
:10C590009716882391F18150809397168D9DC00145
:10C5A000112462E08756984F0F94095BE09197162B
:10C5B00024E0E29FF0011124EB56F84F6081718175
:10C5C000828193810E94642A0E94DEE17BCF1A82DD
:10C5D000198281E00F94D53480919C1690919D161C
:10C5E000A0919E16B0919F16809353119093541171
:10C5F000A0935511B0935611BFCF0E9474E9E092F9
:10C600006C0860CF4F9DA0011124465A5E4E9E01DA
:10C610002F5F3F4F6CEA74E0802F0E947C2452CF42
:10C620000F94344E6B017C01B11004C08091A906B7
:10C63000882351F0C092B308D092B408E092B508B4
:10C64000F092B608BB24B39480912A0590912B05F3
:10C65000A0912C05B0912D050097A105B10551F1D0
:10C660004091B3085091B4086091B5087091B60834
:10C67000840F951FA61FB71FA7019601281B390B12
:10C680004A0B5B0BDA01C901B7FD14C00E94DF59E8
:10C690006091BF087091C00882E198E00E945160EB
:10C6A0008AE00E94184340E070E060E090E080E0A3
:10C6B0000E940C5E80911B0290911C02A0911D02B1
:10C6C000B0911E02892B8A2B8B2B79F090912E161C
:10C6D00080912F16981709F4ACC1C092B308D0927C
:10C6E000B408E092B508F092B6088091BD0490912C
:10C6F000BE049099E0C101969093BE048093BD045E
:10C700008091BD049091BE048E3E92406CF00E94D8
:10C71000DF598FEE97E00E94514340E070E060E007
:10C7200090E080E00E940C5E0F94344E4B015C015F
:10C730008091BC08811108C020912E1690912F166F
:10C7400081E0291301C080E020919015309191156E
:10C7500091E089272A3A31050CF480E091E040917C
:10C76000B1045091B2046091B3047091B404452BAC
:10C77000462B472B09F490E0981789F0882309F499
:10C78000A0C1D501C40180569444A24FBF4F8093ED
:10C79000B1049093B204A093B304B093B404409056
:10C7A000D9095090DA096090DB097090DC0920917A
:10C7B000AD043091AE044091AF045091B004C30178
:10C7C000B2010F947F6A882319F18091B10490918E
:10C7D000B204A091B304B091B4044092AD0450925D
:10C7E000AE046092AF047092B004892B8A2B8B2B1D
:10C7F00009F449C0D501C40180569444A24FBF4FEB
:10C800008093B1049093B204A093B304B093B404A2
:10C810008091B1049091B204A091B304B091B4049A
:10C820000097A105B10579F1881A990AAA0ABB0AED
:10C83000B7FC29C01092B1041092B2041092B30454
:10C840001092B4048AED97E00E94514360E086ECB8
:10C8500097E00E9447CB80919215909193151816FE
:10C86000190624F490E080E00E94A2F38091E3088E
:10C870009091E4081816190634F41092E408109206
:10C88000E3080E94A6DD8091B9049091BA04A091BA
:10C89000BB04B091BC0446015701881A990AAA0A40
:10C8A000BB0AD501C401B7FD9CC120912E16909101
:10C8B0002F164091640280916302291306C1909162
:10C8C0000B0A899FC0011124880F892F881F990B9B
:10C8D00091958D8380910C0A489FC0011124880F87
:10C8E000892F881F990B91958E830F94344E6983FD
:10C8F0007A838B839C8340E0BE016F5F7F4FCE01C4
:10C9000005960E9479F46D8170E089E00F942B4DBB
:10C9100041E0BE016F5F7F4FCE0105960E9479F422
:10C920006E8170E087E00F942B4D8091A8068823DC
:10C9300009F44AC100913B0210913C02C8010297E0
:10C940002091921530919315281739070CF43CC1AA
:10C9500080902F168F82188619861A861B868091E2
:10C960002E169F80891509F4CAC0892D90E030E603
:10C97000A32EA89EF001A99EF00D1124E05EF54FB4
:10C98000458956896789708D452B462B472B81F445
:10C99000418D528D638D748D452B462B472B41F471
:10C9A000458D568D678D70A1452B462B472BE1F1A8
:10C9B00020E6B22EB89E9001B99E300D1124A90137
:10C9C000405E554F1A01FA01618172818381948121
:10C9D0000F941F744B015C01F10161A172A183A14D
:10C9E00094A10F94846A2B013C01F10165A176A109
:10C9F00087A190A50F94846A9B01AC01C301B20189
:10CA00000F946B72A50194010F94E56A4B015C01D0
:10CA1000288539854A855B850F94D173181624F4CF
:10CA200088869986AA86BB868F818F5F8F708F8359
:10CA300096CFBB2019F01092BF0457CE0F94344EFE
:10CA40000091B3081091B4082091B5083091B60850
:10CA500080901B0290901C02A0901D02B0901E02BC
:10CA6000080D191D2A1D3B1D601B710B820B930BBA
:10CA700097FDE1CF8091BF04811137CE81E0809393
:10CA8000BF045F9A8091B1088E7F8093B1088A9A23
:10CA90008091B1088D7F8093B108809108018095C5
:10CAA0008170809306018091B1088B7F8093B108DB
:10CAB0000E94D1261ACE181619060CF021CE019725
:10CAC0001BCE80E090E0DC0162CE20912F1650E674
:10CAD000259F90011124205E354FF901EA5AFF4F3E
:10CAE0009081899FC0011124880F892F881F990B7D
:10CAF00091958D83295A3F4FF9018081EDCE209188
:10CB000035023091360240913702509138026885E3
:10CB100079858A859B850F94E56A4B015C01B80194
:10CB2000012E000C880B990B0F94866A9B01AC01B7
:10CB3000C501B4010F94717169837A838B839C83DF
:10CB40004091390250913A02B801CE0101960E94FB
:10CB500051ED89809A80AB80BC804090B5045090A4
:10CB6000B6046090B7047090B804A3019201C501A7
:10CB7000B4010F947F6A87FF16C028E431EE4AE7BC
:10CB80005FE3C301B2010F94E56A20E037ED43EAA9
:10CB90005CE30F947171A50194010F94E56A6983B8
:10CBA0007A838B839C8369817A818B819C8160935A
:10CBB000B5047093B6048093B7049093B8040F94AF
:10CBC000DD72CB010E94A2F3F4E6CF0ED11CE11C72
:10CBD000F11CC092B904D092BA04E092BB04F09266
:10CBE000BC040F943E0980916C08882309F4F0C1BD
:10CBF00080915D02882309F471C08091BA08811187
:10CC00006DC00E947240811105C08091A9068823E1
:10CC100009F464C0F894649B10C08091590290910B
:10CC20005A02A0915B02B0915C02809393069093AC
:10CC30009406A0939506B093960660919306709122
:10CC400094068091950690919606789420E030E0C5
:10CC5000A9010F947F6A87FF41C001E00093BA08E1
:10CC60008091A906811138C00E9445450093B908FA
:10CC700040E36EE778E086EB95E40E944A4561E088
:10CC80008AEA95E40E942C4510912E0560E0102759
:10CC900088E39BE069F48CE698E00E94144580E309
:10CCA0000E9418438AE00E94184360E08FE498E0F5
:10CCB0000E9414458AE598E00E94514380E30E9457
:10CCC00018438AE00E941843112331F085E598E06B
:10CCD00090932A08809329080E9420F490910901DA
:10CCE000892F8095817010910802181709F45AC095
:10CCF0002091A01620622093A0168093080290FD38
:10CD000010C064EF71E080E090E00E944E400E940D
:10CD100096E98091A01683FDBEC1112309F442C09B
:10CD200002C00E9485E9123008F46BC100E00E9445
:10CD3000212E83E0809384020F94344E6C597F4FF0
:10CD40008F4F9F4F609356057093570580935805FA
:10CD500090935905002331F1123021F58091A016EE
:10CD600083FF20C00F94EC58882379F081E00F9462
:10CD7000085842EB50E06FE079E086EA96E10E94C5
:10CD8000A3E686EA96E10E946BE90E94BC3B811112
:10CD900044C10E94A63B0F94F75981E080939616F8
:10CDA0000F94395A0F94344E6B017C0110911F027D
:10CDB0001123F1F08091BD088823D1F04091C00487
:10CDC0005091C1046091C2047091C304460157019F
:10CDD000841A950AA60AB70AB501A40177FD1AC0FC
:10CDE000833009F430C10CF01FC181300CF024C134
:10CDF000212F30E0A8EEB3E00F941771C60ED71EB6
:10CE0000E81EF91EC092C004D092C104E092C20490
:10CE1000F092C3048091D608813009F073C00F945A
:10CE2000344E6B017C018091C8049091C904A0919B
:10CE3000CA04B091CB04A7019601281B390B4A0BF9
:10CE40005B0BDA01C901B7FD3AC0D701C601805FAB
:10CE5000984DAF4FBF4F8093C8049093C904A093DF
:10CE6000CA04B093CB0480900D0690900E06A0905B
:10CE70000F06B09010060F94FE16AB01BC01409354
:10CE80000D0650930E0660930F0670931006809166
:10CE9000190890911A08A0911B08B0911C088819D4
:10CEA0009909AA09BB09840F951FA61FB71F809374
:10CEB000190890931A08A0931B08B0931C0880913E
:10CEC000C4049091C504A091C604B091C704460162
:10CED0005701881A990AAA0ABB0AD501C401B7FDED
:10CEE00011C020E8C20E2EEED21E26E3E21EF11C77
:10CEF000C092C404D092C504E092C604F092C70464
:10CF00000E941FF30F94FC1B0E9484CF809129057F
:10CF1000882379F10F94344E6B017C0180912505B3
:10CF200090912605A0912705B0912805460157014B
:10CF3000881A990AAA0ABB0AD501C401B7FD19C00B
:10CF40002091290530E0A8EEB3E00F941771C60ECA
:10CF5000D71EE81EF91EC0922505D0922605E09244
:10CF60002705F092280580E00F9417228AE00E949E
:10CF7000184380912405882359F10F94344E6B0196
:10CF80007C018091200590912105A0912205B0910E
:10CF90002305A7019601281B390B4A0B5B0BDA010D
:10CFA000C901B7FD15C02091240530E0A8EEB3E01B
:10CFB0000F941771C60ED71EE81EF91EC0922005E9
:10CFC000D0922105E0922205F09223050F940F598B
:10CFD0002B960FB6F894DEBF0FBECDBFDF91CF9179
:10CFE0001F910F91FF90EF90DF90CF90BF90AF9087
:10CFF0009F908F907F906F905F904F903F902F9079
:10D00000089560E08FE898E00E9447CB8091630527
:10D0100081118CCE0E945F9B89CE8CEA98E0909320
:10D020002A0880932908BECE843009F0E1CE0E9400
:10D03000E35983EB98E004C00E94E35982EE98E044
:10D040000E945143D5CE0E94E3598BEC98E0F8CF73
:10D050008091C1089091C208A091C308B091C40802
:10D06000A7019601281B390B4A0B5B0BDA01C9019A
:10D07000885E9340A109B109B7FD11C981EB97E022
:10D080000E945143C092C108D092C208E092C308E6
:10D09000F092C40804C9123028F460E08DE998E0E9
:10D0A0000E9447CB01E043CE2F923F924F925F9276
:10D0B0006F927F928F929F92AF92BF92CF92DF92A8
:10D0C000EF92FF920F931F93CF93DF93CDB7DEB70D
:10D0D000EE970FB6F894DEBF0FBECDBF8091DC088F
:10D0E000888B87E50E946339882309F41FC120E0FB
:10D0F00030E0A901609186067091870680918806CC
:10D10000909189060F947F6A811108C00E94DF59AF
:10D1100081E99EE00E94514310E01BC18AE50E9414
:10D12000B139882339F10E9439392091C9093091E8
:10D13000CA094091CB095091CC090F9470716B01D1
:10D140007C0120E030E040E251ECC701B6010F94D1
:10D15000D17387FD0AC020E030E040E251E4C7010E
:10D16000B6010F947F6A181674F40E94DF5984E8A0
:10D170009EE0D0CFC090D509D090D609E090D709D5
:10D18000F090D809DECF40E050E060EC7FE788E522
:10D190000E94373A2091C1093091C2094091C309D8
:10D1A0005091C4090F9470712B013C0140E050E094
:10D1B00060EC7FE789E50E94373A2091C5093091FC
:10D1C000C6094091C7095091C8090F9470714B016D
:10D1D0005C016FEF89E40E942B3A182F6FEF8AE40D
:10D1E0000E942B3A082FA3019201C301B2010F94B0
:10D1F000637481116EC0A5019401C501B4010F943F
:10D200006374811166C08BA19CA1ADA1BEA18BAB43
:10D210009CABADABBEAB20917E0630917F064091BA
:10D22000800650918106C301B2010F9470712B01E9
:10D230003C0120E030E040E05FE36BA97CA98DA9D0
:10D240009EA90F94E56A9B01AC01C301B2010F9442
:10D2500071712BA93CA94DA95EA90F946B720F9413
:10D26000DD72162F4FA058A469A47AA420918206DB
:10D27000309183064091840650918506C501B40122
:10D280000F9470714B015C0120E030E040E05FE3FF
:10D29000C301B2010F94E56A9B01AC01C501B40161
:10D2A0000F947171A30192010F946B720F94DD7250
:10D2B000062F812F012E000C990B97FD2FC005978B
:10D2C0007CF5802F002E000C990B97FD2BC0059745
:10D2D0005CF5153008F020CF053008F01DCF80E058
:10D2E0000E94623E95E01902F0011124E00FF11D49
:10D2F00007FDFA95EE0FFF1FEE0FFF1FE65EF94FD9
:10D30000C082D182E282F38288890E94623E88894B
:10D31000882309F401CF0F94BD10FECE10E0D1CFC9
:10D3200014E0CFCF00E0D5CF04E0D3CF8AE40E9451
:10D330006339182F811127C070E060E086E50E94F4
:10D34000823B9A838983059708F18FE59EE00E94CE
:10D350005143812FEE960FB6F894DEBF0FBECDBFBE
:10D36000DF91CF911F910F91FF90EF90DF90CF90C1
:10D37000BF90AF909F908F907F906F905F904F90F5
:10D380003F902F9008950E94B03EC6CE60E084E4A6
:10D390000E94913B8F8740E050E0BA018AE50E94ED
:10D3A000373A6BA77CA78DA79EA740E050E86BE3B8
:10D3B00076E483E50E94373A20E030E040E752E42B
:10D3C0000F946B72609378027093790280937A0263
:10D3D00090937B02E0902916F0902A16D7018D9049
:10D3E0009D90AD90BC9020E030E0A901C501B40152
:10D3F0000F9471716BAF7CAF8DAF9EAF20E030E0CA
:10D4000040E450E40F947F6A87FF06C01BAE1CAE59
:10D41000B0E4BDAFE0E4EEAF20E030E84DE953E426
:10D42000C501B4010F947171662E7BAB8FAB98AFC1
:10D4300020E030E844E953E40F94D17318163CF42B
:10D44000612CF0E8FBAB24E92FAB83E488AFD70174
:10D4500014968D909D90AD90BC90179720E030E091
:10D46000A901C501B4010F947171D62EE72EF82ED3
:10D47000092F20E030E040E951E40F947F6A87FFF4
:10D4800005C0D12CE12CF0E9FF2E01E420E030E0D2
:10D490004BE953E4C501B4010F947171B62EC72E48
:10D4A00089AF9AAF20E030E04DE853E40F94D17398
:10D4B000181634F4B12CC12CBDE8B9AFE3E4EAAFDF
:10D4C00088E40E946339882309F415C20E9439391F
:10D4D0000F94DD721B0177FF02C06F5F7F4F759560
:10D4E00067957195619571096A567F4F072E000CFB
:10D4F000880B990B0F94866A762E872E982EA92E6C
:10D500002D2D3E2D4F2D502F0F94D17318161CF436
:10D51000D72C74010A2D2BAD3CAD4DAD5EAD672D02
:10D52000782D892D9A2D0F94D173181624F07BAC89
:10D530008CAC9DACAEAC872D982DA92DBA2D8B8BC4
:10D540009C8BAD8BBE8B8D2D9E2DAF2DB02F8F8BD9
:10D55000988FA98FBA8FB101330C880B990B0F9458
:10D56000866A1B012C01AC019B016D2D7E2D8F2D38
:10D57000902F0F947171D62EE72EF82E092F2B2D98
:10D580003C2D49AD5AAD0F947F6A87FF04C0BD2C76
:10D59000CE2CF9AE0AAFA2019101672D782D892D0D
:10D5A0009A2D0F947171D62EE72EF82E092F262D65
:10D5B0003BA94FA958AD0F947F6A87FF04C06D2C1B
:10D5C000EBAAFFAA08AF862D9BA9AFA9B8AD8B8F98
:10D5D0009C8FAD8FBE8F8B2D9C2DA9ADBAAD8F8F3B
:10D5E00098A3A9A3BAA3BE01695E7F4FCE0143965B
:10D5F0000E941534882309F4AFC1BE01615E7F4FDC
:10D60000CE014B960E941534E82E882309F4A4C15C
:10D610002F89388D498D5A8D6F8D78A189A19AA156
:10D620000F94707120E030E040E85EE30F94E56A0B
:10D630004B015C012B893C894D895E896B8D7C8D0A
:10D640008D8D9E8D0F94707120E030E040E85EE398
:10D650000F94E56A6BA37CA38DA39EA38FA298A6CB
:10D66000A9A6BAA689819A811816190674F48DE2C2
:10D670009EE00E9451438F85882321F083E29EE043
:10D680000E9451438AE00E9418430E9420F40F94A4
:10D69000F90680E00E94623E80E090E0A0E2B1E402
:10D6A0008FA798ABA9ABBAAB60E0CE018F960F9471
:10D6B0003008209186063091870640918806509167
:10D6C00089066BA17CA18DA19EA10F947F6A811117
:10D6D00030C020918A0630918B0640918C06509183
:10D6E0008D066FA178A589A59AA50F947F6A8111EF
:10D6F00020C020917E0630917F0640918006509197
:10D7000081066B897C898D899E890F947F6A81113E
:10D7100010C020918206309183064091840650917A
:10D7200085066F89788D898D9A8D0F947F6A8823FD
:10D73000A9F00E94B03E88E0FE01B396A6E8B6E0EC
:10D7400001900D928A95E1F788E0FE017396AEE7AD
:10D75000B6E001900D928A95E1F7188A60E085E4C1
:10D760000E94913B88248394811102C062E0862E3E
:10D770001B861C861D861E861A8A9E2C43EFC42E8D
:10D780004DE0D42E51E0A52E5EE0B52E1A8915305D
:10D790000CF0ECC06B857C858D859E859B01AC0172
:10D7A0000F9463748111E2C03324339435E0232E47
:10D7B000911005C033243A9422242A9484E091E005
:10D7C0009926F12EFF0CFF0CF10EF394898B198929
:10D7D0006A89121509F4C6C0062E000C770B880B57
:10D7E000990B0F94866A2FA138A549A55AA50F94C5
:10D7F000E56A2F89388D498D5A8D0F9471712B01EF
:10D800003C01612F110F770B880B990B0F94866ADF
:10D810002BA13CA14DA15EA10F94E56A2B893C8907
:10D820004D895E890F9471716B837C838D839E8398
:10D830004F82588669867A8689819A81892B79F008
:10D840006F2D8FE09EE00E94334669E170E08DE02D
:10D850009EE00E94C54B8AE09EE00E9451431F92C9
:10D86000F9E1FF931F92FF92DF92CF92BF92AF92A6
:10D870001F920E942CCB2981482DBE01695F7F4FEA
:10D88000CE0103960F94F2442B013C014B865C863B
:10D890006D867E860FB6F894DEBF0FBECDBFAC019D
:10D8A0009B010F94637481115AC009898A8925E00C
:10D8B000020380011124080F111D87FD1A95000F26
:10D8C000111F000F111F065E194FA30192016BA5D6
:10D8D0007CA58DA59EA50F947171D8016D937D9344
:10D8E0008D939C931397188A81E00E942061F39492
:10D8F0008989830D6BCF4D2D5E2D6F2D702F86E4A2
:10D900000E94373A1B012C014BAD5CAD6DAD7EAD75
:10D910008CE40E94373A6B8B7C8B8D8B9E8B2F8A8D
:10D92000388E498E5A8E4B2D5C2D69AD7AAD82E4CE
:10D930000E94373A6B017C01462D5BA96FA978AD37
:10D9400082E50E94373A6B8F7C8F8D8F9E8FCF8EB2
:10D95000D8A2E9A2FAA247CE83E49EE0F8CC888957
:10D960000E94623E8A898F5F8A8B10CF0F94774323
:10D970000E940C34882359F088890E94623E80E01E
:10D9800090E0A0ECBFE78B879C87AD87BE876B8557
:10D990007C858D859E859B01AC010F9463748111FC
:10D9A00059C08F85811126C082E0F82E02E094E0F4
:10D9B000C92E12E0DC2CD11A21E041E0612F802F2A
:10D9C0000E942E2521E04FEF612F8F2D0E942E25E2
:10D9D0002FEF41E06D2D802F0E942E252FEF4FEF6E
:10D9E0006D2D8F2D0E942E25115020F70150F3949C
:10D9F0000F3FF9F60E94A4450E94D43F8F85811104
:10DA000024C085ED99E00E9447354B015C018DEC07
:10DA100099E00E94753C9B01AC01C501B4010F94D3
:10DA2000E56A9B01AC016091D5097091D60980919E
:10DA3000D7099091D8090F9470716093D5097093AC
:10DA4000D6098093D7099093D8098F858111E888EA
:10DA5000E092DC080F94E0068091DC0881110F94BD
:10DA60003C090E94102C0F94BD106B857C858D8520
:10DA70009E8511E09B01AC010F946374811169CC08
:10DA80004BCBCF93DF93C82FD62F8091211083FDEE
:10DA900014C080911D0A811110C08091890290915B
:10DAA0008A02AC0141505109209192153091931591
:10DAB0002417350714F40E94A2F340E06D2F8BE089
:10DAC0000E94489CCC2339F040E061E080E0DF9187
:10DAD000CF910D940F2480911D0A91E089278093A6
:10DAE000740280917402882389F08091901590913E
:10DAF00091152091921530919315821B930B97FFEE
:10DB000003C0919581959109029744F41092740293
:10DB10008091211083FF06C0C1E01AC080E00E94FE
:10DB20002061DFCFC0911D0AC11112C0809189020E
:10DB300090918A02019720919215309193152817A0
:10DB4000390754F70E94E3598CE99AE00E94514347
:10DB50008C2FDF91CF910895AF92BF92CF92DF9239
:10DB6000EF92FF920F931F93CF93DF93CDB7DEB762
:10DB700064970FB6F894DEBF0FBECDBF0E94825AE5
:10DB8000D82E87FDB5C08AE50E94B139882309F4F3
:10DB9000C0C040E050E0BA018AE50E94373A7B01FC
:10DBA0008C014D2D63E085E00E94489C2091D509B1
:10DBB0003091D6094091D7095091D80960E070E0C2
:10DBC00088EC93E40F9470715B016C019701A801DC
:10DBD0000F94D173181614F07501860120E030E01F
:10DBE000A901B701C8010F94D173181624F4E12CD0
:10DBF000F12C00E010E0B701C8010F94DD72072E90
:10DC0000000C880B990B0F94866A6D837E838F833B
:10DC1000988720E030E0A9010F947F6A882321F0E3
:10DC2000CE0105960E94B22A80E090E0A0EAB1E41D
:10DC300089879A87AB87BC871D861E861F86188AB0
:10DC40008CE40E946339882309F468C00E94393942
:10DC50006B017C0120E030E0A901C701B6010F94FF
:10DC6000D17387FF04C0F7FAF094F7F8F094C98AEB
:10DC7000DA8AEB8AFC8A2091921530919315243030
:10DC8000310574F08091901590919115821B930B42
:10DC900097FF03C091958195910901E004970CF4D9
:10DCA00000E063E080E00E94416D811140C083E0AC
:10DCB00080933002109262050E945F9B6D817E818D
:10DCC0008F8198858B019C01305809831A832B839F
:10DCD0003C8320E030E0A9010F947F6A882321F083
:10DCE000CE0101960E94B22A109262050E945F9BAB
:10DCF00064960FB6F894DEBF0FBECDBFDF91CF9113
:10DD00001F910F91FF90EF90DF90CF90BF90AF9059
:10DD10000895E12CF12C00E211E443CFC0901506E8
:10DD2000D0901606E0901706F090180693CF83E087
:10DD3000E82E22E0AE01475F5F4FBE016F5E7F4F6E
:10DD4000CE010D960F94DF43B9CF6F927F928F92E1
:10DD50009F92AF92BF92CF92DF92EF92FF920F937A
:10DD60001F93CF93DF9300D000D01F921F92CDB7A7
:10DD7000DEB75C014B013A01F22E68010091A10669
:10DD800010929D0610929E0610929F061092A00679
:10DD90001092A1060F94404E809192159091931588
:10DDA0008C159D051CF4C6010E94A2F360E080E082
:10DDB0000E94416D811124C1109262050E945F9BF7
:10DDC0001C141D0444F4C6010E94A2F340E060E06C
:10DDD00080E00F940F2440E060E088E00E94489CBF
:10DDE00060E081E00E94416D80E090E0A0E7B2E455
:10DDF00089839A83AB83BC8380E090E0A0E8B0EC99
:10DE00008D839E83AF83B887BE016F5F7F4FCE0146
:10DE100005960F94800887E00F941206811158C070
:10DE20008091D5099091D609A091D709B091D809D0
:10DE30004091010550910205609103057091040520
:10DE4000C090FD04D090FE04E090FF04F090000527
:10DE5000C092A108D092A208E092A308F092A40870
:10DE60004093A5085093A6086093A7087093A8084C
:10DE70008093A9089093AA08A093AB08B093AC082C
:10DE800080E090E0A8E4B2E489839A83AB83BC830A
:10DE9000CE0101960F942D108091050590910605F5
:10DEA000A0910705B09108058093A9089093AA084E
:10DEB000A093AB08B093AC0880E090E0A0EAB0E497
:10DEC00089839A83AB83BC83CE0101960F942D1076
:10DED000C12CD12C80E7E82E82E4F82EC982DA82A8
:10DEE000EB82FC8280E090E0A0E8B0E48D839E832A
:10DEF000AF83B887BE016F5F7F4FCE0105960F9449
:10DF0000800820E030E0A9016091090570910A05C0
:10DF100080910B0590910C050F947F6A87FF0BC0D1
:10DF2000C982DA82EB82FC82BE016F5F7F4F89E09B
:10DF300095E00F9480088091090590910A05A091C1
:10DF40000B05B0910C058093D9099093DA09A09341
:10DF5000DB09B093DC098093AD089093AE08A093E1
:10DF6000AF08B093B0088DEA98E00F944A0480910E
:10DF7000190681110F943258109262050E945F9B1E
:10DF800061E085E49BE00E9414458091A9068150E0
:10DF90008093A90645E651E26DE47BE085E00F94AD
:10DFA000E9448091A906882339F00E94DEE180913E
:10DFB000A90681508093A90680E00F9499430E949E
:10DFC000BE268091D608823011F40F94C0170F94AA
:10DFD00077430E945F9B28960FB6F894DEBF0FBE72
:10DFE000CDBFDF91CF911F910F91FF90EF90DF9008
:10DFF000CF90BF90AF909F908F907F906F9008953B
:10E00000E12C2F2DA301B401C5010F94DF43D8CE1D
:10E010004F925F926F927F92AF92BF92CF92DF92B8
:10E02000EF92FF921F93CF93DF9300D000D01F9207
:10E030001F92CDB7DEB75C01E62EF42E642F80E090
:10E040000E94416D182F81111BC0EE2021F010920B
:10E0500062050E945F9B812F28960FB6F894DEBF61
:10E060000FBECDBFDF91CF911F91FF90EF90DF905A
:10E07000CF90BF90AF907F906F905F904F9008953A
:10E08000EE2029F040E06F2D83E00E94489C80E064
:10E0900090E0A0E7B2E48D839E83AF83B88780E0F1
:10E0A00090E0A0E8B0EC89839A83AB83BC83BE0187
:10E0B0006B5F7F4FCE0101960F94800868E873E193
:10E0C00080E090E00E944E40C12CD12C88ECE82EDC
:10E0D00081E4F82ECD82DE82EF82F88680E090E047
:10E0E000A0E8B0E489839A83AB83BC83BE016B5FF5
:10E0F0007F4FCE0101960F94800840905A105090A7
:10E100005B1060905C1070905D10C0925A10D092BD
:10E110005B10E0925C10F0925D1080E090E0A0E275
:10E12000B2E48D839E83AF83B887F50180819181AE
:10E13000A281B38189839A83AB83BC83BE016B5F69
:10E140007F4FCE0101960F94800840925A10509252
:10E150005B1060925C1070925D10129A64E670E041
:10E1600080E090E00E944E4076CF8F929F92AF92D7
:10E17000BF92CF92DF92EF92FF921F93CF93DF93E4
:10E1800000D000D01F921F92CDB7DEB70E94825AF6
:10E19000182F87FDADC08AE50E94B139812C912CE2
:10E1A00090E2A92E91E4B92E882341F040E050E09E
:10E1B000BA018AE50E94373A4B015C01412F64E0C5
:10E1C00083E00E94489C20E030E0A901C501B40131
:10E1D0000F94D17318167CF580E090E0A0EAB0E4CB
:10E1E0008D839E83AF83B8872091D5093091D6095E
:10E1F0004091D7095091D809C501B4010F947171AC
:10E200006B017C0120E030E048EC53E40F947F6A1E
:10E2100087FD06C0C12CD12C88ECE82E83E4F82EB3
:10E22000C982DA82EB82FC82BE016B5F7F4FCE0136
:10E2300001960F94110885E50E946339882309F43B
:10E2400069C00E9439396B017C0120E030E0A901EE
:10E25000C701B6010F94D17387FF04C0F7FAF09499
:10E26000F7F8F094F7FAF094F7F8F094C982DA82AC
:10E27000EB82FC8244E061E0CE0101960E940870CE
:10E2800020E030E0A901C501B4010F94D173181644
:10E290005CF580E090E0A0EAB0E48D839E83AF83DC
:10E2A000B887A50194016091D5097091D609809134
:10E2B000D7099091D8090F9470716B017C0120E00F
:10E2C00030E0A9010F94D17318161CF0C12CD12C89
:10E2D0007601C982DA82EB82FC82BE016B5F7F4FDE
:10E2E000CE0101960F941108109262050E945F9B67
:10E2F00028960FB6F894DEBF0FBECDBFDF91CF9149
:10E300001F91FF90EF90DF90CF90BF90AF909F90C4
:10E310008F90089588E01802F0011124EF5EF94F04
:10E32000C080D180E280F38090CFBF92CF92DF9205
:10E33000EF92FF920F931F93CF93DF9300D01F9222
:10E34000CDB7DEB77C016B018A01B22E61E088E3B4
:10E350009BE00E94144545E651E26FE37BE085E0D7
:10E360000F94E9449091A90681E0890F8093A90652
:10E370008091A01682FF06C08B7F8093A0169E5FBF
:10E380009093A9060F94F81780E1EDECF9E0ADEF5A
:10E39000B4E001900D928A95E1F70E9420F481E0AB
:10E3A0000F94994320E030E0A901F7016081718169
:10E3B000828193810F947F6A8823F1F080911D0AF6
:10E3C00081110CC08091890290918A02019720915D
:10E3D0009015309191152817390774F080E090E07E
:10E3E000A0E7B2E489839A83AB83BC83BE016F5FED
:10E3F0007F4FC7010F94800887E00F9412068111A8
:10E4000003C0B6010F94501B20E030E0A901F801D1
:10E4100060817181828193810F947F6A882329F0C2
:10E4200042E06B2DC8010E940870129A64E670E009
:10E4300080E090E00E944E4081E00F900F900F909E
:10E440000F90DF91CF911F910F91FF90EF90DF9090
:10E45000CF90BF900895CF92DF92EF92FF92CF932B
:10E46000DF936B017C01D42FC091BD0883E08093C2
:10E47000BD0881E08093BC08C114D104E104F1041B
:10E4800031F00F94344EC60ED71EE81EF91E80914F
:10E49000BC08882389F0C114D104E104F10421F4FB
:10E4A0008D2F0E942061F3CF0F94344E6C197D099B
:10E4B0008E099F0997FDF4CF1092BC08C093BD0848
:10E4C000DF91CF91FF90EF90DF90CF9008951F9351
:10E4D000CF93DF93D82FC62F0E944C5D61E08C2F25
:10E4E0000E94D43B0F94344E685370458F4F9F4F1A
:10E4F00060939D0670939E0680939F069093A0065E
:10E500001092A1061091BD0883E08093BD0830E011
:10E5100020E04BED55E46AE27BE082E00E946D452D
:10E5200081E08093BC088091BC08882309F463C013
:10E5300060E08C2F0E94D43B8091A106882309F4CF
:10E5400056C040E060E08AE00E94489C0E94E35987
:10E5500080E19BE00E94514330E020E04AEF5AE026
:10E5600061E07BE082E00E946D4541E060E070E0A8
:10E57000CB010E942B7230E020E050E040E06DEED5
:10E580007AE085E00E946D4510929D0610929E06ED
:10E5900010929F061092A0061092A1060F94404E72
:10E5A00060E080E00E94416D8D2F0E944C5D0F94D1
:10E5B000344E685370458F4F9F4F60939D06709304
:10E5C0009E0680939F069093A0061092A10630E0CD
:10E5D00020E04BED55E461EE7AE082E00E946D456B
:10E5E00081E08093BC0861E08C2F0E94D43B81E0E5
:10E5F0000E94206198CF1093BD08DF91CF911F91A9
:10E600000895CF92DF92EF92FF920F931F93CF93D3
:10E61000DF93CDB7DEB7A0970FB6F894DEBF0FBE7D
:10E62000CDBF0E94825A87FDD1C0482F61E081E0B2
:10E630000E94489C85E40E946339882309F4D5C070
:10E640000E9439396B017C0120E030E0A9010F9470
:10E65000D17387FF04C0F7FAF094F7F8F094F7FA53
:10E66000F094F7F8F094C98ADA8AEB8AFC8A8CE095
:10E67000EBE9F2E0DE01119601900D928A95E1F747
:10E680008AE50E94B139882351F040E050E0BA0198
:10E690008AE50E94373A69877A878B879C8788E565
:10E6A0000E94B139882351F040E050E0BA0188E57A
:10E6B0000E94373A69837A838B839C8389E50E9421
:10E6C000B139882351F040E050E0BA0189E50E9459
:10E6D000373A6D837E838F83988785E50E946339FF
:10E6E000882309F489C00E9439396B017C0120E03C
:10E6F00030E0A901C701B6010F94D17387FF04C0B0
:10E70000F7FAF094F7F8F094F7FAF094F7F8F09439
:10E71000CD8ADE8AEF8AF88E198E1A8E1B8E1C8E99
:10E720008CE40E946339882309F46FC00E94393950
:10E730006B017C0120E030E0A901C701B6010F9414
:10E74000D17387FF04C0F7FAF094F7F8F094CD8EF8
:10E75000DE8EEF8EF8A262E070E082E40E94823BDF
:10E76000F82E8091A906811131C021E0AE014B5EE7
:10E770005F4FBE016F5F7F4FCE0141960E94957142
:10E78000882321F16F2D81E00E94677282E50E944B
:10E79000B139882309F442C00E94353940E050E085
:10E7A00060EA71E44D875E876F87788B2091A906B8
:10E7B000222361F08C012F2DAE01435F5F4FBE011C
:10E7C000635E7F4FCE0149960E94A56EA0960FB65C
:10E7D000F894DEBF0FBECDBFDF91CF911F910F9197
:10E7E000FF90EF90DF90CF900895C12CD12C80E85E
:10E7F000E82E80E4F82E33CFC0901106D090120698
:10E80000E0901306F090140672CFC0901506D090D9
:10E810001606E0901706F09018068CCF90E080E086
:10E82000BDCFCF92DF92EF92FF920F931F93CF93C2
:10E83000DF93CDB7DEB76C970FB6F894DEBF0FBE8F
:10E84000CDBF8CE40E946339882309F4C3C00E94C1
:10E8500039396B017C0120E030E0A9010F94D173BC
:10E8600087FF04C0F7FAF094F7F8F094F7FAF09401
:10E87000F7F8F094C98EDA8EEB8EFC8E8CE0EBE923
:10E88000F2E0DE01119601900D928A95E1F788E59C
:10E890000E94B1398823A1F040E050E0BA0188E538
:10E8A0000E94373A2091C1093091C2094091C309B1
:10E8B0005091C4090F94707169837A838B839C8310
:10E8C00089E50E94B1398823A1F040E050E0BA0107
:10E8D00089E50E94373A2091C1093091C2094091DF
:10E8E000C3095091C4090F9470716D837E838F8327
:10E8F00098878AE50E94B139882351F040E050E0C2
:10E90000BA018AE50E94373A69877A878B879C87A4
:10E91000F090A016F2FAFF24F0F840E061E080E009
:10E920000E94489C60E080E50E94913BE82E1D8695
:10E930001E861F86188A8091A90681113CC02E2D43
:10E94000AE01435F5F4FBE016F5F7F4FCE014996BF
:10E950000E949571882379F18091190681110F9495
:10E960003258FF2011F0EE2031F160E080E00E948B
:10E970006772898D9A8DAB8DBC8DB0588D8B9E8BB7
:10E98000AF8BB88F198A1A8A1B8A1C8A1D861E862D
:10E990001F86188A8091A906882369F010E000E09C
:10E9A00020E0AE014B5E5F4FBE016F5E7F4FCE0138
:10E9B0000D960E94A56E6C960FB6F894DEBF0FBE42
:10E9C000CDBFDF91CF911F910F91FF90EF90DF901E
:10E9D000CF900895C12CD12C80E8E82E80E4F82E49
:10E9E00045CF2F923F924F925F926F927F928F927C
:10E9F0009F92AF92BF92CF92DF92EF92FF920F93CE
:10EA00001F93CF93DF93CDB7DEB7E5970FB6F8949A
:10EA1000DEBF0FBECDBF8DAB2091BD082CAB21E07A
:10EA20002093BD0880914C058D3409F409C68435C6
:10EA300011F40C941F8A873409F091C180914A0522
:10EA400090914B058B31910509F4DDC108F079C136
:10EA50008430910508F030C120916C088230910516
:10EA600008F48EC1213009F091C111E0029709F03C
:10EA700010E00E944E3A19821A821B821C821D826B
:10EA80001E821F82188682E50E94B139882309F40C
:10EA900090C10E9439396B017C0120E030E0A9016E
:10EAA0000F947F6A882309F4EAC04090CD09509002
:10EAB000CE096090CF097090D0098091D1099091D2
:10EAC000D209A091D309B091D4098CA79DA7AEA774
:10EAD000BFA78090A1089090A208A090A308B09032
:10EAE000A4088091A5089091A608A091A708B091CC
:10EAF000A80888AB99ABAAABBBABA5019401C30135
:10EB0000B2010F947F6A81110DC028A939A94AA9C1
:10EB10005BA96CA57DA58EA59FA50F947F6A882310
:10EB200009F4ADC0A3019201C501B4010F94707145
:10EB300020E030E040E05FE30F94E56A68A779A742
:10EB40008AA79BA72CA53DA54EA55FA568A979A975
:10EB50008AA99BA90F94707120E030E040E05FE348
:10EB60000F94E56A2B013C0120E030E0A901C701C8
:10EB7000B6010F947F6A881F8827881F181709F429
:10EB80000FC180E090E0A0E8BFEB8CA79DA7AEA7E7
:10EB9000BFA728A539A54AA55BA5CA01B9010F944D
:10EBA000E56A4B015C01A3019201C301B2010F941C
:10EBB000E56A9B01AC01C501B4010F9471710F941A
:10EBC0001F744B015C01AC019B01C701B6010F949E
:10EBD000707168AB79AB8AAB9BABA5019401C7019F
:10EBE000B6010F9471719B01AC0168A979A98AA93A
:10EBF0009BA90F94E56A6B017C0120E030E0A9013C
:10EC00000F94D17387FDD1C0C701B6010F941F7453
:10EC10006B017C01C301B2019058A50194010F94CE
:10EC20006B722CA53DA54EA55FA50F94E56AA701C3
:10EC300096010F94E56A28A539A54AA55BA50F940E
:10EC4000717169837A838B839C83A501940168A584
:10EC500079A58AA59BA50F946B722CA53DA54EA501
:10EC60005FA50F94E56AA70196010F94E56AA301D9
:10EC700092010F9471716D837E838F83988720E05A
:10EC800030E0A90169817A818B819C810F947F6A30
:10EC90008111A3C020E030E0A9016D817E818F81C8
:10ECA00098850F947F6A811198C00E94DF598CE388
:10ECB00091E10E9451436AC08531910509F466C013
:10ECC0008A31910509F49CC0049709F048C080E599
:10ECD0000E94B139C12CD12C7601882321F00E94E9
:10ECE0002A2C6B017C0183E50E94B139882361F0F5
:10ECF0000E94393920E030E04AE754E40F94E56A95
:10ED00000F94E4726B017C010E9420F48091211326
:10ED1000811105C060E082E591E10E9447CB0F942C
:10ED2000344EC60ED71EE81EF91E0F94344E6C19D1
:10ED30007D098E099F0997FF29C080E00E9420610C
:10ED4000F4CF8A32910509F4F0C260F48D31910557
:10ED500009F418C208F470C04E9709F46CC20F94FD
:10ED6000D14314C08B35910509F4C2C38C3591058C
:10ED700009F4C2C38A35910591F71092D70806C0ED
:10ED8000213021F40E944E3A0F947A0DFDA9F11121
:10ED900002C00F94954E2CA92093BD080C94B48208
:10EDA00080E090E0A0E8BFE3F0CEC12CD12C76014A
:10EDB00031CF89E40E94B139882331F00E9439397A
:10EDC00069837A838B839C838AE40E94B139882388
:10EDD00009F455CF0E9439394ECF412FBE016F5FE4
:10EDE0007F4F81EA98E00F942E4F0F94344E60933A
:10EDF000B3087093B4088093B5089093B608C6CF53
:10EE00000E94E750C3CF87E00F94FC2C8111BECF46
:10EE10008CE0E7EAF2E0DE01119601900D928A950E
:10EE2000E1F770E060E080E50E94BE39BE016F5FEF
:10EE30007F4F0F94501BAACF87E00F9412068111C9
:10EE400006C060E08FE40E94913B81119FCF0E9439
:10EE500020F4109240026091DC088CE40E94913B07
:10EE6000E82E80E00E94623E0F94344E6093B30817
:10EE70007093B4088093B5089093B6080F94F90680
:10EE800081E0809326080F94EC118AE50E94633993
:10EE9000F82E882369F081E00F941206182F82E083
:10EEA0000F94120611110C94848A11E0811101C093
:10EEB00010E088E50E946339082F81110C94348A90
:10EEC00011110CC089E50E946339811342C1012FE1
:10EED000F11204C001E011E0FF24F39482E50E94E6
:10EEE000B139882309F438C10E9439396CA37DA354
:10EEF0008EA39FA320E030E0A9010F947F6A8823AE
:10EF000081F0011105C0111103C0FF2009F410C1E7
:10EF100060E0CE0184960F9430080E94A1420E94C6
:10EF20005042002309F47FC0112309F479C01092E4
:10EF3000CD091092CE091092CF091092D0091092EB
:10EF4000D1091092D2091092D3091092D4090F94CA
:10EF50003C0985E39DE20E9406344B015C0189E394
:10EF60009DE20E9406342B013C01AC019B01C501CE
:10EF7000B4010F94D17318160CF0F3C0A5019401DD
:10EF8000C301B2010F946B729B01AC010F94E56A4F
:10EF900020E030E040E85FE30F9471710F941F743C
:10EFA00020E030E048E452E40F94E56A68A379A3D6
:10EFB0008AA39BA320E030E040EC5FE3C301B201F1
:10EFC0000F94E56A905869837A838B839C8320E051
:10EFD00030E040EC5FE3C501B4010F94E56A90585E
:10EFE0006C8F7D8F8E8F9F8FAE01405E5F4FBE0115
:10EFF0006F5F7F4FCE014C960F94EF070F9428144C
:10F000001092CD091092CE091092CF091092D0091A
:10F010001092D1091092D2091092D3091092D409FA
:10F0200080E00F941D15112319F081E00F941D1538
:10F03000FF2009F47DC083E00F94FC2C811178C07F
:10F040000F943C092091030930910409409105096E
:10F050005091060960E070E086E193E40F947071CE
:10F060002B013C01209107093091080940910909C1
:10F0700050910A0960E070E086E193E40F947071AA
:10F080004B015C018091D5099091D609A091D709D7
:10F09000B091D8098093A9089093AA08A093AB08CF
:10F0A000B093AC080091291610912A16D8012D9121
:10F0B0003D914D915C91C301B2010F9470716093C9
:10F0C000A1087093A2088093A3089093A408F80164
:10F0D0002481358146815781C501B4010F94707137
:10F0E0006093A5087093A6088093A7089093A8083A
:10F0F00081EA98E00E94ED248823C1F11C8E1D8EC8
:10F100001E8E1F8E88E0E1EAF8E0DE011196019084
:10F110000D928A95E1F7AE01445E5F4FBE016B5FD1
:10F120007F4FCE0101960F94EF0782E00F941D15DB
:10F130000F943C0980912508809326088E2D0E940B
:10F14000623E0F94E00683E0809384020F94BD102A
:10F150001DCE012F182FC2CE60E070E080E890E451
:10F16000C5CEA3019201C501B4010CCF60E08DE6CC
:10F1700091E10E9447CB0E94E3598BE591E10E9407
:10F180005143D6CF14E00F94344E6093B30870937C
:10F19000B4088093B5089093B6088091DC0881117B
:10F1A00027C08EE40E946339882321F08EE791E125
:10F1B0000E94B78A87E00F94FC2C81111FC00E9427
:10F1C00054688823D9F0115001F130E020E045E681
:10F1D00051E269EA71E185E00E946D4561E08CE9E8
:10F1E00091E10E94144584E891E10E94B78ACBCF57
:10F1F00060E08FE40E94913B882399F20E9445458C
:10F2000087E492E10E94B78AC1CD61E08AE392E18E
:10F210000E94144585EC91E10E94B78A61E080E587
:10F2200091E20E94144540E070E060E086EB91E1DD
:10F230000E940C5EABCD0091291610912A16D801C0
:10F240002D913D914D915C916091CD097091CE09C8
:10F250008091CF099091D0090F947171AB01BC01DD
:10F2600088E50E94373A69837A838B839C83F8010F
:10F2700024813581468157816091D1097091D209ED
:10F280008091D3099091D4090F947171AB01BC01A5
:10F2900089E50E94373A6D837E838F839887BE010C
:10F2A0006B5F7F4FCE0101960E941534882309F4CD
:10F2B0006DCD80E00E94623E0F94F90661E085E426
:10F2C0000E94913B182F21E0482FBE016B5F7F4FBA
:10F2D000CE0101960F94F2446B017C01AC019B01BD
:10F2E0000F946374811119C049815A816B817C81AB
:10F2F00089E692E10E943B464D815E816F8178856F
:10F3000084E692E10E943B46B701A6018FE592E1B7
:10F310000E943B468AE00E9418430F94E0061111B8
:10F320000E94102C0F94BD1031CD80916C0881305B
:10F3300009F02CCD89E40E94B139082FF12C8823E3
:10F3400019F00E943539F82E8AE40E94B139E82E6E
:10F35000882379F00E943539182F002309F4C0C0A2
:10F36000F4E0FF1508F0B9C081E792E10E94514333
:10F370000DCD10E00111F4CF80E1EDECF9E0A1EA50
:10F38000B8E001900D928A95E1F7002319F16F2DF5
:10F39000FF0C770B880B990B0F94866A20918606D9
:10F3A0003091870640918806509189060F94E56A4E
:10F3B00020917E0630917F06409180065091810613
:10F3C0000F9471716093A1087093A2088093A308B1
:10F3D0009093A408EE2019F1612F110F770B880B81
:10F3E000990B0F94866A20918A0630918B06409182
:10F3F0008C0650918D060F94E56A2091820630911B
:10F40000830640918406509185060F947171609334
:10F41000A5087093A6088093A7089093A80860E0B9
:10F4200080E50E94913B8823C1F10023D1F0E09157
:10F430002916F0912A1620813181428153816091F1
:10F44000A1087091A2088091A3089091A4080F943C
:10F4500070716093A1087093A2088093A3089093A1
:10F46000A408EE20D1F0E0912916F0912A1624810B
:10F470003581468157816091A5087091A6088091D9
:10F48000A7089091A8080F9470716093A5087093D5
:10F49000A6088093A7089093A80840E050E0BA011E
:10F4A00086E40E94373A6B017C0120E030E0A9013C
:10F4B0000F94D1731816C4F420E030E040E752E412
:10F4C000C701B6010F946B7269837A838B839C8327
:10F4D000CE0101960F942D1059CCEE2009F44CCF9B
:10F4E000153008F449CF40CF60E070E0CB01ECCF9D
:10F4F0008FE08093D7084ACC80914905882381F119
:10F50000893009F043CC63EBA62E62E0B62E7DEC89
:10F51000C72E79E0D72EE12C00E010E0D5018D91C7
:10F520005D010E94B139F82E882361F0133011F487
:10F53000082FFE2C0E943939F60160837183828383
:10F540009383EF2C1F5FF4E0CF0ED11C143031F702
:10F55000EE2009F457C00F943C090F94BD1016CC4F
:10F5600053EBC52E52E0D52EF12CE12C00E010E03B
:10F57000D6018D916D010E94B139382E8823D9F1C1
:10F580000E9439394B015C01133059F0F701EF53F8
:10F59000F64F20813181428153810F9470714B016C
:10F5A0005C01F701E353F64F2081318142815381A1
:10F5B000C501B4010F9470712B013C012DEB37E3B1
:10F5C00046E855EB0F94D17387FD0AC02DEB37E366
:10F5D00046E855E3C301B2010F947F6A18165CF444
:10F5E0001330C1F48092D9099092DA09A092DB0914
:10F5F000B092DC09032D1F5FB4E0EB0EF11C143058
:10F6000009F0B6CF002309F4A8CF89ED99E00F9453
:10F610004A04A3CFF701E950F74F5F01A30192011C
:10F6200060817181828193810F947171D5016D9395
:10F630007D938D939C931397812F0F94F205DBCFCD
:10F6400080914A0590914B058937910511F40C94EE
:10F65000B08408F0C4C18D34910509F47FC608F068
:10F66000D0C08A31910509F4B4C508F073C0843163
:10F67000910509F4FAC408F050C08131910509F4EC
:10F68000BBC408F044C0029708F069CB80E50E9433
:10F69000B139C12CD12C7601882321F00E942A2C6B
:10F6A0006B017C0183E50E94B139882361F00E94DF
:10F6B000393920E030E04AE754E40F94E56A0F94CA
:10F6C000E4726B017C010E9420F4809151059091BD
:10F6D0005205009709F48AC40F94F33380914A05C8
:10F6E00090914B0562E972E1892B11F46AE872E1AD
:10F6F00030E020E04BED55E482E00E946D4540E0B3
:10F70000C701B6010E942B720F9477433FCB4297FB
:10F7100009F025CB0E94CC3939CB8731910509F40A
:10F72000D9C470F48531910509F4D0C4469709F025
:10F7300016CB8091A01682FD29CB0E9485E926CBAD
:10F740008831910509F4DBC4499709F008CB0E9480
:10F7500011741CCB8032910509F4BFC5C0F58D3101
:10F76000910509F4A3C570F48B31910509F444C5E2
:10F770004C9709F0F4CA80915105909152050F946D
:10F78000C05A04CB8E31910509F497C54F9709F003
:10F79000E6CA0F94FE166C8F7D8F8E8F9F8FBE01F1
:10F7A0006F5F7F4FCE014C960E94BD31CE01019616
:10F7B0000F94F3330E94E359BE016F5F7F4F85E0E2
:10F7C00093E10E9451608AE00E941843DFCA8934A5
:10F7D000910509F4AFC550F48132910509F4A6C52D
:10F7E000C09709F0BCCA0E94114DD0CA8B34910554
:10F7F00009F4B0C58C34910509F0B1CA0F94F8171B
:10F80000C5CA8C36910509F4C1CA08F083C0853594
:10F81000910509F492C790F58235910509F47DC7E9
:10F8200020F58E34910509F49DC58135910509F0C7
:10F8300096CA0E9486EC0E9431F40E94D4400E9435
:10F84000D7401092C8081092C7081092C60868EEF8
:10F8500073E080E090E00E944E400E94D32660E07A
:10F8600080ED93E10E9447CB91CA8335910509F45D
:10F870005CC78435910509F44DCF71CA893691056D
:10F8800009F460C690F58C35910509F47BC788367C
:10F89000910509F064CA8091211083FD77CA0E9406
:10F8A000825A87FD73CA89E40E94B139882311F412
:10F8B0000C943A8A0E945B2C90E01816190614F4F6
:10F8C00081E090E026E0289FF001299FF00D1124AF
:10F8D000E359F74F808191810E94A2F361E080E0BB
:10F8E0000F94215E0F943A5E51CA8A36910509F44D
:10F8F00054C68B36910509F032CA60E080E50E945B
:10F900002B3A823008F042CAE82FF0E0E55FF54F6D
:10F9100010823CCA8237910509F4D5C7A0F58F360D
:10F92000910509F474C6C8F48D36910509F4ACC587
:10F930008E36910509F013CA8EE40E94B1398823EE
:10F9400009F424CA0E944B2C6093EC107093ED10C4
:10F950008093EE109093EF1019CA8037910509F447
:10F9600015CA8137910509F0FAC983E50E94B139BA
:10F97000882309F493C60E945B2C8D3308F089C656
:10F9800080931F0203CA8637910509F4ACC7B8F407
:10F990008337910509F49FC78537910509F0DFC9C1
:10F9A0008091510590915205009709F498C7DC01A8
:10F9B0002C91222309F493C70F94F333E7C98737B7
:10F9C000910509F4C9C78837910509F0C8C981E0D4
:10F9D00080932608809325080F94EC11D7C98239AB
:10F9E000E1E09E0711F40C94D58708F095C1833DA2
:10F9F000910511F40C94948508F0F6C0883C9105AB
:10FA000011F40C94318508F06CC08139910509F42A
:10FA1000AFC760F58D37910509F499CE8C38910503
:10FA200009F09DC98091211083FDB0C989E40E942D
:10FA3000B139882311F40C94608A0E945B2C90E009
:10FA40001816190614F481E090E026E0289FF001D2
:10FA5000299FF00D1124E359F74F828193810E9471
:10FA60002A3961E080E00F94215E90C98B399105BD
:10FA700009F42CC68E3B910509F071C980912110C3
:10FA800083FD84C989E40E94B139882311F40C9460
:10FA90006B8A0E945B2C90E01816190614F481E022
:10FAA00090E026E0289FF001299FF00D1124E359F2
:10FAB000F74F8281938110E00E942A3960E081E053
:10FAC0000F94215E2091E3083091E4088091E108D1
:10FAD0009091E208821793070CF0EDC581EC93E159
:10FAE000ECC58C3C910511F40C948C8540F5893C57
:10FAF000910509F4E7C78B3C910509F030C90E94D4
:10FB0000825A87FD43C913EBE12E12E0F12E10E07B
:10FB100000E0D7018D917D010E946339882349F06F
:10FB20000E943939F801EE5DFF4E64A375A386A3E8
:10FB300097A30C5F1F4F0031110559F727C98D3C62
:10FB4000910511F40C949085B3E0EB2EB9E0FB2EF7
:10FB500010E08E3C910509F002C988E5810F0E94F2
:10FB60006339882351F00E943939F701608371832A
:10FB700082839383812F0F94F2051F5FF4E0EF0ED1
:10FB8000F11C133051F780914F0587FDE6CC809131
:10FB90005005837009F0E1CC4091030950910409AC
:10FBA000609105097091060986E094E10E943B4648
:10FBB00040910709509108096091090970910A095B
:10FBC00084E696E40E943B4640910B0950910C0953
:10FBD00060910D0970910E0981E696E40E943B4602
:10FBE0008AE00E941843D2C88D3221E0920711F4B6
:10FBF0000C94958608F06AC08831A1E09A0711F448
:10FC00000C94F58508F043C08C3D910509F490C72C
:10FC10008D3D910509F0A3C80E94825A082F87FDE7
:10FC2000B5C883E50E94B139002E000C110B780194
:10FC3000EE0CFF1C882309F4BEC70E943539F7017A
:10FC4000E35CFD4F91838083000F111F000F111F94
:10FC500098012B573D4F7901BC01990F880B990BE7
:10FC60000F94866A2AE037ED43E25CE30F94E56A7D
:10FC70000B5F194FD8012D913D914D915C910F94DF
:10FC8000E56AF70160837183828393837FC8823240
:10FC9000E1E09E0711F40C9491868C32914009F0BA
:10FCA0005EC864E071E083E50E94BE398C0168EEB5
:10FCB00073E080E50E94BE39893823E1920710F095
:10FCC00088E893E1B8010E946A9660C8803321E019
:10FCD000920711F40C94178768F48E32A1E09A070A
:10FCE00011F40C948B878F32914009F038C80E9430
:10FCF000D1464CC88039E1E09E0711F40C94D187BD
:10FD00008139914009F02BC88091B208811125CC2E
:10FD100081E00F94A21321CC883F31E0930711F4C6
:10FD20000C94478908F0E6C08C3AB1E09B0711F4C7
:10FD30000C941C8808F0B3C08D39F1E09F0711F4D2
:10FD40000C94028A88F58A3931E0930709F41EC8B9
:10FD50008C39914011F00C94AF7680914D058878E4
:10FD600011F00C94DD8780914F05867011F00C9492
:10FD7000DD870E94E35983EB94E10E945143809117
:10FD80005D020E941D464091590250915A026091B5
:10FD90005B0270915C0283E994E10E943B468AE039
:10FDA0000E9418430C94C676843AB1E09B0711F484
:10FDB0000C940D88853A914011F00C94AF766FEF5A
:10FDC0007FEF89E40E94823B082F6FEF7FEF8AE488
:10FDD0000E94823B182F8AE50E94B139D12C8111F3
:10FDE00008C081E50E94B139D82E882311F40C9403
:10FDF0007C8AC02E81E0800F863010F00C9414882D
:10FE0000912E81E0810F863010F00C9414880E94AE
:10FE100039392B013C01F02E07FDF12C07FF02C000
:10FE200004E0C02E812E17FD812C17FF02C014E0C4
:10FE3000912EB5E03B2ECF1410F40C94C676E82C2E
:10FE40003F9C500111249E1410F40C9411880E2D27
:10FE500010E020E030E0A901DD2069F0F501E00FBD
:10FE6000F11FEE0FFF1FEE0FFF1FE65EF94F20811F
:10FE70003181428153810A0D1B1D000F111F000F9C
:10FE8000111F065E194FC301B2010F947171D801A1
:10FE90006D937D938D939C931397E394D4CF853F7B
:10FEA000F1E09F0711F40C943F8978F4863E31E02D
:10FEB000930711F40C94CD88843F914011F00C9479
:10FEC000AF760E9405F00C94C676863FB1E09B07A2
:10FED00011F40C944389873F914011F00C94AF7654
:10FEE00061E083E50E94913B91E089270F949D2575
:10FEF0000C94C6768335F3E09F0711F40C94EE89D9
:10FF000028F58B3532E0930711F40C946A8978F464
:10FF10008C30B2E09B0711F40C94598988359240DB
:10FF200011F00C94AF760E9401730C94C6768D3B51
:10FF3000F2E09F0711F40C94EA898E3B924011F095
:10FF40000C94AF760E94B5700C94C676873E33E071
:10FF5000930711F40C94F289C8F48C36B3E09B0734
:10FF600011F40C94C676803A934011F00C94AF765D
:10FF700020915105309152059091A0169260909376
:10FF8000A016C9010F94C05A0C94C676883EF3E0BF
:10FF90009F0711F40C941B8A893E934011F00C9436
:10FFA000AF760F94395A81110C94C6760E94A63B05
:10FFB0000F94F7590F94FE166D3371058105910565
:10FFC00020F085E795E10E94B78A81E795E10E94DC
:10FFD000B78A84EE80935B058DE595E10E945143DD
:10FFE00089E595E10E94B78A0C94C67660E08AE9BB
:10FFF00092E10E9447CB72CB80914D0584FD17C0E2
:020000021000EC
:1000000080914F0587FD13C080915005837079F46E
:1000100060E08DEA92E10E9447CB5F988A988091D8
:10002000080181708093060112980C94C67688E5C9
:100030000E94633981115F9889E50E9463398111BB
:100040008A988AE50E946339882329F08091080103
:1000500081708093060185E40E946339882311F43E
:100060000C94C67612980C94C6768091A01683FFE5
:1000700025C085EC92E10E9451438091A01683FF38
:1000800017C081EC96E10E9469EA8BE1E1ECF6E1B0
:10009000DE01119601900D928A95E1F770E060E023
:1000A000CE0101960F948C20CE0101960E94CE3B8A
:1000B00086EB92E10E9451430C94C6760E94E3596C
:1000C00086ED92E10E9451430C94C6760E9496E917
:1000D0000C94C6768091510590915205FC012191B6
:1000E000222331F02032D9F7DF0111971C92F7CF8C
:1000F00060E00F94095B10925B050C94C67683E573
:100100000E94B139882321F00E944B2C0E94642A5E
:1001100084E50E94B1398823A9F00E944B2C6B0121
:100120007C010F94A517C0920906D0920A06E092AE
:100130000B06F0920C06CD28CE28CF2819F081E0CE
:100140008093D6088091A9068823F9F080E090E09A
:10015000A0EAB1E489839A83AB83BC831C8E1D8E95
:100160001E8E1F8E18A219A21AA21BA210E000E078
:1001700020E0AE014F5F5F4FBE01645E7F4FCE0156
:1001800080960E94A56E0C94C6760E949D4088239E
:1001900081F00E94DEE10E94C1408DE499E00F945D
:1001A00048591092531110925411109255111092F7
:1001B000561161E08DE991E20E94144545E651E255
:1001C00060EE72E185E00F94E9440F9477430C945C
:1001D000C6768091A01683FD02C00C94C67683E596
:1001E0000E94B139882311F40C94C6760E944B2CDE
:1001F0000E94642A0C94C67683E40E9463398823A3
:1002000061F186EF92E10E945143809108188823A2
:10021000F9F0BE016F5F7F4F85E098E10E94FCE935
:10022000CE0101960E9403E6CE0101960F94925AE8
:100230008091DE12882339F080E20E9418438EED0F
:1002400092E10E9403E68AE00E9418430C94C6766D
:100250008CEE92E10E945143F6CF83E50E94B139C2
:10026000882301F10E945B2C182F8C3308F08CE35B
:10027000809324050F94344E6B017C01212F30E0D4
:10028000A8EEB3E00F941771C60ED71EE81EF91E34
:10029000C0922005D0922105E0922205F09223051C
:1002A0000C94C6760F940F590C94C6768091A016C4
:1002B0008E7F8093A0160C94C6768091A01683FD45
:1002C00002C00C94C6760F94B7438091510590916B
:1002D00052050F948F590C94C6768091A01682FD1A
:1002E0000E9420F48091A01683FD02C00C94C67673
:1002F00060E080E50E94913B182F682F80915105A6
:10030000909152050F94095B83E50E94B1398823CF
:1003100021F00E944B2C0E94642A0E94DEE1111100
:100320000C94C6760E94C1400C94C6760E945B6015
:100330000C94C67680E50E946339882311F40C94EE
:10034000C6760E945B2C853608F084E680935B05B8
:100350000C94C6760E94C1400C94C6760E94D4408C
:100360000C94C67670E060E083E50E94823B8E3498
:10037000910531F40E9441F30F9477430C94C676B3
:1003800080E793E10E94514360911508709116082F
:1003900087E693E10E94294660911708709118083A
:1003A0008AE593E10E94294660911508709116082C
:1003B0008091170890911808681B790B8091D608D6
:1003C000815021E030E0823010F030E020E0621B0C
:1003D000730B8FE493E10E9429468AE00E94184340
:1003E00087E493E10E9451438091190890911A0883
:1003F000A0911B08B0911C088C8F9D8FAE8FBF8F72
:10040000BE016F5F7F4FCE014C960E94BD31BE0191
:100410006F5F7F4F8AE393E10E94516080911D08D6
:1004200090911E08A0911F08B09120088C8F9D8F7D
:10043000AE8FBF8FBE016F5F7F4FCE014C960E9483
:10044000BD31BE016F5F7F4F8AE293E10E94516030
:1004500020E030E04AE754E46091210870912208DE
:1004600080912308909124080F946B72AB01BC011A
:1004700082E193E10E943B468DE60E9418438AE0A8
:100480000E9418430C94C6768091211083FF02C00D
:100490000C94C6760E94825AF82E87FF02C00C94F4
:1004A000C67689E40E94B139882311F40C94458AF8
:1004B0000E945B2C90E01816190614F481E090E07D
:1004C00026E0289FF001299FF00D1124E359F74FF2
:1004D0008081918110E00E94A2F361E081E00F949D
:1004E000215E2091921530919315809190159091F5
:1004F000911582179307F4F483E893E19F938F9308
:100500008EE893E19F938F931F920E942CCB0F90C4
:100510000F900F900F900F9001E00F943A5E002320
:1005200011F40C94C67640E0612F8F2D0F940F24A8
:100530000C94C67688E793E1112301F3012FEDCFE8
:10054000182FEBCF0E94825A182F87FD0AC083E92B
:1005500093E10E945143812F0F9417228AE00E9459
:1005600018433CA93093BD08E5960FB6F894DEBF5A
:100570000FBECDBFDF91CF911F910F91FF90EF90F4
:10058000DF90CF90BF90AF909F908F907F906F90B3
:100590005F904F903F902F90089560E080E50E941B
:1005A0002B3AF82E81E08F1510F40C94C67681E476
:1005B0000E94633960910B0A062F10E0811102C07E
:1005C0000FEF10E089E40E94B139882309F46EC767
:1005D0000E945B2C90E01816190614F481E090E05C
:1005E00026E0289FF001299FF00D1124E359F74FD1
:1005F00004811581EF2DF0E0E55FF54F0F3F110508
:1006000019F010F00FEF10E000830C94C67683E52C
:100610000E946339882331F060E083E50E942B3A21
:10062000809321100E94E35984EA93E10E94514390
:1006300080912110882351F110E000E020E08091AA
:10064000211090E0B0E0A0E0002E04C0B695A79580
:10065000979587950A94D2F780FF12C0FF24F394F0
:10066000F20E222319F08CE20E941843F801EE0FDB
:10067000FF1FE656FC4E859194910E9451432F2D09
:100680000F5F1F4F05301105D1F6DDCD86E993E1EF
:10069000E1CD8CE380931F020C94C6760E94E3594F
:1006A00060911F028BEA93E10E9433468AE00E9428
:1006B00018430C94C67682EB93E160E00E9447CB2E
:1006C00060E0812F0F948A220C94C67683E50E9405
:1006D000B139882311F40C94C6760E945B2C182F34
:1006E0008C3308F08CE3809329050F94344E6B0112
:1006F0007C01212F30E0A8EEB3E00F941771C60EF5
:10070000D71EE81EF91EC0922505D0922605E0925C
:100710002705F09228050C94C6768091D7088F7D26
:1007200080618093D7080C94C6768091D7088F7E1D
:1007300080628093D7080C94C67683E50E94633963
:10074000882311F40C94C6760F94344E6093B3084A
:100750007093B4088093B5089093B6080E94393915
:1007600020E030E04AE754E40F94E56A0F94E47225
:1007700060932A0570932B0580932C0590932D058B
:100780000C94C6760E94825A87FF02C00C94C676EB
:1007900080914D0584FD09C080914F0587FD05C0FE
:1007A00080915005837009F489C023EBC22E22E0AA
:1007B000D22E32E2E32E30E1F32E10E0D6018D91FD
:1007C0006D010E94B139882309F465C0133009F026
:1007D0006DC00E9439394B015C0120E030E040EAF5
:1007E00051E40F947F6A87FF4EC0A5019401609188
:1007F00042107091431080914410909145100F94D5
:100800006B722B013C01AC019B016091EF0970916F
:10081000F0098091F1099091F2090F94E56A6093D3
:10082000EF097093F0098093F1099093F209A30105
:1008300092016091521070915310809154109091D8
:1008400055100F94E56A6093521070935310809383
:100850005410909355106091FF097091000A809197
:10086000010A9091020A0F94846AA30192010F94E5
:10087000E56A0F94E4726093FF097093000A809315
:10088000010A9093020A8092421090924310A09223
:100890004410B09245101F5FF4E0EF0EF11C1430CD
:1008A00009F08CCF0E94FCF30C94C6760E94393973
:1008B000F701648B758B868B978BEDCF81E00F945E
:1008C0003C430C94C6760F94D74280E396E10E9495
:1008D00053EF0C94C6760E9478430C94C6760F941E
:1008E00077430C94C676009151051091520594E01F
:1008F000F12C40E09150F9F0F8018081282F2B7FF6
:10090000213499F421812133B1F4813411F18534FA
:1009100009F441E098012E5F3F4F89012F5F3F4F5F
:10092000F80180818032C9F3E5CF803521F48181DF
:1009300080538A3078F341110E94E359FF2021F05F
:1009400081EE93E10E945143C8010E941F430C9421
:10095000C676FF24F394DECF0F94A1110C94C676D3
:1009600010922608109225080F94EC110C94C6766C
:1009700070E060E083E50E94823B823040F00E949C
:10098000DF5984EE93E10E9451430C94C6768C01AA
:10099000112788E40E94B1398823C1F00E943539BB
:1009A0008A3A91050CF44BC00E943539843B914042
:1009B0000CF048C00E94353926E0209FF001219FAD
:1009C000F00D1124E359F74F9183808382E40E9454
:1009D000B1398823A9F00E9435390597B4F10E94F6
:1009E00035398D389105A4F50E94353926E0209FD0
:1009F000F001219FF00D1124E359F74F9383828377
:100A000086E40E94B139882311F40C94C6760E94C2
:100A1000353997FD20C00E9435398F3F910509F087
:100A2000ECF40E94353926E0209FF001219FF00D63
:100A30001124E359F74F958384830C94C6768AEA90
:100A400090E0BACF83EB91E0B7CF85E090E0CECFD6
:100A50008CE890E0CBCF90E080E0E5CF8FEF90E0A6
:100A6000E2CF0E94825A182F87FF02C00C94C676EC
:100A70000091F60884E40E94B139F82E8823B1F081
:100A80000E9439394B015C0120E030E0A9010F944C
:100A90007F6A8823A9F024E01202F0011124EE50AD
:100AA000F74F80829182A282B3820F2D602F83E55F
:100AB0000E94913B8093F6080E940EDD0C94C6764E
:100AC00080E0F8CF0E94825A87FF02C00C94C6765D
:100AD00003EB12E082E2E82E80E1F82E97EBC92EBC
:100AE00092E0D92ED8018D918D010E94633988231F
:100AF00059F00E9439390F94E472F70160837183D1
:100B0000828393830E94AEF3F4E0EF0EF11CC016D3
:100B1000D10641F70C94C6760E944C460C94C676DA
:100B20000E9413440C94C6760E94A75A0C94C67671
:100B300082E40E946339882341F08091760290918B
:100B40007702909321028093200282E50E9463390C
:100B5000882341F0809120029091210290937702A6
:100B60008093760283E50E94B139882331F00E9498
:100B70003539909377028093760280914D0590915C
:100B80004E05A0914F05B0915005892B8A2B8B2BD8
:100B900011F00C94C67660917602709177028DE028
:100BA00094E10E94C54B85E20E9418438AE00E94AE
:100BB00018430C94C6760E94E35985E40E941843BA
:100BC00080E3800F0E941843F701E35CFD4F6081D2
:100BD000718181E194E10E94C54B85E20E94184336
:100BE0008AE00E9418430C94C67680E50E9463391F
:100BF000882311F40C94C6760E9435398C01892B18
:100C000009F082C083E50E946339882391F00E9435
:100C100035398F3F980731F48AE196E10E94DE4032
:100C20000C94C676BC018AE196E10E944C410C947A
:100C3000C6760E94E35970E060E08CE194E10E9486
:100C4000C54B80911C1658E5C52E52E0D52EC81A0A
:100C5000D10887FDD394CC0CDD1CCC0CDD1C0D2CF5
:100C6000000CEE08FF0880911B1678E8872E912C67
:100C7000881A910887FD9394880C991C880C991CFC
:100C8000092C000CAA08BB0880911A1690E08F3F2F
:100C9000C9F1FC01EE0FFF1FE80FF91FEF52FA4EEA
:100CA0008181928133E0880F991F3A95E1F7B0E096
:100CB000A0E044E0B595A795979587954A95D1F71B
:100CC00002969C012F5F3F4F032E000C440B550BE7
:100CD000281939094A095B09A4EBB0E00F940471A3
:100CE000A7019601281939094A095B090F94E57093
:100CF000B90189E194E10E94C54B8AE00E94184342
:100D00000C94C67680E0DDCF0E94DF59B80183E302
:100D100094E10E94C54B84E294E10E9451430C94FB
:100D2000C6760E94E7590C94C67660E085E40E947E
:100D30002B3A811174C080E50E946339882351F0F9
:100D40000E94393960939515709396158093971585
:100D50009093981589E40E946339882381F00E945A
:100D600039392CEA35EC47E25EE30F94E56A60938B
:100D7000991570939A1580939B1590939C1584E414
:100D80000E946339882381F00E9439392CEA35ECBE
:100D900047E25EE30F946B7260939D1570939E150E
:100DA00080939F159093A0150E94E359409195154B
:100DB00050919615609197157091981582E494E181
:100DC0000E943B462CEA35EC47E25EE360919915C0
:100DD00070919A1580919B1590919C150F946B7250
:100DE000AB01BC018EE394E10E943B462CEA35EC5A
:100DF00047E25EE360919D1570919E1580919F156D
:100E00009091A0150F94E56AAB01BC018AE394E1CF
:100E10000E943B468AE00E9418430C94C6760E94CA
:100E2000DF5986E494E10E9451430C94C67680E534
:100E30000E946339882351F00E9439396093E60893
:100E40007093E7088093E8089093E90889E40E948A
:100E50006339882381F00E9439392CEA35EC47E266
:100E60005EE30F94E56A6093EA087093EB08809361
:100E7000EC089093ED0884E40E946339882381F0A4
:100E80000E9439392CEA35EC47E25EE30F946B722D
:100E90006093EE087093EF088093F0089093F10848
:100EA0000E94E3594091E6085091E7086091E808F4
:100EB0007091E90880E694E10E943B462CEA35EC0B
:100EC00047E25EE36091EA087091EB088091EC08DC
:100ED0009091ED080F946B72AB01BC018CE594E12D
:100EE0000E943B462CEA35EC47E25EE36091EE0857
:100EF0007091EF088091F0089091F1080F94E56AE5
:100F0000AB01BC0188E594E10E943B468AE00E9467
:100F100018430C94C67683E50E946339182F882302
:100F200069F00E9435399C0190938A02809389026E
:100F300091E0232B09F090E090931D0A80E50E9438
:100F40006339882361F02091890230918A02232B32
:100F500011F00E946F2C80931D0A0C94C67611111B
:100F60000C94C6760E94E35980E894E10E945143B4
:100F700080911D0A882391F088E694E10E945143F4
:100F80006091890270918A028FE694E10E94C54BBC
:100F90008BE694E10E9451430C94C67684E694E17A
:100FA000EDCF0E9420F40C94C6760E940C340E946F
:100FB000102C0F94BD100C94C67688E40E946339FF
:100FC000882321F00E946F2C80932E0582E50E94D9
:100FD0006339082F83E50E946339182F011102C07D
:100FE000882341F00E94BE26112321F00E946F2C1D
:100FF00080935D0284E40E946339882311F40C9489
:10100000C6760E9439396093590270935A028093D0
:101010005B0290935C020C94C6760E94965B0C94E3
:10102000C676F3940C941B7F0E94DF5984EE94E102
:101030000E9451430C94C67687E00F94FC2C8111DA
:101040000C94C67669E2C62E6DE2D62EEDECF9E080
:10105000F9A7E8A79E012F5F3F4F1901790110E022
:1010600000E0C6010E940634A8A5B9A58D909D9008
:10107000AD90BD90B9A7A8A7A50194010F94707178
:101080002B013C01F701408251826282738220E091
:1010900030E040EA51EC0F94D17387FD0AC020E0A4
:1010A00030E040EA51E4C301B2010F947F6A1816A0
:1010B00084F4F801E35BF24DE4911E1654F4B7FAA0
:1010C000B094B7F8B094D7018D929D92AD92BC9236
:1010D0001397F70181909190A190B1907F0120E04A
:1010E00030E040EA51ECC501B4010F94D17387FDA3
:1010F0003FC020E030E040EA51E4C501B4010F9464
:101100007F6A1816ACF10F5F1F4FF4E0CF0ED11CB1
:101110000330110509F0A5CF53E0E52E59E0F52E77
:1011200010E0F10181919191A191B1911F01F7011D
:1011300081939193A193B1937F01812F0F94F20535
:101140001F5F133071F70F94BD1060E08DEF94E1D5
:101150000E9447CB63E972E084E690E00E946A96C1
:101160006AEB72E084E690E00E946A960C94C67680
:101170000E94DF598BE195E10E94514361E08DE0CF
:1011800095E10E9447CB0E945F9B68E270E088EC8B
:1011900090E00E946A960C94C67684E50E946339BA
:1011A0008823A1F010925C0510925D0510925E05F7
:1011B00010925F05109260058FEF0E94722A61E025
:1011C00070E084E50E94823B8093600583E50E9485
:1011D0006339882321F00E9435390E94722A83E402
:1011E0000E946339882331F080912F02803210F4FD
:1011F0000E94493C80E50E946339882331F00E94B7
:101200003539803210F40E94493C85E50E946339EB
:10121000882311F40C94C6760E943539803210F080
:101220000C94C67641E050E060E070E0082E04C007
:10123000440F551F661F771F0A94D2F740955095AB
:101240006095709500915C0510915D0520915E059B
:1012500030915F05402351236223732340935C0543
:1012600050935D0560935E0570935F0590912F022A
:1012700089130C94C676109220100C94C6760F94A5
:10128000E62C0C94C6760F94FB110C94C676209332
:101290008E060F94DA2C10928E06882311F40C948B
:1012A000C6760E94E35989E395E10E9451430C946C
:1012B000C6768091A01682FF05C080648093A01638
:1012C0000C94C67683FD02C00C94C6760F94B74387
:1012D0000C94C6760E94825A082F87FF02C00C9495
:1012E000C67685E50E946339882359F10E94393911
:1012F0004B015C01E02E002E000CFF0820E030E0E6
:10130000A9010F94D17387FF04C0B7FAB094B7F85E
:10131000B09420E030E84BE354E4C501B4010F94ED
:10132000D173970143E0220F331F4A95E1F72F5EF7
:10133000394F1816D4F1D9018D929D92AD92BC927D
:1013400013978CE40E946339882311F40C94C676B9
:101350000E9439396B017C01002E000C110B20E03A
:1013600030E0A9010F94D17387FF04C0F7FAF0941D
:10137000F7F8F09420E030E84BE354E4C701B601FD
:101380000F94D173980193E0220F331F9A95E1F7E0
:101390002F5E394F18169CF0D9011496CD92DD922C
:1013A000ED92FC9217970C94C67680E090E8ABE340
:1013B000B4E4F90180839183A283B383C2CF80E038
:1013C00090E8ABE3B4E4F90184839583A683B78303
:1013D0000C94C6760E94AC6D0C94C6760E94CF4BDE
:1013E0000C94C67681E080936C081092761360E0CE
:1013F00083E50E94913B81110C94C6760F94FE34D4
:101400000C94C67683E50E946339882341F00E94DC
:101410006F2C809319060E94AE3B0C94C6760E94F6
:10142000E35984E495E10E945143809119060E949A
:101430001D460C94C6760E94298B0C94C67610919A
:101440004A050F94344E6093B3087093B4088093A8
:10145000B5089093B608112311F40C94C676812F29
:101460000E943CEC0C94C67611110C94677711E045
:101470000C94627783E50E94B139882311F40C94AF
:10148000727C0E9435390C946C7C83E50E94B139E2
:10149000182F811107C082E50E94B139082F8823D7
:1014A00009F44EC80E9435390C946B8283E50E9482
:1014B000B139882309F49EC80E944B2C8B019AC82D
:1014C00083E50E94B139882311F40C94C6760E94FA
:1014D00035390C942F7D83E50E94B139182F811185
:1014E00007C082E50E94B139882311F40C94C676B6
:1014F0000E9435390C945C7D0E94DF5984EC94E1A4
:101500000E9451430C94C676882309F4B0CF0C9402
:101510006A77DF92EF92FF920F931F93CF93DF933F
:10152000EC01E090BF08F090C0088AE0D82E6AE095
:1015300070E0CE010F94C6748C01009711F0FC018D
:101540001082CE010E949C3281E00E94F17401154C
:10155000110519F0E801D992EACFC701DF91CF91C7
:101560001F910F91FF90EF90DF900C949C324F925F
:101570005F926F927F928F929F92AF92BF92CF9223
:10158000DF92EF92FF920F931F93CF93DF93CDB72C
:10159000DEB77C014DB65EB66090BF087090C008A3
:1015A0008DB69EB66AE070E0C7010F94BA696C010F
:1015B0008C010E191F09892B21F4C7010F94CC69E6
:1015C0008C01C80101962DB73EB7281B390B0FB609
:1015D000F8943EBF0FBE2DBF8DB79EB701965C013C
:1015E000A801B7010F94ED69F501E00FF11F10821A
:1015F000C5010E949C3281E00E94F174C114D104A3
:1016000051F076019FEFE91AF90A0FB6F8949EBEE1
:101610000FBE8DBEC5CF0FB6F8949EBE0FBE8DBE59
:10162000C3010E949C320FB6F8945EBE0FBE4DBE41
:10163000DF91CF911F910F91FF90EF90DF90CF90AE
:10164000BF90AF909F908F907F906F905F904F90E2
:1016500008954F925F926F927F928F929F92AF9276
:10166000BF92CF92DF92EF92FF920F931F93CF938F
:10167000DF93CDB7DEB7C059D1090FB6F894DEBFFE
:101680000FBECDBF0E94BC3B882369F083E50E945A
:101690006339882301F120E040E070E060E089E8F0
:1016A0009BE90E947099C057DF4F0FB6F894DEBFD8
:1016B0000FBECDBFDF91CF911F910F91FF90EF90A3
:1016C000DF90CF90BF90AF909F908F907F906F9062
:1016D0005F904F90089583E40E946339882319F046
:1016E0000E947E9BE0CF8090B6099090B709A090B1
:1016F000B809B090B9098091BF0980FF05C09091E9
:1017000021109860909321108695817080931D0A16
:101710008EE191E10E94B78A809145099091460936
:101720009E012F5F3F4F7901009799F09F938F9310
:1017300085E191E19F938F933F932F930F94166AC6
:10174000C7010E94898A0F900F900F900F900F9001
:101750000F908091430990914409009799F09F93CD
:101760008F938CE091E19F938F93FF92EF920F9470
:10177000166AC7010E94898A0F900F900F900F90F0
:101780000F900F906E0131E8C30ED11C60912209B9
:10179000709123098091240990912509860123E005
:1017A00041E00F944C659F938F938AEF90E19F9354
:1017B0008F93FF92EF920F94166AC7010E94898A55
:1017C00082EF90E10E94B78A87E08093B10880930E
:1017D00004060F900F900F900F900F900F90809134
:1017E0003E098823F9F060913F097091400980918A
:1017F00041099091420923E041E00F944C659F9389
:101800008F9389EE90E19F938F93FF92EF920F94C5
:10181000166AC7010E94898A0F900F900F900F904F
:101820000F900F90809147098823A1F01F928F930A
:101830001F921F928CED90E19F938F93FF92EF92F6
:101840000F94166AC7010E94898A0FB6F894DEBF0A
:101850000FBECDBF809148098823A9F01F928F93B6
:101860001F9281E08F938CED90E19F938F93FF9275
:10187000EF920F94166AC7010E94898A0FB6F894F6
:10188000DEBF0FBECDBF4090490950904A0960901D
:101890004B0970904C0920E030E0A901C301B2016E
:1018A0000F947F6A811104C08091BF0982FF20C01C
:1018B000860121E041E0C301B2010F944C659F9382
:1018C0008F938091BF0982FB882780F91F928F93A5
:1018D0008FEC90E19F938F93FF92EF920F94166A93
:1018E000C7010E94898A0FB6F894DEBF0FBECDBF34
:1018F000609114097091150980911609909117094A
:101900008E010F581F4F23E041E00F944C65782E55
:10191000692E6091100970911109809112099091BE
:101920001309860123E041E00F944C656F927F928A
:101930009F938F938EEB90E19F938F93FF92EF9203
:101940000F94166AC7010E94898A609118097091E4
:10195000190980911A0990911B0923E041E00F9425
:101960004C6583EB90E10E94B78ADF92CF9289EABF
:1019700090E19F938F93FF92EF920F94166AC701A5
:101980000E94898A809121098F93809120098F93E9
:1019900082EA90E19F938F93FF92EF920F94166AE1
:1019A000C7010E94898A60911C0970911D0980916C
:1019B0001E0990911F0923E041E00F944C659F930D
:1019C0008F9388E990E19F938F93FF92EF920F940A
:1019D000166AC7010E94898A8CE0E6E2F9E0A3E07A
:1019E000B9E001900D928A95E1F78CE0E2E3F9E02D
:1019F000A7EFB8E001900D928A95E1F780E00F948F
:101A0000F20581E00F94F20582E00F94F2058091D7
:101A1000BE098093D70881E0809319060E94AE3BEF
:101A20008DE499E09F938F938AE39DE39F938F9337
:101A3000FF92EF920F94166A0FB6F894DEBF0FBEB6
:101A4000CDBFC7010E94898A8091BD098F93809183
:101A5000BC098F938091BB098F938091BA098F93B2
:101A6000BF92AF929F928F928AE890E19F938F935B
:101A7000FF92EF920F94166AC7010E94898A0FB6EF
:101A8000F894DEBF0FBECDBF0ECECF93DF93C091D3
:101A90005811C093E20981E6C89FE0011124C65A9B
:101AA000DE4E8091211080FF05C00E94E359CE01D7
:101AB0000E941F43CE010E949C3280E0DF91CF91B3
:101AC0000C94F17460913D0270913E02072E000C5F
:101AD000880B990B0F94866A2AE037ED43E25CE3AA
:101AE0000F94E56A2091050630910606409107069D
:101AF000509108060F94E56A609385027093860200
:101B000080938702909388020895E0919C08E230C8
:101B100030F4F0E0E55FF54F80918A088083089506
:101B2000809195168823C1F0815080939516E1EC41
:101B3000F6E1882351F08150990B2BE1289FF001A9
:101B4000299FF00D1124E950F94E8BE1ACEDB6E17F
:101B500001900D928A95E1F720919516211105C00B
:101B60008091A01680628093A01681E090E0A0E0B2
:101B7000B0E0211103C080E090E0DC018093820896
:101B800090938308A0938408B093850810928708E7
:101B900081E08093810883E0809384020895CF934D
:101BA000DF93EC01CB01BA010F94866A29EC38EC83
:101BB00048EC5EE30F946B7220E030E040E05FE3BE
:101BC0000F9471710F94E4726883DF91CF9108953F
:101BD000E0919C0886E0E802F0011124E359F74FF8
:101BE00080918A0890E09583848308958F929F92D4
:101BF000AF92BF92CF92DF92EF92FF92CF936B01A1
:101C00007C0120E030E0A9010F947F6A87FD9FC02E
